:100000000C945E070C948F070C948F070C948F0749
:100010000C948F070C948F070C948F070C948F0708
:100020000C948F070C948F070C948F070C948F07F8
:100030000C948F070C94CA7D0C948F070C948F0737
:100040000C948F070C94C57B0C948F070C948F072E
:100050000C948F070C948F070C948F070C94F17AF3
:100060000C948F070C94D8770C94AE770C948F0770
:100070000C948F070C948F070C948F070C948F07A8
:100080000C94977B0C948F070C948F070C948F071C
:100090000C948F070C948F070C948F070C9441805D
:1000A0000C948F070C948F070C94697B0C948F072A
:1000B0000C948F070C948F070C948F070C943B7B48
:1000C0000C948F070C948F070C948F070C948F0758
:1000D0000C948F070C948F070C9478770C944E77C0
:1000E0000C948F070C944A6F0C94B86D0C94967610
:1000F0000C94F8880C94AC6F0C941A8D0C94256FAA
:100100000C94070D0C9401080C94196F0C94A86EB4
:100110000C9427080C9491070C94386F0C94D66FAC
:100120000C94136F0C9424080C94D10C0C94AD6FA8
:100130000C94D8070C94FF0A0C94B96D0C94BC6F06
:100140000C946A0A0C94216F0C9422080C948C195C
:100150000C94D9890C9459120C94B9070C94161369
:100160000C9403700C94ED110C94F8940C94020808
:100170000C942B8D0C94F76D0C945B6E0C941808FA
:100180000C94466F0C94586F0C940B6E0C94F27F89
:100190000C94AE0C0C9402890C94536F0C941F14A5
:1001A0000C94D1070C94290B0C942E6F0C94286F8F
:1001B0000C944E6F0C94F5130C94406F0C94687073
:1001C0000C94F90F0C94196E0C94D75D0C94BD0728
:1001D0000C948A130C94EE070C94790C0C94270A57
:1001E0000C94BB6D0C940F0A0C947F0B0C945495DB
:1001F0000C94E1190C94C1070C9432700C946C109F
:100200000C94E00A0C94F9070C94E70B0C941D6F06
:100210000C9452700C94326F0C94CF6F0C94A30713
:100220000C947B0B0C94E86D0C94BA6D0C946F6479
:100230000C943C6F0C94580C0C94390D0C94546F26
:100240000C943E144E414E494E495459494E46CDA8
:10025000CCCC3D0AD7233C17B7D13877CC2B32957D
:1002600095E6241FB14F0A000020410000C842005B
:10027000401C4620BCBE4CCA1B0E5AAEC59D740025
:10028000407A10F35A00A0724E18090010A5D4E865
:100290000000E87648170000E40B54020000CA9AF8
:1002A0003B000000E1F5050000809698000000404A
:1002B000420F000000A0860100000010270000008F
:1002C00000E803000000006400000000000A0000D5
:1002D0000000000100000000002C76D888DC674F89
:1002E0000823DFC1DFAE59E1B1B796E5E3E453C6B9
:1002F0003AE651997696E8E6C28426EB898C9B62B1
:10030000ED407C6FFCEFBC9C9F40F2BAA56FA5F45A
:1003100090055A2AF75C936B6CF9676DC11BFCE082
:10032000E40D47FEF520E6B500D0ED902E030094D5
:100330003577050080841E080000204E0A0000006A
:10034000C80C333333330F986E12831141EF8D2174
:1003500014893BE65516CFFEE6DB18D1844B381BDB
:10036000F77C1D901DA4BBE424203284725E2281A0
:1003700000C9F124ECA1E53D27436F6E74656E74EE
:100380002D547970653A20746578742F68746D6C9B
:100390000D0A0D0A3C68313E45504943204641490B
:1003A0004C3C2F68313E00485454502F312E3020A1
:1003B0003430302042616420526571756573740D6C
:1003C0000A004163636573732D436F6E74726F6CC3
:1003D0002D416C6C6F772D4F726967696E3A202AD8
:1003E0000D0A436F6E74656E742D547970653A20F2
:1003F000005365727665723A205765626475696E5E
:100400006F2F312E370D0A00485454502F312E30A3
:1004100020323030204F4B0D0A00436F6E6E656303
:1004200074696F6E3A20636C6F73650D0A436F6E6B
:1004300074656E742D547970653A206170706C69C2
:10044000636174696F6E2F782D7777772D666F7281
:100450006D2D75726C656E636F64656400506F73AB
:1004600074206661696C65640055706C6F6164200E
:100470004661696C65643A2000234E6F2073656E97
:10048000736F7220666F722074656D70202620680D
:10049000756D696469747921004E6F2053656E73C0
:1004A0006F72210020666F722074656D70202620A7
:1004B00068756D696469747921002353656E736F83
:1004C00072204572726F72200053656E736F7220D6
:1004D0004572726F7221002357726F6E67207365C9
:1004E0006E736F7220666F722074656D70202620A7
:1004F00068756D6964697479210057726F6E672041
:1005000053656E736F7221004320483D00543D00D7
:1005100020202020202020202020202020202020DB
:1005200000202020202020202020202020202020EB
:1005300020002020202020202020202020202020DB
:1005400020200020202020202020202020202020CB
:1005500020200020202020202020202020202020BB
:1005600020200054696D657374616D702075706C26
:100570006F6164206661696C6564005365747469B9
:100580006E6720636C6F636B2074696D6500236513
:1005900072726F72202D2000495020616464726570
:1005A00073733A2000416E676C654000496E766156
:1005B0006C696420534D207374657073207065728C
:1005C00020616E676C653D00534D207374657073D8
:1005D0002070657220616E676C653D003C703E5412
:1005E000696D653A20003C2F68333E0A003C627218
:1005F0003E4254206E616D653D003C62723E50612A
:1006000074683D003C68333E53797374656D3A20DD
:1006100056657273696F6E3D00506172616D6574ED
:1006200065727320726573657420646F6E65210056
:100630002F6F652F736D6C69676874706F2F7333DC
:100640002F00616E676C6520646972656374696F01
:100650006E3A200043757272656E7420534D2069A6
:1006600073202300534D3A5461626C6520737465A6
:1006700070732070657220616E676C653D00534D2C
:100680003A506F6C6172697A657220737465707329
:100690002070657220616E676C653D00234448548C
:1006A00050494E3D00234448543D00236E65743D3F
:1006B000424C4500236E65743D5769466900236EC0
:1006C00065743D4254002366747020757365726EC4
:1006D000616D653A003A0023486F73742073657248
:1006E00076657220495020616E6420506F72743AB2
:1006F000002354696D6520736572766572204950D8
:100700003A002352656C617920646576696365738C
:100710003A002352656C617920737461747573209B
:100720006C6162656C733A20002352656C617920BC
:100730007374617465733A002352656C617920703B
:10074000696E733A00234E6F2E206F6620636F6EC2
:1007500074726F6C2072656C6179733D00234E6F0B
:100760002E206F662072656C6179733D00234C6F9B
:1007700067676572204E616D653A200046696E6458
:10078000696E672057694669204950004E45543DBF
:10079000426C7565746F6F7468204C45004E45540B
:1007A0003D426C7565746F6F7468004E45543D57DB
:1007B000694669005344206F70656E206661696CFC
:1007C000004E6577206461746120636F6C6C6563B3
:1007D00074696F6E2073746172746564004375721E
:1007E00072656E742073657474696E67733A005332
:1007F000797374656D20726573657420617420006F
:1008000023445320546865726D6F6D657465722062
:1008100063616C6962726174656420666F72202323
:1008200000496E76616C696420616E676C65206654
:100830006F72200020737465707320706572206180
:100840006E676C653D00207374657073207065720F
:1008500020616E676C653D005461626C6520536574
:1008600074203000235475726E7461626C6520537D
:100870006574203000506F6C6172697A6572205324
:10088000657420300023506F6C6172697A65722044
:100890005365742030005461626C65205365742088
:1008A0003000235475726E7461626C6520536574F8
:1008B000203000506F6C6172697A657220536574E4
:1008C00020300023506F6C6172697A657220536525
:1008D00074203000576946692049503A00234C6F14
:1008E00067676572204E616D653A20004C4F47473F
:1008F00045520056455253494F4E005265626F6F44
:1009000074696E672E2E2E005245424F4F5400538D
:10091000657276657220506F7274207570646174B0
:1009200065640053504F52543D0049502075706427
:1009300061746564005349503D002354696D65201E
:1009400053657276657220495020757064617465D4
:100950006400545349503D004352454C41590044B2
:10096000485450494E3D0074696D6520696E746548
:100970007276616C3D0054494D455354414D503D94
:100980000054494D455354414D50002377656273DF
:10099000657276657220626567696E73005365746F
:1009A00074696E672049500053657474696E6720DE
:1009B000446576696365204950202E2E2E00506FC5
:1009C0006C6172697A65722053657420300023501F
:1009D0006F6C6172697A65722053657420300054BF
:1009E000657374204C616D70732F46616E73006582
:1009F00072726F72206F70656E696E672066696CC7
:100A0000653A20004C616D70204D6F746F72002349
:100A100054696D65202020202020446174652020C9
:100A20002020205365636F6E647320506F6C617279
:100A3000697A6572205461626C652054286F43297D
:100A40002048282529202000696E69742E20646FB3
:100A50006E652E00534420696E69742E20666169AC
:100A60006C65642100696E69742E206661696C652D
:100A70006421002323204F452057656C636F6D650B
:100A800020232300496E697469616C697A696E6715
:100A900020534420636172642E2E2E0075706C6F9B
:100AA000616420627920465450206661696C6564F7
:100AB000210075706C6F616420627920465450206B
:100AC0004F4B210053797374656D20737461727498
:100AD000696E672E2E2E003C703E4C616D70206159
:100AE0006E64204D6F746F72204472697665727304
:100AF00020537461747573EFBC9A3C2F703E003CB8
:100B000021646F63747970652068746D6C3E3C6815
:100B1000746D6C3E3C686561643E3C6D657461203B
:100B2000636861727365743D227574662D38223E68
:100B30003C7469746C653E4F6E6C696E65206578B7
:100B4000706572696D656E74202D20506F6C6172D6
:100B5000697A6174696F6E20656666656374732077
:100B60006F66206C696768743C2F7469746C653EAD
:100B70003C2F686561643E3C626F64793E3C68313D
:100B80003E4F6E6C696E65206578706572696D6543
:100B90006E74202D20506F6C6172697A6174696F78
:100BA0006E2065666665637473206F66206C696786
:100BB00068743C2F68313E003C68343E436F707966
:100BC0007269676874284329323032302D323032EE
:100BD000322E50726F662E205945554E472059616E
:100BE00075205975656E3C2F68343E3C2F626F64EA
:100BF000793E3C2F68746D6C3E003C68313E436129
:100C00006E6E6F74206765742073656E736F7220EB
:100C100072656164696E6773213C2F68313E007CA8
:100C20003C3E5E2B3D3F2F5B5D3B2C2A225C00004F
:100C3000002100240027002A002D0030003300018D
:100C4000010000040107010A01000022002500281C
:100C5000002B002E003100340002010000050108C5
:100C6000010B01000020002300260029002C002F8A
:100C7000003200000100000301060109010505051D
:100C800005070508080808020202020A0A08080403
:100C90000404040101010101010101030303030331
:100CA000030303040707070C0C0C0C0C0C0C0C02C0
:100CB00002020206060606060606060B0B0B0B0BC7
:100CC0000B0B0B01021020200808102040102040C0
:100CD0008002010201080402010102040810204000
:100CE000808040201008040201800402018040201E
:100CF0001008040201080402010102040810204047
:100D000080010204081020408000000A0B02090C38
:100D10000D0E0807030401000000000000000000A1
:100D200000000000000000000000000000000000C3
:100D30000000000000121110000000000000000080
:100D40000000000000000000000000000000005350
:100D5000797374656D207265737461727465642152
:100D6000002053797374656D2072657374617274B9
:100D7000656421004E6574776F726B206D61696EDA
:100D80007461696E656420617420002323436F6D74
:100D90006D616E644000417070656E64206D6561C8
:100DA000732E200053696E676C65206D6561732E2C
:100DB000200053617665206D6561737572652074DE
:100DC0006F3A0020202020202020202020202020DA
:100DD000202020000000010001001010020001008E
:100DE0000100B00000001600000028000000100004
:100DF00000002000000001000100000000000000D1
:100E000000000000000000000000000000000000E2
:100E1000000000000000FF000000FFFF0000FFFFD7
:100E20000000FFFF0000CFBF0000C7BF0000C3BF2E
:100E30000000C1BF0000C0BF000000000000C0BF34
:100E40000000C1BF0000C3BF0000C7BF0000CFBF8C
:100E50000000FFFF0000FFFF000000000000000096
:100E60000000000000000000000000000000000082
:100E70000000000000000000000000000000000072
:100E80000000000000000000000000000000000062
:100E900000000000000000000000557365722D6125
:100EA00067656E743A202A0D0A446973616C6C6F31
:100EB000773A202F0D0A00005495F89411241FBE94
:100EC000CFEFD1E2DEBFCDBF00E00CBF1AE0A0E063
:100ED000B2E0ECE1F3E601E00BBF02C007900D9237
:100EE000AA31B107D9F725E1AAE1BAE001C01D9204
:100EF000A43FB207E1F717E0CDE5D7E000E006C078
:100F000021970109802FFE010E9495AECC35D107B3
:100F100080E00807A9F70E94E6980C947CB10C9435
:100F20000000CF93DF93EC01898D9A8D892B41F0DE
:100F3000E881F9810284F385E02DCE011995F4CF83
:100F4000DF91CF910895CF93DF931F92CDB7DEB796
:100F50006983DC01ED91FC910280F381E02D41E099
:100F600050E0BE016F5F7F4F19950F90DF91CF91D9
:100F70000895FC01818D928D0895FC0184899589E5
:100F8000089527E134E0FC0131832083FB0140898F
:100F9000518962897389FC01428353836483758319
:100FA0000895DC01ED91FC91048CF58DE02D1994F0
:100FB000CF93DF931F92CDB7DEB76983DC01ED914C
:100FC000FC910280F381E02D41E050E0BE016F5FB3
:100FD0007F4F19950F90DF91CF910895FC01948573
:100FE000FB018485981303C081E0943009F480E00C
:100FF000089521E0FC018485843009F420E0822FEB
:1010000008950895CF93DF931F92CDB7DEB769831C
:10101000DC01ED91FC910280F381E02D41E050E094
:10102000BE016F5F7F4F19950F90DF91CF910895AB
:10103000DC01ED91FC91068CF78DE02D199591E086
:1010400089270895862F089581E08627089590E0E6
:1010500080E0089590E0982F882744E050E0845F76
:101060009B4F0C949790EF92FF920F931F93CF9307
:10107000DF93182FC6EFDBE061E08A810E942B79B5
:101080006091B50B8A810E940E7864EF71E080E078
:1010900090E00E94817922968BE0CC3FD80761F7DF
:1010A000112309F44AC008EF1BE0E8017E016091BA
:1010B000B70B88810E940E7868EE73E080E090E0C4
:1010C0000E9481796091B70B8A810E940E7868EE48
:1010D00073E080E090E00E94817922966091B50BE8
:1010E000D7018C910E940E7868EE73E080E090E06A
:1010F0000E948179BBE0CC3FDB07C1F668EE73E06C
:1011000080E090E00E948179C1EDD2E0E991F9910F
:10111000D8018C910E5F1F4FEE0FFF1FEB54F44F61
:1011200060810E940E7868EC70E080E090E00E94A0
:101130008179B2E0C73DDB0749F7DF91CF911F917D
:101140000F91FF90EF9008959F92AF92BF92CF9230
:10115000DF92EF92FF920F931F93CF93DF935C0187
:101160007B018B01D0E0C0E0F80191908F01650117
:10117000CC0EDD1EC6010E94CDAC981621F0692D63
:10118000C6010E94D5AC2196C233F1E0DF0761F7BA
:10119000C701DF91CF911F910F91FF90EF90DF90EA
:1011A000CF90BF90AF909F90089581E08093EF0221
:1011B0008091F002882341F088E08093FA1160E08A
:1011C0008FEE91E10C94877F08958091F00288233F
:1011D000F9F08091EF028823D9F081E00E94B47F7A
:1011E0008BE39FE10197F1F760E080E00E94C57F0B
:1011F00063E575E08FEE91E10E941E7761E080E08B
:101200000E94C57F63E475E08FEE91E10C941E7738
:1012100008950F931F93CF93DF932091F002222321
:1012200009F45CC02091EF02222309F457C0EA01BF
:101230008C016F3F7F4FF1F461E080E00E94C57F39
:10124000B8018FEE91E10E94FC7662E375E08FEECB
:1012500091E10E941E7761E0F80184810E94C57FC0
:10126000BE01DD0F880B990BDF91CF911F910F917C
:101270000C9481790E943F7AAB01BC018091E70A0E
:101280009091E80AA091E90AB091EA0A8C599F4F1F
:10129000AF4FBF4F84179507A607B707F8F461E073
:1012A00080E00E94C57FB8018FEE91E10E94FC763C
:1012B00061E275E08FEE91E10E941E7761E0F80136
:1012C00084810E94C57F0E943F7A6093E70A7093F1
:1012D000E80A8093E90A9093EA0AC2CFDF91CF919E
:1012E0001F910F9108952C9A08952C9808958EBD02
:1012F00000000DB407FEFDCF8EB508959B0190E070
:101300000496982F8827642F820F931F0C94419284
:10131000CF93DF93C82FD62F472F60E170E00E9454
:101320007E094D2F61E170E08C2FDF91CF910C94FD
:101330007E09CF93DF93C82FD0E02496DC2FCC27F3
:10134000C60FD71F0E9475098FE00E9477098D2F65
:101350000E9477098C2F0E94770980E00E9477090C
:10136000C82F0E9473098C2FDF91CF9108951F938E
:10137000CF93DF93182F66E270E00E949909C82F7F
:1013800067E270E0812F0E9499099C2FDF91CF9135
:101390001F9108951F93CF93DF93182F60E270E0A1
:1013A0000E949909C82F61E270E0812F0E9499097B
:1013B0009C2FDF91CF911F91089544E050E0BC0134
:1013C0008FE090E00C94979008958CBD9DBD08959A
:1013D000EF92FF920F931F93CF93C82F7B0180E56D
:1013E00090E00E94E50968E270E08C2F0E94990964
:1013F000082F69E270E08C2F0E949909282F302F66
:10140000B90121E030E0A7018C2F0E94AD7281E08C
:1014100090E0CF911F910F91FF90EF900895CF939F
:10142000DF931F92CDB7DEB7FC01218D328D8FEF98
:101430009FEF232B41F0BE016F5F7F4F808D0E9495
:10144000E809898190E00F90DF91CF9108950F9383
:101450001F93CF93DF931F92CDB7DEB78C01DC01D2
:10146000ED91FC910084F185E02D1995892B79F09F
:10147000BE016F5F7F4FF80184850E94E809898172
:1014800090E00F90DF91CF911F910F9108958FEF12
:101490009FEFF7CFFF920F931F93CF93DF93F82E19
:1014A00080E590E00E94E50910E000E08F2D0E94A9
:1014B000B709EC01892B21F08F2D0E94B7098C010F
:1014C000C017D10799F7CE01DF91CF911F910F91EE
:1014D000FF900895FC018485843011F00C944A0A31
:1014E00090E080E00895AF92BF92CF92DF92EF92AA
:1014F000FF921F93CF93DF93182F6B017A0180E542
:1015000090E00E94E509B12CA12C812F0E94B7091F
:10151000EC01892B21F0812F0E94B7095C01CA15CB
:10152000DB0599F72097E9F463E070E0812F0E94D2
:101530009909843159F0882349F0C1E0D0E08C3119
:1015400011F4D0E0C0E0D195C195D109CE01DF9171
:10155000CF911F91FF90EF90DF90CF90BF90AF9011
:101560000895EC16FD060CF4E7011C161D0674F731
:1015700068E270E0812F0E949909E82E69E270E02C
:10158000812F0E949909282F3E2D79019E01A601E5
:10159000B701812F0E94AD72EC0EFD1E4F2D68E247
:1015A00070E0812F0E947E094E2D69E270E0812F4C
:1015B0000E947E0960E470E0812F0E948172C6CF94
:1015C000CF93DF93FC01218D328D2115310529F454
:1015D0008FEF9FEFDF91CF910895EC01808D42173F
:1015E000530708F0A9010E94730A1816190684F718
:1015F000298D3A8D281B390B3A8F298FEBCF0F930A
:101600001F93CF93DF931F92CDB7DEB7FC01218DDF
:10161000328D232B41F48FEF9FEF0F90DF91CF910D
:101620001F910F9108958C0141E050E0BE016F5F62
:101630007F4FFC01808D0E94730A181619065CF713
:10164000F801818D928D0197928F818F898190E031
:10165000E4CF0F931F93CF93DF9300D000D01F925E
:101660001F92CDB7DEB78C01DC01ED91FC910680B5
:10167000F781E02D1995F801808D0E944A0A18160D
:101680001906B4F548E050E0BE016F5F7F4FD80106
:1016900058968C910E94730A18161906F4F4D80112
:1016A000509684E0FE01319601900D928A95E1F703
:1016B0008D8190E0982F88272E81820F911DF8014F
:1016C000958B848B8F81282F30E0322F22278885BD
:1016D000820F932F911D928F818F28960FB6F894C9
:1016E000DEBF0FBECDBFDF91CF911F910F91089547
:1016F00090E080E0F2CFFC0184850C94730ACF93D4
:10170000DF931F92CDB7DEB741E050E0BE016F5FBF
:101710007F4FFC0184850E94730A1816190634F461
:10172000898190E00F90DF91CF9108958FEF9FEF27
:10173000F9CFCF93C82F80E590E00E94E50960E1E2
:1017400070E08C2F0E9481724FEF62E070E08C2F6E
:10175000CF910C947E09FF920F931F93CF93DF9349
:10176000C82FD62F8A01F22E0E94990B80E590E0B7
:101770000E94E5094D2F4F2970E060E08C2F0E94F8
:101780007E0901151105C1F0412F64E070E08C2F36
:101790000E947E09402F65E070E08C2F0E947E0938
:1017A00061E070E08C2F0E94817281E0DF91CF9127
:1017B0001F910F91FF9008950091FF0B1091000C65
:1017C0000F5F1F4F1093000C0093FF0BDDCFBF92F4
:1017D000CF92DF92EF92FF920F931F93CF93DF93FD
:1017E00000D000D0CDB7DEB7FC01208D243009F049
:1017F0005DC06A017B018C01B12C63E070E08B2D30
:101800000E94990981114AC0F801B08EF801808DBB
:10181000843009F44BC096E0EBEFF2E0DE01119664
:1018200001900D929A95E1F7F70193819F779C8340
:1018300094819D8395819E83B7016E5F7F4F0E9447
:101840002A08B601F801808D0E948809F801808D70
:1018500090E0982F882746E050E0BE016F5F7F4FF1
:101860008A5F9B4F0E949790F801128E118E20E89C
:10187000A60162E0808D0E94AB0B81E026960FB638
:10188000F894DEBF0FBECDBFDF91CF911F910F91B6
:10189000FF90EF90DF90CF90BF900895883109F4CA
:1018A000B3CFB394F4E0BF12A8CFB0CF80E0E6CFBF
:1018B000CF93DF93EC01888D843061F00E94990B07
:1018C000E88DF0E0EE0FFF1FE65DF34F118210820E
:1018D00084E0888FDF91CF910895CF93C82F80E562
:1018E00090E00E94E50963E070E08C2FCF910C94AA
:1018F0009909EF92FF921F93CF93DF93FC01208D04
:10190000243039F080E0DF91CF911F91FF90EF906C
:1019100008957B01EC0110E0812F0E946D0C811174
:101920000FC0188F888D843069F3FD86EC861A8E7F
:10193000198E20E0A70162E00E94AB0B81E0E3CFAB
:10194000883179F31F5F143039F7ECCFFC018485BF
:10195000843011F00C946D0C80E00895CF93DF93E8
:10196000FC0124852430D9F0EC010E94A60C8431BE
:1019700089F0882379F0883169F021E08C3159F4BD
:10198000E881F9810084F185E02DCE01199521E0EF
:10199000892B09F420E0822FDF91CF91089580E018
:1019A000FBCFAF92BF92CF92DF92FF920F931F9324
:1019B000CF93DF938C015B01EA01FC01C688D788D5
:1019C000F08C80E590E00E94E5098F2D0E949172D5
:1019D0008C179D0720F48F2D0E949172EC019E01BF
:1019E000A501B6018F2D0E94C690F80186899789BE
:1019F0008C0F9D1F978B868BCE01DF91CF911F910E
:101A00000F91FF90DF90CF90BF90AF900895CF934C
:101A1000FC01C08D80E590E00E94E50960E270E085
:101A20008C2F0E94817262E070E08C2F0E949909D5
:101A300084FD16C062E070E08C2F0E94990983FF3C
:101A40000AC048E162E070E08C2F0E947E0990E0BD
:101A500080E0CF91089580E590E00E94E509E3CF12
:101A600040E162E070E08C2F0E947E0981E090E00E
:101A7000F0CFFF920F931F93CF93DF93EB01FC0105
:101A8000178A168A2A81211109C02B81211106C0CB
:101A90002C81211103C02D812223E1F04115510534
:101AA000C9F08A01FC01F08C80E590E00E94E50914
:101AB000BE016E5F7F4F8F2D0E942A08B8018F2DC7
:101AC0000E94880981E090E0DF91CF911F910F91F2
:101AD000FF90089590E080E0F7CF4F925F926F9271
:101AE0007F928F929F92AF92BF92CF92DF92EF92AE
:101AF000FF920F931F93CF93DF93CDB7DEB763971A
:101B00000FB6F894DEBF0FBECDBF7C016B013A016A
:101B1000FB0120E090E080E06AE03191332309F49A
:101B200061C040ED430F4A3008F04DC0689FA001EE
:101B3000699F500D1124CA01C097830F911D37FD75
:101B40009A958F3F910549F340F3F7014281538104
:101B50006481758180913A0E90913B0EA0913C0E6C
:101B6000B0913D0E481759076A077B0709F439C23F
:101B70008701085F1F4F0E943F7A6F7077277C5F55
:101B8000C8010E94790C813009F030C287E194E0ED
:101B90009A838983F70182819381A481B5818B83A4
:101BA0009C83AD83BE8345E350E0BE016F5F7F4FF2
:101BB000C8010E94390D892BA9F5D12CC12CC8016F
:101BC0000E94580C17C03E3209F0BFCF233009F4F1
:101BD000BCCFD301A20FB11D12968C932F5F90E062
:101BE00080E09BCF233009F0B0CFF3018583CC2474
:101BF000C394D12CC60163960FB6F894DEBF0FBE16
:101C0000CDBFDF91CF911F910F91FF90EF90DF90AB
:101C1000CF90BF90AF909F908F907F906F905F908C
:101C20004F9008950E943F7AF70177836683762765
:101C3000672776277A83698342E050E0BE016F5FB1
:101C40007F4FC8010E94D10C81E090E09E878D8774
:101C500042E050E0BE01635F7F4FC8010E94D10C9B
:101C600080E091E09E878D8742E050E0BE01635F97
:101C70007F4FC8010E94D10C1E861D8642E050E0B5
:101C8000BE01635F7F4FC8010E94D10C42E050E06B
:101C9000BE01635F7F4FC8010E94D10C42E050E05B
:101CA000BE01635F7F4FC8010E94D10C5601F6014F
:101CB0008081882301F16501F60181912F0188233C
:101CC00011F08E32B1F446018A189B0818141904D9
:101CD00074F48F8641E050E0BE01615F7F4FC80120
:101CE0000E94D10CA401B501C8010E94D10C52017F
:101CF000DECF6201E1CF1F8641E050E0BE01615FAF
:101D00007F4FC8010E94D10CC12CDD24D394DE8604
:101D1000CD8642E050E0BE01635F7F4FC8010E9464
:101D2000D10CDE86CD8642E050E0BE01635F7F4F7E
:101D3000C8010E94D10CC8010E94070D892B09F42B
:101D40003CCFF3E0AF2EB12C230122E0420E511C18
:101D50005EC0F7014281538164817581808D918DD0
:101D6000A28DB38D481759076A077B0709F02FC169
:101D7000848D958DC59709F02AC181A192A10C97F8
:101D80000CF42AC14CE050E0BE016F5F7F4FC801E8
:101D90000E94E00A8B819C819827892798279A8B3B
:101DA000898B29813A81322723273227F7014681FF
:101DB000578142175307D1F497FF18C08F70927064
:101DC000892B09F042C06F807884762467247624BA
:101DD000D12CC12C6114710409F051C0C8010E94BA
:101DE00091076AEFC62EDD24DA9407C0C8010E946D
:101DF0009107ECEFCE2EDD24DA9481E0A81AB10829
:101E000009F4DDCEFFEFCF16DF0609F0D8CE0E9431
:101E10003F7A3B014C01C8010E94290B1816190694
:101E20000CF497CF0E943F7A6619770988099909BF
:101E3000693873418105910508F0C5C062E370E01F
:101E400080E090E00E948179E6CFC8010E9491076E
:101E50007BEFC72EDD24DA94D0CF8D85811117C09A
:101E6000C8010E94FF0AC8010E94FF0AC8010E941F
:101E7000FF0AC8010E94FF0AFFEFCF1ADF0A8D8117
:101E80009E81982789279827C816D906A8F441E08B
:101E900050E0BE01635F7F4FC8010E94E00A8D855C
:101EA0008823D9F28D859FEF980F9D878823A9F20B
:101EB000C8010E94FF0AF6CF912C812C41E050E02E
:101EC000BE016D5E7F4FC8010E94E00A8B89982F8A
:101ED000907C61F4882389F08B899FEF980F9B8B0E
:101EE000882341F0C8010E94FF0AF6CFC8010E9472
:101EF000FF0A1B8A8B898111E1CF42E050E0BE01CD
:101F0000615F7F4FC8010E94E00A42E050E0BE01DD
:101F1000635F7F4FC8010E94E00AC8010E94FF0A68
:101F2000C8010E94FF0AC8010E94FF0AC8010E945E
:101F3000FF0A42E050E0BE016F5E7F4FC8010E9481
:101F4000E00A8F85988981159140E9F4CD84DE847B
:101F5000DC24CD24DC2481E0C816D104A1F48989D5
:101F60009A898115944041F0C8010E94910757EF6A
:101F7000C52EDD24DA9441CF44E050E0B201C8011F
:101F80000E94E00A3ACFD12CC12C89899A899827DE
:101F900089279827C816D90638F4C8010E94FF0A75
:101FA000FFEFCF1ADF0AF1CF2FEF821A920A6814DF
:101FB000790409F083CFC8010E94910746EFC42E2F
:101FC000DD24DA941ACFCC24CA94DC2C16CF2EEF61
:101FD000C22EDD24DA9411CF9DEFC92EDD24DA94D0
:101FE0000CCF8EEFC82EDD24DA9404CED12CC12C78
:101FF00001CECF92DF92EF92FF920F931F93CF9378
:10200000DF93CDB7DEB7AF970FB6F894DEBF0FBE44
:10201000CDBF7C016A0107E114E01A8309831C86A5
:102020001B8688EE93E0A0E0B0E08D879E87AF87A7
:10203000B88B8BEA93E09A878987188F0F8B198E5C
:102040001A8E1B8E1C8E84E089A31BA70AA71CA6D0
:102050001DA61EA61FA68091320E9091330EA09150
:10206000340EB091350E8EA39FA3A8A7B9A78B837A
:102070009C83AD83BE8318861F82AE01465D5F4F91
:10208000CE0101960E946D0D81309105B1F4D7010A
:10209000ED91FC910488F589E02D1DA30CA38CA57E
:1020A0009DA5AEA5BFA58EA39FA3A8A7B9A7A6016E
:1020B000BE016C5D7F4FC7011995AF960FB6F894BE
:1020C000DEBF0FBECDBFDF91CF911F910F91FF906B
:1020D000EF90DF90CF900895CF92DF92EF92FF9232
:1020E0000F931F93CF93DF93CDB7DEB7AF970FB6A4
:1020F000F894DEBF0FBECDBF7C016A0107E114E09A
:102100001A8309831C861B8688EE93E0A0E0B0E06A
:102110008D879E87AF87B88B8BEA93E09A878987F4
:10212000188F0F8B198E1A8E1B8E1C8E84E089A33C
:102130001BA70AA71CA61DA61EA61FA68091320ECD
:102140009091330EA091340EB091350E8EA39FA3C3
:10215000A8A7B9A78B839C83AD83BE8318861F82F3
:10216000AE01465D5F4FCE0101960E946D0D81303C
:102170009105B1F4D701ED91FC910684F785E02D2E
:102180001DA30CA38CA59DA5AEA5BFA58EA39FA343
:10219000A8A7B9A7A601BE016C5D7F4FC70119951D
:1021A000AF960FB6F894DEBF0FBECDBFDF91CF91D3
:1021B0001F910F91FF90EF90DF90CF9008957F9245
:1021C0008F929F92AF92BF92CF92DF92EF92FF9247
:1021D0000F931F93CF93DF93CDB7DEB7A6970FB6BC
:1021E000F894DEBF0FBECDBF8C01762E942E852EC7
:1021F00020E2A22ECE0101967C01DC01EA2D1D9287
:10220000EA95E9F76801F3E4CF0ED11C87E194E089
:102210009AA389A38FEF8BA38CA38DA38EA343E4F2
:1022200050E0BE016F5D7F4FC6010E94390D0196DF
:1022300009F4BFC081E089838A8386E0B82EBB821F
:102240001C82D80114966D917D918D919C91179768
:102250000E949DAE6D837E838F83988789869A8640
:1022600080E890E09C878B874CE150E0B701C60185
:102270000E94D10CFE0137968AE1DF011D928A95FA
:10228000E9F74801B8E08B0E911CF401D7010190E9
:102290000D92BA94E1F740E150E0B701C6010E9407
:1022A000D10CF7011192AA94E9F796E0A92EB12C6E
:1022B00040E250E0B701C6010E94D10CF1E0AF1A34
:1022C000B108B1F783E6898392E89A8393E59B830B
:1022D0008C8385E38D8381E08E837F829DE3988765
:1022E00097E099878A8786E0F401DE011B960190CA
:1022F0000D928A95E1F78CE0898B8A8B69E174E015
:10230000CE0143960E940EB1D8011B966C91CE016E
:1023100049960E94F572F8016485CE014B960E94A1
:10232000F572D8011D966C91CE014D960E94F57202
:102330004EE150E0B701C6010E94D10CB3E07B1220
:102340001EC082E3898384E08A83F80196859B839B
:1023500097859C8390899D8391899E8396E39F8333
:102360008887828D8987838D8A87848D8B87858DE9
:102370008C874CE050E0B701C6010E94D10C87E386
:10238000898386E08A8391E09B8393E09C838D839D
:102390008FE08E838AE38F838BE388878FEF898733
:1023A00049E050E0B701C6010E94D10CC6010E946D
:1023B000070DA6960FB6F894DEBF0FBECDBFDF9116
:1023C000CF911F910F91FF90EF90DF90CF90BF9032
:1023D000AF909F908F907F9008958F929F92AF9231
:1023E000BF92CF92DF92EF92FF920F931F93CF9302
:1023F000DF93CDB7DEB72D970FB6F894DEBF0FBED3
:10240000CDBF7C0110E000E038EE832E33E0932E48
:10241000A12CB12C43EDC42E43E0D42E1C821B8290
:102420008D829E82AF82B886DA82C9820D87CE0104
:1024300001960E94A60C811135C0F7014481558197
:1024400020E061E0802F0E94AB0B80E590E00E94CD
:10245000E50963E070E0802F0E949909833129F437
:1024600062E070E0802F0E948172F7018481958183
:10247000000F111FF801E65DF34F918380832D96C5
:102480000FB6F894DEBF0FBECDBFDF91CF911F9185
:102490000F91FF90EF90DF90CF90BF90AF909F9003
:1024A0008F9008950F5F1F4F0430110509F0B6CFCC
:1024B000E6CFCF92DF92EF92FF921F93CF93DF93FD
:1024C000FC011485143089F1EC0180E590E00E9454
:1024D000E50968E070E0812F0E9481720E943F7AD6
:1024E0006B017C01CE010E94A60C8823A1F061E063
:1024F00070E080E090E00E9481790E943F7A6C1940
:102500007D098E099F09683E73408105910550F34E
:102510008C850E94990BEC85F0E0EE0FFF1FE65DC5
:10252000F34F1182108284E08C87DF91CF911F914D
:10253000FF90EF90DF90CF9008954F925F926F924F
:102540007F928F929F92AF92BF92CF92DF92EF9243
:10255000FF921F93CF93DF93CDB7DEB72D970FB6C2
:10256000F894DEBF0FBECDBF7C019AE2A92E9CE09D
:10257000B92E10E0D12CC12C28EE422E23E0522E91
:10258000612C712C33ED832E33E0932E1C821B8241
:102590004D825E826F8278869A8289821D87D501FC
:1025A0002D913D915D01F7018481958128173907AF
:1025B000B1F4CE0101960E94A60C843199F1CE01AE
:1025C00001960E94A60C8C3151F4CE0101960E9416
:1025D0006A0A892B21F4CE0101960E9459121F5FCD
:1025E0001430A1F6CD2841F4D701ED91FC9100847F
:1025F000F185E02DC70119952D960FB6F894DEBF31
:102600000FBECDBFDF91CF911F91FF90EF90DF9074
:10261000CF90BF90AF909F908F907F906F905F9082
:102620004F900895CC24C394D12CD9CF8F929F92F0
:10263000AF92BF92CF92DF92EF92FF920F931F93D0
:10264000CF936C015B017A01FC01C485C430A1F415
:1026500081E090E0F60193838283F12CE12CC701A5
:10266000CF911F910F91FF90EF90DF90CF90BF908F
:10267000AF909F908F9008958A014130584010F09C
:1026800000E018E080E590E00E94E5098C2F0E94B0
:1026900091724C0163E070E08C2F0E9499098731A0
:1026A00011F08C3129F58016910660F380E590E0F9
:1026B0000E94E5099801A50170E060E08C2F0E945E
:1026C000C69060E270E08C2F0E94817262E070E040
:1026D0008C2F0E94990984FD13C063E070E08C2F59
:1026E0000E949909811107C08C2F0E94990BB0CFCD
:1026F00010E000E0DBCF80E590E00E94E509E6CF46
:1027000040E162E070E08C2F0E947E09012B09F00D
:10271000A6CF9ECF3F924F925F926F927F928F9201
:102720009F92AF92BF92CF92DF92EF92FF920F9360
:102730001F93CF93DF93CDB7DEB72D970FB6F894E5
:10274000DEBF0FBECDBF6C015B014A010E949D122E
:102750008AE2E82E8CE0F82E312C10E000E098EEB2
:10276000492E93E0592E612C712C1C821B824D82C4
:102770005E826F82788683ED93E09A8389833D86BB
:10278000F701219131917F01F6018481958128170C
:10279000390771F4CE0101960E94A60C873141F4ED
:1027A000A401B501CE0101960E941613080F191F4E
:1027B0003394F4E03F12D9CFC8012D960FB6F894A8
:1027C000DEBF0FBECDBFDF91CF911F910F91FF9064
:1027D000EF90DF90CF90BF90AF909F908F907F90C1
:1027E0006F905F904F903F900895CF92DF92EF925D
:1027F000FF920F931F93CF93DF938B017A016C01AC
:1028000027EBC20ED11CF6014081EC012A9644232D
:1028100049F050E0BC0169567F4FCE010E9416136B
:10282000F6011082A701B801CE01DF91CF911F916F
:102830000F91FF90EF90DF90CF900C941613CF93F1
:10284000DF93EC01C954DF4FE88121E02E0F28838C
:10285000E80FF92FF11DE956FF4F6083203249F44C
:10286000BC0169567F4F40E250E00A960E94161361
:10287000188281E090E0DF91CF910895CF92DF92AE
:10288000FF920F931F93CF93DF93FC012485243095
:1028900051F090E080E0DF91CF911F910F91FF9078
:1028A000DF90CF9008956A01EB018C01F12C8F2D00
:1028B0000E946D0C811129C0F801F486F80184850D
:1028C000843039F320916802309169022F5F3F4FC5
:1028D00021F130936902209368024091680250917F
:1028E000690220E061E00E94AB0B8A818F3FC1F456
:1028F0008B818F3F01F58C818F3FE9F48D818F3F74
:10290000D1F484E0F8018487C4CF8B7F8831A1F2B1
:10291000F394F4E0FF12CBCFD1CF20E030ECD9CF4D
:10292000811109C08B81811106C08C81811103C086
:102930008D81882331F3C114D10419F3F801F48493
:1029400080E590E00E94E509BE016E5F7F4F8F2D0C
:102950000E942A08B6018F2D0E94880964E070E069
:102960008F2D0E948172C8010E94A60C873161F0F0
:1029700061E070E080E090E00E948179C8010E94EF
:10298000A60C8111F0CFBDCF81E090E084CFCF9332
:10299000CFB7F8948091FE0B811127C0E2EBFCE0E9
:1029A0008491E8EFFCE09491E82FF0E0EE0FFF1F38
:1029B000E15DF34FA591B491EC91E92321F461E03D
:1029C00085E30E940E7861E085E30E942B798CB547
:1029D00080618CBD8CB580648CBD61E084E30E9415
:1029E0002B7961E083E30E942B798091FE0B8F5F4E
:1029F0008093FE0BCFBFCF9108954F925F926F925D
:102A00007F928F929F92AF92BF92CF92DF92EF927E
:102A1000FF920F931F93CF93DF93EC0118161906C3
:102A20001CF44C0104972CF0C1E0D0E063E0862E4A
:102A3000912C8E01000F111F7E01EE0CFF1CEE0C7D
:102A4000FF1C8C169D060CF4B3C097012C5B3D4F08
:102A50005901F90180819181A281B38197012152AD
:102A60003D4F6901181619061A061B063CF50E940F
:102A7000187CF6014080518062807380641975096A
:102A800086099709F501408051806280738046165F
:102A900057066806790658F4108211821282138252
:102AA0000E94187CF6016083718382839383219650
:102AB0000E5F1F4FF4E0EF0EF11CC3CF98012952B7
:102AC0003D4F3901F90180819181980121533D4F9A
:102AD0005901F9012081318182179307C1F0880FD4
:102AE000991FFC01EB54F44F6081F801EA50F44F58
:102AF00080810E940E78F30180819181F50191839C
:102B000080836CE271E080E090E00E948179F601C0
:102B100080819181A281B381181619061A061B06BD
:102B200034F60E94187CF601208131814281538164
:102B3000621B730B840B950BF701E154FD4F208151
:102B4000318142815381261737074807590708F01A
:102B5000AECFF601108211821282138298012C5A94
:102B60003D4F6901F90180819181F5012081318119
:102B70008217930709F49BCF880F991FFC01EB5430
:102B8000F44F6081F801EA50F44F80810E940E7882
:102B9000F60180819181F50191838083F301918316
:102BA00080836CE271E080E090E00E9481797FCFC9
:102BB000DF91CF911F910F91FF90EF90DF90CF9019
:102BC000BF90AF909F908F907F906F905F904F904D
:102BD0000895CF93DF93FC0124813581232B69F085
:102BE000EC01BC018CE39DE00E940A77BE018FE9F5
:102BF0009CE0DF91CF910C940A77DF91CF910895FB
:102C0000CF93DF93FC0124813581232B69F0EC0104
:102C1000BC018CE39DE00E94FC76BE018FE99CE044
:102C2000DF91CF910C94FC76DF91CF9108958F9234
:102C30009F92AF92BF92CF92DF92EF92FF920F934B
:102C40001F93CF93DF938C01862F0B30110509F072
:102C50009FC090917811992309F0F89462E10E9445
:102C6000B479EC0180917811882309F07894209749
:102C700001F180E090ECA9E7B4EC80936B119093A4
:102C80006C11A0936D11B0936E1180936F1190939E
:102C90007011A0937111B0937211CE3F8FEFD807CE
:102CA00009F4A9C0CF3FDC0709F462C0CCEFDFEF25
:102CB00030C1C0917311E09074116E2D70E090E0FE
:102CC00080E00E94B0AB2DEC3CEC4CEC5DE30E944C
:102CD0000FAC4B015C016C2F70E090E080E00E9433
:102CE000B0AB9B01AC01C501B4010E9457AD60932C
:102CF0006B1170936C1180936D1190936E11D09144
:102D00007511F09076116D2F6F7770E090E080E094
:102D10000E94B0AB4B015C016F2D70E090E080E051
:102D20000E94B0AB2DEC3CEC4CEC5DE30E940FAC90
:102D30009B01AC01C501B4010E9457ADD7FD26C06F
:102D400060936F1170937011809371119093721151
:102D5000CE0DCD0FCF0D81E090E020917711C21301
:102D600002C090E080E0892B09F493C0CFEFDFEF41
:102D7000CE01DF91CF911F910F91FF90EF90DF90E7
:102D8000CF90BF90AF909F908F9008959058D8CFDC
:102D9000CFEFDFEF0631110509F0BBC0909178113C
:102DA000992309F0F89461E00E94B479EC018091D4
:102DB0007811882309F07894209701F180E090EC55
:102DC000A9E7B4EC80936B1190936C11A0936D11F3
:102DD000B0936E1180936F1190937011A093711145
:102DE000B0937211CF3FDC0719F2209709F451C05C
:102DF000229609F05BCFCEEFDFEF8BC0C09174114C
:102E0000D0917311609173117091741176276727B7
:102E1000762790E080E00E94AEAB2DEC3CEC4CECD1
:102E20005DE30E940FAC60936B1170936C11809303
:102E30006D1190936E11E0907611F09075116F2DD9
:102E40006F77762F6E2D90E080E00E94AEAB2DEC78
:102E50003CEC4CEC5DE30E940FACF7FC18C06093B7
:102E60006F117093701180937111909372118C2F68
:102E70008D0F8E0D8F0DC1E0D0E0909177118913E9
:102E800002C0D0E0C0E0D195C195D109ABCF905838
:102E9000E6CFC0906B11D0906C11E0906D11F09066
:102EA0006E1120E030E048EC52E4C701B6010E9408
:102EB0006BAED0E0C0E0181614F4CBEFDFEF20E0EB
:102EC00030E0A901C701B6010E94A9AB87FF02C08B
:102ED000CAEFDFEFC0906F11D0907011E0907111C8
:102EE000F090721120E030E048EC52ECC701B601DE
:102EF0000E94A9AB87FF02C0C9EFDFEF20E030E0FE
:102F000040EF52E4C701B6010E946BAE18160CF4F4
:102F100083C00C30110509F02BCF81E080939B0C0E
:102F20008CE580939D0C10929C0C10929E0C60E09E
:102F300089ED9DE00E94037081E00E94977E0E94CF
:102F40005C796B017C018091950C811168C081E0F6
:102F50008093950C8093940C9FEF9093930C109218
:102F6000920C94E09093910C8093700C8091700C73
:102F7000886B8093700C80916F0C813009F028C1B0
:102F800010926F0C0E945C796B017C018091700C37
:102F90008093BB008091970C9091980CA091990C14
:102FA000B0919A0C892B8A2B8B2BA1F00E945C7913
:102FB0000091970C1091980C2091990C30919A0CDB
:102FC0006C197D098E099F0906171707280739070D
:102FD00008F446C08091BC0083FDD8CF85EC809377
:102FE000BC000E945C796B017C018091950C813062
:102FF00009F4F0C08091920C853008F00DC18091E9
:10300000920CA1E7BCE0E1E0FCE090E0981769F1E8
:103010002D9121939F5FFACFC8EFDFEF7ACF809198
:10302000970C9091980CA091990CB0919A0C892BC7
:103030008A2B8B2B09F487CF0E945C790091970C27
:103040001091980C2091990C30919A0C6C197D0973
:103050008E099F09061717072807390708F073CF4D
:103060008091960C0E94767E80E01092550C8093A1
:10307000540C082F10E0CEEFDFEF882309F478CE50
:10308000CDEFDFEF053011050CF472CECAEDDAE0BA
:1030900089ED9DE00E94BC6F88872196CE018A5DF4
:1030A0009A4080179107A4F3C091E20A0091E30AC5
:1030B000602F70E090E080E00E94B0AB2DEC3CEC23
:1030C0004CEC5DE30E940FAC6B017C016C2F70E057
:1030D00090E080E00E94B0AB9B01AC01C701B6015B
:1030E0000E9457AD6B017C01C092DA0AD092DB0AD4
:1030F000E092DC0AF092DD0AD091E40A1091E50A30
:103100006D2F6F7770E090E080E00E94B0AB4B01D4
:103110005C01612F70E090E080E00E94B0AB2DEC8C
:103120003CEC4CEC5DE30E940FAC9B01AC01C50193
:10313000B4010E9457ADD7FD71C06093DE0A709351
:10314000DF0A8093E00A9093E10AC00FCD0FC10F10
:103150008091E60AC8130ACE20E030E048EC52E441
:10316000C701B6010E946BAED0E0C0E0181614F49F
:10317000CBEFDFEF20E030E040EA50E4C701B601DA
:103180000E94A9AB87FF02C0CAEFDFEFC090DE0A42
:10319000D090DF0AE090E00AF090E10A20E030E011
:1031A00040EF51ECC701B6010E94A9AB87FF02C0F6
:1031B000C9EFDFEF20E030E040EF52E4C701B60195
:1031C0000E946BAE18160CF0D3CDC8EFDFEFD0CD58
:1031D00085EE05CF8091970C9091980CA091990C59
:1031E000B0919A0C892B8A2B8B2B09F4FECE0E946E
:1031F0005C790091970C1091980C2091990C30916A
:103200009A0C6C197D098E099F0906171707280764
:10321000390708F0EACE24CF85E0F3CE90588DCF61
:10322000CF93DF93FB0122813381DC0113963C9322
:103230002E931297448155816681778114964D9320
:103240005D936D937C931797408551856285738557
:1032500018964D935D936D937C931B971C96EF018D
:103260002C969C01275E3F4F49914D93A217B307BF
:10327000D9F7218D328DFC01328F218FDF91CF91D3
:1032800008950F931F93CF93DF938C01EB01FE0101
:1032900064912196662349F0D801ED91FC9101904B
:1032A000F081E02DC8011995F2CFDF91CF911F91E8
:1032B0000F910895EF92FF920F931F93CF93DF9397
:1032C000EC017B018A0168E074E00E94411961EF22
:1032D00073E0CE010E94411962EC73E0CE010E94BE
:1032E0004119B701CE010E94F47663EC79E0CE017A
:1032F0000E94F4760115110521F0B801CE010E945B
:10330000F47663EC79E0CE01DF91CF911F910F91BC
:10331000FF90EF900C94F476CF93DF93EC0167EA83
:1033200073E00E94411961EF73E0CE010E944119E0
:1033300069E773E0CE01DF91CF910C944119CF93EF
:10334000DF93EC01FB01248135810E94D875CE0109
:10335000DF91CF910895EF92FF920F931F93CF9338
:10336000DF9300D000D0CDB7DEB78C017B0163ECDA
:1033700078E00E94C3758AE0E816F1042CF461E855
:1033800076E0C8010E949E74B701CE0101960E94AA
:103390001173BE016F5F7F4FC8010E94A874CE01F8
:1033A00001960E942475C80126960FB6F894DEBFD8
:1033B0000FBECDBFDF91CF911F910F91FF90EF9086
:1033C0000895CF92DF92EF92FF920F931F93CF93C6
:1033D000DF93CDB7DEB7C455D1090FB6F894DEBF81
:1033E0000FBECDBF65965FAF4EAF65972091320C93
:1033F0003091330C2F5F3F4F3093330C2093320CBE
:1034000020914F0C2111C1C08B016C0181E0809390
:103410004F0C1092330C1092320C63EC78E0CE011A
:10342000895B9F4F0E94C37563EC78E0CE01835B9C
:103430009F4F0E94C37550E040E060E274E0C60117
:103440000E945A190130110509F08EC063EC78E032
:1034500087E090E10E94077363EC78E083EE9FE0E1
:103460000E9407736596EEADFFAD65978081882356
:1034700009F474C000E210E09E012F5F3F4F40E26C
:1034800050E0BE016F5D7F4FCE018D5A9F4F0E946D
:103490006571049739F3BE016F5D7F4FCE018F5B7D
:1034A0009F4F0E94C375BE016F5B7F4FCE01895B4A
:1034B0009F4F0E94EB74CE018F5B9F4F0E9424753B
:1034C000BE016F5F7F4FCE018F5B9F4F0E94C37520
:1034D000BE016F5B7F4FCE01835B9F4F0E94EB74F9
:1034E000CE018F5B9F4F0E9424752D968EAD9FADB0
:1034F0002D970297029730F469E374E083EE9FE022
:103500000E940773BE01695B7F4F87E090E10E94D4
:10351000A87463968EAD9FAD6397892B09F4A2CFF3
:1035200062EF75E0CE018F5B9F4F0E94C375BE01B5
:10353000635B7F4FCE018F5B9F4F0E943F746FEEA6
:1035400075E00E942974BC0187E090E10E94A87494
:10355000CE018F5B9F4F0E94247584CF67E070E19E
:1035600083EE9FE00E94A87410924F0CCE01835B03
:103570009F4F0E942475CE01895B9F4F0E94247546
:103580000FB6F894DEBF0FBECDBFCC5ADF4F0FB6DB
:10359000F894DEBF0FBECDBFDF91CF911F910F9189
:1035A000FF90EF90DF90CF9008950F931F93CF93EC
:1035B000DF9300D000D0CDB7DEB72091B90B222326
:1035C000A9F08C016BE777E0CE0101960E94C375EC
:1035D000B801CE0101960E943F74BC018CE39DE0CE
:1035E0000E940A77CE0101960E94247526960FB696
:1035F000F894DEBF0FBECDBFDF91CF911F910F9129
:1036000008950F931F93CF93DF93CDB7DEB72C9719
:103610000FB6F894DEBF0FBECDBF8C010E94C27DF5
:10362000BC01C8010E94AB190E94BA7DBC01CE0149
:1036300007960E94AB196FEA76E0CE0101960E94D0
:10364000C375BE01695F7F4FCE0101960E943F7432
:10365000BC01C8010E94A874CE0101960E94247585
:10366000CE0107960E9424756FEE75E0C8010E9496
:103670009E740E94B27DBC01CE0101960E94AB19DE
:10368000BE016F5F7F4FC8010E94A874CE010196F2
:103690000E94247560E474E0C8010E949E740E9438
:1036A000AA7DBC01CE0101960E94AB19BE016F5FDD
:1036B0007F4FC8010E94A874CE0101960E94247514
:1036C00060E474E0C8010E949E740E94A07DBC0169
:1036D000CE0101960E94AB19BE016F5F7F4FC801FA
:1036E0000E94A874CE0101960E942475C8012C96F0
:1036F0000FB6F894DEBF0FBECDBFDF91CF911F9103
:103700000F9108950F931F93CF93DF93CDB7DEB73B
:103710002C970FB6F894DEBF0FBECDBF8C010E9470
:10372000C27DBC01C8010E94AB190E94BA7DBC01D8
:10373000CE0107960E94AB196FEA76E0CE010196A2
:103740000E94C375BE01695F7F4FCE0101960E9442
:103750003F74BC01C8010E94A874CE0101960E946A
:103760002475CE0107960E9424750E94187C0E9441
:10377000A77C6091210C70E0CE0107960E94AB19E6
:103780006FEA76E0CE0101960E94C375BE01695FC3
:103790007F4FCE0101960E943F74BC01C8010E9478
:1037A000A874CE0101960E942475CE0107960E944E
:1037B00024756FEE75E0C8010E949E740E94B27D70
:1037C000BC01CE0101960E94AB19BE016F5F7F4F15
:1037D000C8010E94A874CE0101960E94247560E47D
:1037E00074E0C8010E949E740E94AA7DBC01CE01B3
:1037F00001960E94AB19BE016F5F7F4FC8010E9406
:10380000A874CE0101960E94247560E474E0C8019A
:103810000E949E740E94A07DBC01CE0101960E9470
:10382000AB19BE016F5F7F4FC8010E94A874CE0123
:1038300001960E942475C8012C960FB6F894DEBF3D
:103840000FBECDBFDF91CF911F910F910895CF9201
:10385000DF92EF92FF920F931F93CF93DF9300D0ED
:1038600000D0CDB7DEB77C01FB01848195818A0150
:10387000081B190B101611069CF0C7010E94A875B1
:10388000C70126960FB6F894DEBF0FBECDBFDF91FD
:10389000CF911F910F91FF90EF90DF90CF900895FF
:1038A000CE0101960E94BA75CC24C394D12C6FEE40
:1038B00075E0CE0101960E949E74FFEFCF1ADF0AD9
:1038C0000C151D05A4F7BE016F5F7F4FC7010E9455
:1038D000A875CE0101960E942475D2CFDF92EF9297
:1038E000FF920F931F93CF93DF93CDB7DEB762970D
:1038F0000FB6F894DEBF0FBECDBF8C011092EB0A5D
:1039000063EC78E0CE010D960E94C375FF24F3941A
:103910008CE39DE00E94196E2091EB0A181619069F
:103920007CF521112DC08CE39DE00E94F76D8A305B
:1039300009F07EC089899A89892B09F481C0F092A7
:10394000EB0A62E474E0CE0101960E94C375BE01E9
:10395000635F7F4FCE0101960E943F74BC01CE0190
:1039600007960E94BA75CE0107960E94D51ACE011D
:1039700007960E942475CE0101960E94247560C0AE
:10398000F12CE12CDD24D394222309F460C0898931
:103990009A89019709F045C061EE74E0CE0107965F
:1039A0000E94C375BE01695F7F4FCE010D960E94D4
:1039B0000E74F12C811115C062E574E0CE01019600
:1039C0000E94C375BE016F5F7F4FCE010D960E94AE
:1039D0000E74FF24F3948111F12CCE0101960E9404
:1039E0002475CE0107960E942475FF20A1F050E0B7
:1039F00040E0BE01635F7F4FCE0101960E949F1998
:103A0000BE016F5F7F4F8AEA9FE00E94EB74CE0198
:103A100001960E94247564E170E080E090E00E94CD
:103A20008179BE01635F7F4FC8010E94A8758EC077
:103A30008D3009F47FCF682FCE010D960E947C74E3
:103A40006AE070E080E090E00E94817961CF8FE9C8
:103A50009CE00E94196E1816190614F58FE99CE077
:103A60000E94F76D8A30A9F08D3099F09091EB0AA1
:103A700091110FC0682FCE010D960E947C748FEFBC
:103A8000E81AF80A65E070E080E090E00E94817931
:103A9000DECF89899A89892BA9F3D092EB0AF2CFDC
:103AA00064E170E080E090E00E948179EF2809F401
:103AB0003FC089899A89892BD9F18091B90B8823D4
:103AC00089F16BE777E0CE0101960E94C375BE01D4
:103AD0006F5F7F4FCE010D960E940E74F82ECE01BF
:103AE00001960E942475F1101DC06BE474E0CE01B4
:103AF00001960E94C375CE0101960E940016CE0168
:103B000001960E942475BE01635F7F4FCE0101962E
:103B10000E94BA75CE0101960E94E915CE01019668
:103B20000E94247564E170E080E090E00E94817959
:103B300089899A892091EB0A21112BCF009709F0EE
:103B400028CF63EC78E0C8010E94C375CE010D96C2
:103B50000E942475C80162960FB6F894DEBF0FBEAE
:103B6000CDBFDF91CF911F910F91FF90EF90DF902C
:103B700008950F931F93CF93DF93CDB7DEB72C97A4
:103B80000FB6F894DEBF0FBECDBF2C893D89FE0174
:103B90007496A6EFBBE090E080E0329628173907D4
:103BA00034F0408151814D935D930196F6CFCE5B09
:103BB000DE4F88819981C254D140281739070CF013
:103BC0001CC2DC01AA0FBB1FAA50B44F880F991F5B
:103BD000FC01EC50F44F8081918101968D939C9370
:103BE0008C8D9D8D9093B60B8093B50B8E8D9F8D94
:103BF0009093B80B8093B70BAD968FADAD97BE0188
:103C000064597F4F8F3209F001C2CE0107960E949E
:103C1000C37564E574E0CE0101960E94C375BE01D0
:103C2000695F7F4FCE0101960E943F74BC0187E916
:103C300091E10E94D474CE0101960E942475CE01B8
:103C400007960E94247567E971E1CE0101960E94F2
:103C5000BA75CE0101960E94E915CE0101960E9427
:103C600024756AE674E0CE0101960E94C375BE0118
:103C70006F5F7F4F87E991E10E94EE73182FCE01AD
:103C800001960E94247540919B1150919C11112323
:103C900009F4C3C1BA016250710987E991E10E9438
:103CA000DD73682FCE0101960E948F75BE016F5F94
:103CB0007F4F89E791E10E94EB74CE0101960E944B
:103CC000247569E670E1CE0107960E94C3756CE623
:103CD00074E0CE0101960E94C375BE01695F7F4FFB
:103CE000CE0101960E943F74BC0181E991E10E94DE
:103CF000D474CE0101960E942475CE0107960E94CD
:103D0000247524968FAD24971F928F9323968FADA1
:103D100023971F928F9322968FAD22971F928F9396
:103D200021968FAD21971F928F9382E794E09F9306
:103D30008F9386EE9BE09F938F930E944CB1CE525F
:103D4000DF4F88819981C25DD04090938F0280932C
:103D50008E02BE016C527F4FCE0101960E94C37548
:103D6000BE016F5F7F4F8BE891E10E94EB74CE0143
:103D700001960E942475BE0161527F4FCE010196CB
:103D80000E94C375BE016F5F7F4F85E891E10E947D
:103D9000EB74CE0101960E942475409189115091D7
:103DA0008A114250510965E871E1CE0101960E94E5
:103DB0009F19CE0101960E9475736C59609397020A
:103DC000CE0101960E942475CC5EDE4F6881798118
:103DD0008A819B81C451D1400E94B0AB0FB6F89448
:103DE000DEBF0FBECDBF9B01AC010E9470AE882329
:103DF00089F08CE390E0A0E0B0E0CC5EDE4F8883F9
:103E00009983AA83BB83C451D140CD5EDE4F188213
:103E1000C351D140CD5EDE4F8881C351D14088234C
:103E200099F0CC5EDE4F88819981AA81BB81C45113
:103E3000D1408093700290937102A0937202B0936C
:103E4000730281E08093580CC85EDE4F68817981EF
:103E50008A819B81C851D1409B01AC010E9470AE08
:103E6000882361F080E090E0A0E7B2E4C85EDE4F16
:103E700088839983AA83BB83C851D140C45EDE4F37
:103E800068817981CC51D140072E000C880B990BA9
:103E90000E94B0AB9B01AC010E9470AE882341F040
:103EA00082E090E0C45EDE4F99838883CC51D1409C
:103EB000CE5BDE4F68817981C254D140072E000C61
:103EC000880B990B0E94B0AB9B01AC010E9470AEB5
:103ED000882341F083E090E0CE5BDE4F99838883B6
:103EE000C254D140C45CDE4F08811981CC53D1400B
:103EF000B801012E000C880B990B0E94B0AB9B01FE
:103F0000AC010E9470AE811103C01016110644F07E
:103F100080E590E0C45CDE4F99838883CC53D14028
:103F2000C45CDE4F88819981CC53D14090933F028D
:103F300080933E0288E2FE01E551FF4FAAEBBBE011
:103F400001900D928A95E1F7CE5CDE4F88819981D0
:103F5000AA81BB81C253D1408093290290932A0247
:103F6000A0932B02B0932C02CA5CDE4F888199810A
:103F7000AA81BB81C653D14080932502909326022B
:103F8000A0932702B0932802C65CDE4F88819981F6
:103F9000CA53D14090935D0280935C02CC5BDE4FAC
:103FA00068817981C454D140072E000C880B990B8D
:103FB0000E94B0AB9B01AC010E9470AE882341F01F
:103FC00088E390E0CC5BDE4F99838883C454D14072
:103FD000CC5BDE4F88819981C454D140909391028B
:103FE000809390022C960FB6F894DEBF0FBECDBF23
:103FF000DF91CF911F910F9108958091FA0B9091CD
:10400000FB0B9093FD0B8093FC0BEACDCE01079642
:104010000E94C37569E574E0FECD4150510967E91E
:1040200071E1CE0101960E949F19BE016F5F7F4F23
:1040300089E791E10E94EB74CE0101960E942475FC
:1040400067E971E1CE0101960E94BA756AE674E0F3
:10405000CE0101960E942974BC0187E991E10E947A
:10406000D4742BCEDF92EF92FF920F931F93CF93D6
:10407000DF93CDB7DEB762970FB6F894DEBF0FBE01
:10408000CDBF2091F002222379F12091EF0222236B
:1040900059F17A018C016F3F7F4FA1F560E080E01C
:1040A0000E94C57FD12CB8018FEE91E10E94FC7671
:1040B00060E175E08FEE91E10E941E77F801848146
:1040C00060E08D0D0E94C57F0E943F7A60936B0C6B
:1040D00070936C0C80936D0C90936E0CB701FF0C79
:1040E000880B990B0E94817962960FB6F894DEBF17
:1040F0000FBECDBFDF91CF911F910F91FF90EF9039
:10410000DF90089560E080E00E94C57F0E943F7AC2
:1041100028EE33E040E050E00E94F3ACCA01B90160
:1041200020E831E541E050E00E9415ADAB01BC0153
:1041300020E0CE0101960E946275BE016F5F7F4F45
:10414000CE0107960E94BA7565E678E0CE01079623
:104150000E942974BC01CE010D960E94BA75CE0151
:1041600007960E942475CE0101960E942475BE0117
:10417000635F7F4F8FEE91E10E94FC76D98860E00B
:104180008D2D0E94C57FCE010D960E9424758BCF88
:10419000CF93DF9300D000D0CDB7DEB70E94E50803
:1041A000CE0101960E94011B4AE050E06FEF7FEFC5
:1041B000CE0101960E943220CE0101960E94247504
:1041C00061E080E00E94C57FCE0101960E943D72B1
:1041D0006FEE71E1CE0101960E9496766EE774E073
:1041E0008FEE91E10E94F4760E943F7A60933C0C3E
:1041F00070933D0C80933E0C90933F0C26960FB627
:10420000F894DEBF0FBECDBFDF91CF9108950F931D
:104210001F93CF93DF9300D000D0CDB7DEB78C01D2
:10422000CE0101960E94011B4AE050E06FEF7FEF44
:10423000CE0101960E943220CE0101960E94247583
:10424000B801CE0101960E94BA754AE050E06FEFC6
:104250007FEFCE0101960E940909CE0101960E94CE
:10426000247526960FB6F894DEBF0FBECDBFDF9142
:10427000CF911F910F9108952F923F924F925F928D
:104280006F927F928F929F92AF92BF92DF92EF9246
:10429000FF920F931F93CF93DF93CDB7DEB7E497D1
:1042A0000FB6F894DEBF0FBECDBF7C014A015B01A3
:1042B00019010E943F7A2B013C0187010D5B1F4FC2
:1042C000C8010E94290B181619069CF00E943F7A1B
:1042D000641975098609970986169706A806B9060E
:1042E00008F490C162E370E080E090E00E94817980
:1042F000E7CF42E250E0BE016F5F7F4FC8010E94EE
:10430000E00A8981823009F078C1F80184899589B1
:104310008334910509F071C16D817E818F8198850B
:104320000E949DAE2B013C01F101408251826282CC
:10433000738246E050E0B701685F7F4FCE014D9633
:104340000E94CBB0892B99F4F70180819181A281E1
:10435000B381481659066A067B0648F08481958128
:10436000A681B78184159505A605B705E8F4C801AF
:104370000E949107D12C8D2DE4960FB6F894DEBFE4
:104380000FBECDBFDF91CF911F910F91FF90EF90A6
:10439000DF90BF90AF909F908F907F906F905F90D5
:1043A0004F903F902F90089589899A89AB89BC8955
:1043B00086879787A08BB18B8EECA82EB12CC80175
:1043C0000E94FF0AF1E0AF1AB108C9F7D12CC7016A
:1043D00082969AA789A7F701B696FCA7EBA708963D
:1043E0009EA78DA73C974F01899698AB8FA73897CA
:1043F000FAABE9AB1701F6E12F0E311CC5979CAB68
:104400008BABF801818D928D181619060CF0F6C051
:10441000C8010E94FF0A8333910509F4D4C0A4F5B2
:104420008130910509F474C074F4892B51F3C801EB
:104430000E94FF0AB82EBA94FFEFBF1611F3C8010D
:104440000E94FF0AF8CF8330910509F46CC00697EB
:1044500071F7C8010E94FF0AA82E44E050E06BA942
:104460007CA9C8010E94E00A712C612CEA2DE4505D
:10447000FF0B5F016A147B0424F6C8010E94FF0A47
:10448000FFEF6F1A7F0AF6CF8A33910509F46FC0E8
:1044900074F585339105A1F1C69749F6C8010E94CC
:1044A000FF0AB82EF701828D811109C0838D811119
:1044B00006C0848D811103C0858D8823A1F0EFA5EE
:1044C000F8A94080518062807380B401CE01839648
:1044D0000E9442778DA19EA1AFA1B8A58415950534
:1044E000A605B705D9F544E050E0B40118C08B33F8
:1044F000910509F452C08F3F910509F482CF97CFFF
:10450000C8010E94FF0AC8010E94FF0AD82E79CF75
:10451000C8010E94FF0A44E050E069A97AA9C801D5
:104520000E94E00A6ECFC8010E94FF0AA82E44E054
:1045300050E0B101C8010E94E00A712C612C8A2D63
:104540008450990B5C016A147B040CF05ACFC801AB
:104550000E94FF0A9FEF691A790AF5CFBA94FFEF1C
:10456000BF1609F44ECFC8010E94FF0AF7CFC80159
:104570000E94FF0A44E050E06BA57CA5C8010E94A0
:10458000E00AF70166A177A180A591A50E949DAEE2
:1045900066A377A380A791A734CFC8010E94FF0A22
:1045A00044E050E06DA57EA5C8010E94E00AF70135
:1045B00062A573A584A595A50E949DAE62A773A769
:1045C00084A795A71ECFC8010E94FF0A44E050E0CF
:1045D00069A57AA5C8010E94E00AF70162A173A14A
:1045E00084A195A10E949DAE62A373A384A395A309
:1045F00066A777A780AB91AB04CFD12CC8010E94EE
:104600009107B9CEDD24DA94B6CE2F923F924F9225
:104610005F926F927F928F929F92AF92BF92CF9252
:10462000DF92EF92FF920F931F93CF93DF9300D00F
:1046300000D0CDB7DEB78C010E9414A32FEC37E079
:1046400040E050E00E9415ADDC01CB010196A11DB8
:10465000B11DF80184839583A683B78380839183FA
:10466000A283B3835801F3E4AF0EB11CC5010E94CD
:10467000580C64E470E0C5010E94790C882309F4A9
:1046800045C10E943F7A2B013C01480182E4880E1B
:10469000911C48EEC42E43E0D42EE12CF12C52E0C4
:1046A000252E1E821D82D4018C918330B1F181119F
:1046B00066C0F80184819581A681B7810196A11D0C
:1046C000B11D84839583A683B7830E943F7A6419C2
:1046D000750986099709A70196010E94F3ACA90103
:1046E00061E0C8010E94DF1081E0D4018C938D81CC
:1046F0009E810197C1F20E943F7A6419750986096B
:104700009709D801D6962D913D914D915C91D997FD
:10471000261737074807590720F6C5010E94580C8D
:10472000F80184819581A681B7810196A11DB11DF3
:1047300084839583A683B7830E943F7AF801FE960F
:1047400060837183828393838D819E8126960FB6C9
:10475000F894DEBF0FBECDBFDF91CF911F910F91B7
:10476000FF90EF90DF90CF90BF90AF909F908F9091
:104770007F906F905F904F903F902F90089584307E
:10478000F1F4F80184819581A681B7810196A11D7C
:10479000B11D84839583A683B7830E943F7A6419F1
:1047A000750986099709A70196010E94F3ACA90132
:1047B00063E0C8010E94DF10D4012C9298CF8130B1
:1047C00051F5F80142AD53AD64AD75AD9E012F5F5B
:1047D0003F4FC8010E943C21382EF2E08F1390C059
:1047E00089819A81AB81BC81F80184839583A683FA
:1047F000B7830E943F7A6419750986099709A70152
:1048000096010E94F3ACA90163E0C8010E94DF1089
:10481000D4013C926CCF823009F069CFF80142ADEF
:1048200053AD64AD75AD9E012F5F3F4FC8010E942F
:104830003C21382EF5E08F135DC0E3E0D401EC930A
:10484000F80182A193A1A4A1B5A1892B8A2B8B2B5E
:1048500041F484E893E0A0E0B0E082A393A3A4A392
:10486000B5A3F80186A197A1A0A5B1A5892B8A2B94
:104870008B2B61F482A193A1A4A1B5A1B695A795B4
:104880009795879586A397A3A0A7B1A7F80182A5BE
:1048900093A5A4A5B5A5892B8A2B8B2BA9F482A15E
:1048A00093A1A4A1B5A1AC01BD0123E076956795C4
:1048B000579547952A95D1F7841B950BA60BB70BF7
:1048C00082A793A7A4A7B5A7F80186A197A1A0A541
:1048D000B1A586A797A7A0ABB1AB82A593A5A4A5C8
:1048E000B5A582AB93ABA4ABB5AB81E090E09E8362
:1048F0008D83FDCE96E0891303C0D4011C92F7CEC0
:10490000BFEF3B12F4CEF4011082F1CE1E821D8265
:104910001BCFEF92FF920F931F93CF93DF93CDB7EF
:10492000DEB7E8970FB6F894DEBF0FBECDBF63ECDD
:1049300078E0CE0187960E94C37563EC78E0CE01E3
:104940008D960E94C37582E0E82EF12C2496FFAE6E
:10495000EEAE249786E0E1E0F3E0DE01D39601902D
:104960000D928A95E1F786E0FE01F396DE01AC5BDD
:10497000BF4F01900D928A95E1F72C961FAE1EAEA7
:104980002C9701E010E02E961FAF0EAF2E9788E017
:10499000E7E0F3E0DE01599601900D928A95E1F788
:1049A00088E0FE017996DE01A25BBF4F01900D9277
:1049B0008A95E1F788E1EFE0F3E0DE0111960190DE
:1049C0000D928A95E1F788E1FE013196DE01AA5A3F
:1049D000BF4F01900D928A95E1F780912703909146
:1049E0002803A0912903B0912A03E2968CAF9DAFD2
:1049F000AEAFBFAFE29762E874E0CE0187960E9447
:104A0000077360E0CE0187960E947C744BA55CA57D
:104A1000BE016E587F4FCE0187960E945B7260E3A5
:104A200076E0CE018D960E94AF7468ED74E089E760
:104A300091E10E94077360E0CE018D960E947C7424
:104A400049A95AA9BE0166567F4FCE018D960E9494
:104A50005B7263EC78E0CE0187960E94077363EC8B
:104A600078E0CE018D960E940773C250DF4F198205
:104A70001882CE5FD04080918E0290918F02C050FC
:104A8000DF4F99838883C050D14080E090E0A0E759
:104A9000B2E4CA5BDE4F88839983AA83BB83C65482
:104AA000D140C65BDE4FF982E882CA54D14080E033
:104AB00090E0A0E2B2E4C45BDE4F88839983AA83CE
:104AC000BB83CC54D14080E090E0A4E3B2E4C05B6F
:104AD000DE4F88839983AA83BB83C055D14084EB82
:104AE00090E0CC5ADE4F99838883C455D14088E743
:104AF00090E0CA5ADE4F99838883C655D1408CE234
:104B000091E0A0E0B0E0C85ADE4F88839983AA8381
:104B1000BB83C855D140C45ADE4F19830883CC5596
:104B2000D140C25ADE4FF982E882CE55D14060E0D2
:104B30008BE891E10E947C7460E085E891E10E943D
:104B40007C7440918F1150919011BE016E5F7E4F29
:104B50008BE891E10E945B724091891150918A111A
:104B6000BE01635F7E4F85E891E10E945B7288E23F
:104B7000EAEBFBE0DE01A75EBE4F01900D928A9545
:104B8000E1F78CE390E0A0E0B0E0CE5BDE4F8883FD
:104B90009983AA83BB83C254D140CF5BDE4F188276
:104BA000C154D14084EE98E3AEE8B2E4C05ADE4F7F
:104BB00088839983AA83BB83C056D14084EE98E34F
:104BC000AEE8B1E4CC59DE4F88839983AA83BB83D6
:104BD000C456D140C859DE4F19830883C856D14006
:104BE00080E590E0C659DE4F99838883CA56D1404C
:104BF00083E090E0C059DE4F99838883C057D1404D
:104C000088E390E0CE58DE4F99838883C257D14025
:104C100084EF91E09093670280936602BE016E5B21
:104C20007F4F0E94A40864EF71E080E090E00E9452
:104C3000817969E176E0CE0181960E94B175CE015D
:104C400081960E94E915CE0181960E942475CE01BD
:104C50008D960E942475CE0187960E942475E89651
:104C60000FB6F894DEBF0FBECDBFDF91CF911F917D
:104C70000F91FF90EF9008959F92AF92BF92CF92C5
:104C8000DF92EF92FF920F931F93CF93DF93CDB7F5
:104C9000DEB7C859D1090FB6F894DEBF0FBECDBF3D
:104CA0005C017B016A0161E970E1CE0189579F4F88
:104CB0000E94C3756AE674E08E010F5F1F4FC80142
:104CC0000E94C375B801CE0189579F4F0E940E7490
:104CD000982EC8010E942475911014C06AE674E0F1
:104CE000C8010E94C375BE0169577F4FC8010E9469
:104CF0003F74BC01CE0189579F4F0E94D474C801F4
:104D00000E942475B501CE0183579F4F0E94C37541
:104D10006AE874E0E114F10471F068E974E021E0FC
:104D2000E216F10441F063EA74E032E0E316F104C4
:104D300011F06BEA74E0CE0189579F4F0E949E7478
:104D400060E0CE0189579F4F0E947C74B601C80174
:104D50000E94BA756AE0C8010E949074BC01CE013D
:104D60008D569F4F0E94BA75C8010E942475C55781
:104D7000DF4F48815981CB58D040B801CE018957C7
:104D80009F4F0E945B728091590C882399F163EBCD
:104D900074E0CE018F579F4F0E94C375CE018F578D
:104DA0009F4F0E940016CE018F579F4F0E9424757F
:104DB000BE0169577F4FCE018F579F4F0E94BA7532
:104DC000CE018F579F4F0E940016CE018F579F4FE5
:104DD0000E942475B801CE018F579F4F0E94C37562
:104DE000CE018F579F4F0E940016CE018F579F4FC5
:104DF0000E942475CC56DF4F8881C459D0408F93D0
:104E0000CD56DF4F8881C359D0408F93C257DF4FB3
:104E10008881CE58D0408F93C357DF4F8881CD58BB
:104E2000D0408F9383EC94E09F938F938AE1E82E98
:104E30008AE0F82EFF92EF920E944CB140913E0220
:104E400050913F0266EE7BE08AE190E10E946C1097
:104E50000FB6F894DEBF0FBECDBF019709F07CC03E
:104E60001F930F9389EC94E09F938F9300E21BE0D4
:104E70001F930F930E944CB1B8018AE190E10E9408
:104E8000E07686EE9BE09F938F938AED94E09F936C
:104E90008F931F930F930E944CB1B8018AE190E168
:104EA0000E94E0766AE174E08AE190E10E941E7758
:104EB00063EC79E08AE190E10E942476F7010190A9
:104EC0000020E9F7CF018B519A409F938F9383EE97
:104ED00094E09F938F931F930F930E944CB1B8015E
:104EE0008AE190E10E94E076B7018AE190E10E94B8
:104EF000F47662E370E080E090E00E9481798AE1DC
:104F000090E10E9459120FB6F894DEBF0FBECDBFDC
:104F100011E0CE018D569F4F0E942475CE0183571C
:104F20009F4F0E942475CE0189579F4F0E94247580
:104F3000812FC856DF4F0FB6F894DEBF0FBECDBF2E
:104F4000DF91CF911F910F91FF90EF90DF90CF9065
:104F5000BF90AF909F9008956DE574E0CE018F579C
:104F60009F4F0E94B175CE018F579F4F0E94E91548
:104F7000CE018F579F4F0E94247569E674E0CE01E1
:104F80008F579F4F0E94B175CE018F579F4F0E9440
:104F90000016CE018F579F4F0E9424756AE17AE078
:104FA000CE018F579F4F0E94C375CE018F579F4FE1
:104FB0000E94E915CE018F579F4F0E94247510E083
:104FC000A8CFEF92FF920F931F93CF93DF93CDB7AC
:104FD000DEB768970FB6F894DEBF0FBECDBF81E095
:104FE00080934F0C0E9426918C0160ED77E080E069
:104FF00090E00E9481798BE0E82EF12C0D7F01304A
:10500000110571F481E0E81AF10851F00E9426912F
:105010008C0160ED77E080E090E00E948179EECF36
:105020000E945C927C0168EE73E080E090E00E9458
:1050300081790BE010E0EF2899F40150110981F01B
:1050400060ED77E080E090E00E9481790E945C92C0
:105050007C0168EE73E080E090E00E948179EBCF04
:1050600088ED9EE00E94ED1110924F0C0E94C82026
:1050700063EC78E0CE0107960E94C37568E975E09D
:10508000CE010D960E94B175CE0143960E943D72ED
:10509000888D1F928F938F891F928F938E891F9275
:1050A0008F938D891F928F9382E794E09F938F93C4
:1050B00080E29BE09F938F930E944CB160E27BE083
:1050C000CE0101960E94C375BE016F5F7F4FCE0176
:1050D00007960E94EB74CE0101960E942475BE01D2
:1050E000635F7F4FCE0101960E94BA75CE01019693
:1050F0000E940016CE0101960E942475BE01695FD0
:105100007F4FCE0101960E94BA75CE0101960E9492
:10511000E915CE0101960E942475BE01695F7F4F9B
:10512000CE0101960E94BA75AE014F5F5F4F63E0FA
:1051300070E080E092E00E943C26182FCE0101969C
:105140000E9424750FB6F894DEBF0FBECDBF1111BB
:105150002BC06EE875E0CE0101960E94B175CE01BC
:1051600001960E940016CE0101960E942475BE0190
:10517000635F7F4FCE0101960E94BA75CE01019602
:105180000E940016CE0101960E94247569EE7FE010
:10519000CE0101960E94BA75CE0101960E94E915D2
:1051A000CE0101960E942475CE010D960E942475B1
:1051B000CE0107960E94247568960FB6F894DEBF5C
:1051C0000FBECDBFDF91CF911F910F91FF90EF9058
:1051D00008957F928F929F92AF92BF92CF92DF926B
:1051E000EF92FF920F931F93CF93DF93CDB7DEB76C
:1051F00062970FB6F894DEBF0FBECDBF6BE775E0C8
:10520000CE0101960E94B175CE0101960E94E9156A
:10521000CE0101960E94247504E010E03CEEC32EFE
:105220003AE0D32E40E3E42E53EEB52E66E0A62EF0
:105230007CEE972EE1E3FE2EFEE48F2EA4E37A2E81
:1052400068EB72E28CEB9FE00E94790CF6018E2DE8
:1052500011928A95E9F7B092EC0AA092EE0A909228
:10526000EF0AF092F80A8092F90AF092FA0A709224
:10527000FB0A60E472E0CE0101960E9442774BE7A0
:1052800050E0BE016F5F7F4F8CEB9FE00E94390DB5
:1052900040E350E06CEE7AE08CEB9FE00E94D10C92
:1052A0008CEB9FE00E94070D68EE73E080E090E0D9
:1052B0000E9481798CEB9FE00E94290B892B09F0D9
:1052C0004FC00150110909F07CC080911C0B9091D6
:1052D0001D0BA0911E0BB0911F0B892B8A2B8B2BC2
:1052E00009F089C063EC78E087E090E10E940773E1
:1052F00067E070E1CE0101960E94BA75AE014F5F82
:105300005F4F70E060E084E792E00E943C26182F37
:10531000CE0101960E94247511110EC063E675E05E
:10532000CE0101960E94B175CE0101960E94E91549
:10533000CE0101960E94247562960FB6F894DEBFE6
:105340000FBECDBFDF91CF911F910F91FF90EF90D6
:10535000DF90CF90BF90AF909F908F907F900895F7
:1053600040E350E06CEE7AE08CEB9FE00E94E00AB4
:105370006091140B7091150B76276727762790E0C4
:1053800080E0CB01772766270091160B1091170B51
:1053900010270127102730E020E0602B712B822B93
:1053A000932B7E508A4A93480E94F37B0E94187C7C
:1053B00060931C0B70931D0B80931E0B90931F0B1F
:1053C00084CF68EE73E080E090E00E9481794091A4
:1053D0001C0B50911D0B60911E0B70911F0B2AE04E
:1053E0008CE39DE00E94337663EC79E08CE39DE0F2
:1053F0000E94247625CF68EE73E080E090E00E9462
:1054000081790E94187C6093460C7093470C8093BE
:10541000480C9093490C0E94187C6093400C709348
:10542000410C8093420C9093430CCE0101960E9454
:10543000821BCE0101960E94E915CE0101960E94C1
:1054400024750E94B27DBC01CE0107960E94AB1963
:1054500060E474E0CE0107960E949E740E94AA7DCB
:10546000BC01CE0101960E94AB19BE016F5F7F4F58
:10547000CE0107960E94A874CE0101960E94247561
:1054800060E474E0CE0107960E949E740E94A07DA5
:10549000BC01CE0101960E94AB19BE016F5F7F4F28
:1054A000CE0107960E94A874CE0101960E94247531
:1054B00068EF74E0CE0101960E94C375BE01695F7A
:1054C0007F4FCE0101960E943F74BC01CE010D9624
:1054D0000E94BA754AE050E06FEF7FEFCE010D9663
:1054E0000E943220CE010D960E942475CE010196B5
:1054F0000E942475CE0107960E94247568EE73E021
:1055000080E090E00E9481790E94C27DBC01CE01C2
:105510000D960E94AB190E94BA7DBC01CE01019686
:105520000E94AB196FEA76E0CE0107960E94C37520
:10553000BE016F5F7F4FCE0107960E943F74BC0192
:10554000CE010D960E94A874CE0107960E94247584
:10555000CE0101960E9424750E94187C0E94A77CAF
:105560006091210C70E0CE0101960E94AB196FEAA8
:1055700076E0CE0107960E94C375BE016F5F7F4F34
:10558000CE0107960E943F74BC01CE010D960E9489
:10559000A874CE0107960E942475CE0101960E9440
:1055A00024756EEF74E0CE0101960E94C375BE01B2
:1055B000635F7F4FCE0101960E943F74BC01CE0114
:1055C00007960E94BA754AE050E06FEF7FEFCE0178
:1055D00007960E943220CE0107960E942475CE01C4
:1055E00001960E942475CE010D960E94247568EEE6
:1055F00073E080E090E00E948179CE0101960E94E4
:10560000011B4AE050E06FEF7FEFCE0101960E9450
:1056100032208ECECF92DF92EF92FF920F931F93A4
:10562000CF93DF93CDB7DEB768970FB6F894DEBFA0
:105630000FBECDBF63EC78E0CE0143960E94C375E8
:105640006DE677E0CE0101960E94B175CE0101961C
:105650000E940016CE0101960E94247565E871E152
:10566000CE0101960E94BA75CE0101960E94E915FD
:10567000CE0101960E9424756DE577E0CE0101967A
:105680000E94B175CE0101960E940016CE010196CE
:105690000E9424756CA17DA1CE0101960E94117318
:1056A000CE0101960E94E915CE0101960E94247553
:1056B00065E477E0CE0101960E94B175CE010196B6
:1056C0000E940016CE0101960E942475CE5ADE4F2C
:1056D00068817981C255D140CE0101960E94117333
:1056E000CE0101960E94E915CE0101960E94247513
:1056F00068E377E0CE0101960E94B175CE01019674
:105700000E940016CE0101960E94247506EF1BE050
:10571000EE24E394F12CCE5ADE4F88819981C25554
:10572000D1408E159F050CF44AC0F8018281938107
:10573000C6979CF164E075E0CE0101960E94C375A6
:10574000CE0101960E940016CE0101960E9424759A
:10575000F8016281738166537109CE0101960E943E
:105760001173CE0101960E940016CE0101960E948F
:1057700024756FEE75E0CE0101960E94C375CE01CF
:1057800001960E940016CE0101960E942475FFEF3B
:10579000EF1AFF0A0E5F1F4FBECF6CE676E0CE0118
:1057A00001960E94C375CE0101960E940016CE019B
:1057B00001960E942475F80162817381CECF6FEE4D
:1057C00075E0CE0101960E94C375CE0101960E943C
:1057D000E915CE0101960E94247569E277E0CE01B9
:1057E00001960E94B175CE0101960E940016CE016D
:1057F00001960E9424756091B50B7091B60BCE0195
:1058000001960E941173CE0101960E940016CE01EE
:1058100001960E9424756FEE75E0CE0101960E94FC
:10582000C375CE0101960E940016CE0101960E941A
:1058300024756091B70B7091B80BCE0101960E9450
:105840001173CE0101960E94E915CE0101960E94C6
:10585000247562E177E0CE0101960E94B175CE0118
:1058600001960E940016CE0101960E942475BE0189
:10587000605D7F4FCE0101960E94C375CE010196F7
:105880000E940016CE0101960E9424756FEE75E00D
:10589000CE0101960E94C375CE0101960E940016AA
:1058A000CE0101960E942475BE016C5C7F4FCE0133
:1058B00001960E94C375CE0101960E94E915CE01A2
:1058C00001960E94247562E077E0CE0101960E9465
:1058D000B175CE0101960E94E915CE0101960E9494
:1058E00024758E010C5D1F4FEE24E394F12C6801AA
:1058F00088E0C80ED11C8CA19DA18E159F050CF4CB
:1059000049C0B701CE0107960E9411736BE777E09B
:10591000CE0101960E94C375BE01695F7F4FCE0123
:1059200001960E943F74BC01CE010D960E94BA758B
:10593000CE010D960E940016CE010D960E94247590
:10594000CE0101960E942475CE0107960E9424750F
:105950006FEA76E0CE0101960E94C375CE010196F2
:105960000E940016CE0101960E942475B801645E63
:105970007F4FCE0101960E94C375CE0101960E9411
:10598000E915CE0101960E942475EFEFEE1AFE0A8A
:105990008601ADCF61EF76E0CE0101960E94B17530
:1059A000CE0101960E940016CE0101960E94247538
:1059B0007E01F2EBEF1AFEEFFF0A10E000E0F701C4
:1059C00061917F0170E0CE0101960E941173CE01BA
:1059D00001960E940016CE0101960E9424750330A4
:1059E000110571F06EEC78E0CE0101960E94C3754E
:1059F000CE0101960E940016CE0101960E942475E8
:105A00000F5F1F4F04301105D1F66FEE75E0CE0128
:105A100001960E94C375CE0101960E94E915CE0140
:105A200001960E942475C45BDE4F68817981CC5455
:105A3000D140072E000C880B990B0E94B0AB9B0144
:105A4000AC010E9470AE882341F080E590E0C45B19
:105A5000DE4F99838883CC54D140C45BDE4F88816C
:105A60009981CC54D14090933F0280933E0267EDE0
:105A700076E0CE0101960E94B175CE0101960E949A
:105A80000016CE0101960E94247566EE7BE0CE01E1
:105A900001960E94C375CE0101960E940016CE01A8
:105AA00001960E94247565ED76E0CE0101960E9474
:105AB000B175CE0101960E940016CE0101960E949A
:105AC000247560913E0270913F02CE0101960E94C2
:105AD0001173CE0101960E94E915CE0101960E9434
:105AE000247566EC76E0CE0101960E94B175CE0178
:105AF00001960E940016CE0101960E942475BE01F7
:105B00006C5A7F4FCE0101960E94C375CE0101965B
:105B10000E94E915CE0101960E94247566E075E0A9
:105B2000CE0101960E94C375CE0101960E94001617
:105B3000CE0101960E942475BE0164587F4FCE01AC
:105B400001960E94C375CE0101960E94E915CE010F
:105B500001960E942475C052DF4F88819981C05EF2
:105B6000D040892B71F46EEB76E0CE0101960E9455
:105B7000B175CE0101960E94E915CE0101960E94F1
:105B80002475C052DF4F88819981C05ED040019753
:105B900071F464EB76E0CE0101960E94B175CE01FE
:105BA00001960E94E915CE0101960E942475C0520B
:105BB000DF4F88819981C05ED040029771F46BEA13
:105BC00076E0CE0101960E94B175CE0101960E9449
:105BD000E915CE0101960E94247565EA76E0CE01B2
:105BE00001960E94B175CE0101960E940016CE0169
:105BF00001960E942475CE51DF4F68817981C25E83
:105C0000D040CE0101960E941173CE0101960E94F0
:105C1000E915CE0101960E9424756CE976E0CE016B
:105C200001960E94B175CE0101960E940016CE0128
:105C300001960E942475CC5ADE4F88819981C45503
:105C4000D140C6970CF41FC164E075E0CE01019607
:105C50000E94C375CE0101960E940016CE010196E6
:105C60000E942475CC5ADE4F68817981C455D14099
:105C700066537109CE0101960E941173CE010196FF
:105C80000E94E915CE0101960E9424754091380CBE
:105C90005091390C60913A0C70913B0C21E0CE018F
:105CA00007960E942C7561E175E0CE0101960E9475
:105CB000C375BE01695F7F4FCE0101960E943F749C
:105CC0006CE175E00E942974BC01CE010D960E9422
:105CD000BA75CE010D960E94E915CE010D960E946F
:105CE0002475CE0101960E942475CE0107960E946C
:105CF00024754091340C5091350C6091360C7091A4
:105D0000370C21E0CE0107960E942C7561E275E008
:105D1000CE0101960E94C375BE01695F7F4FCE011F
:105D200001960E943F746CE175E00E942974BC01E9
:105D3000CE010D960E94BA75CE010D960E94E9150E
:105D4000CE010D960E942475CE0101960E94247505
:105D5000CE0107960E9424756EE776E0CE0101968B
:105D60000E94B175CE0101960E940016CE010196E7
:105D70000E9424754091290250912A0260912B02C1
:105D800070912C0225E0CE0101960E942C75CE0167
:105D900001960E94E915CE0101960E94247564E6E1
:105DA00076E0CE0101960E94B175CE0101960E9467
:105DB0000016CE0101960E94247540912502509153
:105DC0002602609127027091280225E0CE010196FB
:105DD0000E942C75CE0101960E94E915CE01019614
:105DE0000E94247564E576E0CE0101960E94B175AB
:105DF000CE0101960E940016CE0101960E942475E4
:105E000060916E0270916F02CE0101960E94117333
:105E1000CE0101960E94E915CE0101960E942475DB
:105E200062E476E0CE0101960E94B175CE01019642
:105E30000E940016CE0101960E942475C65BDE4FBB
:105E400068817981CA54D140CE0101960E941173B4
:105E5000CE0101960E94E915CE0101960E9424759B
:105E6000CE0143960E94247568960FB6F894DEBF63
:105E70000FBECDBFDF91CF911F910F91FF90EF909B
:105E8000DF90CF9008956CE676E0CE0101960E94F7
:105E9000C375CE0101960E940016CE0101960E94A4
:105EA0002475CC5ADE4F68817981C455D140E2CE49
:105EB0002F923F924F925F926F927F928F929F921A
:105EC000AF92BF92CF92DF92EF92FF920F931F9308
:105ED000CF93DF93CDB7DEB7EC970FB6F894DEBF64
:105EE0000FBECDBF3C018B0170E060E00E94DD730E
:105EF0008F8F63EC78E0CE0149960E94C375809144
:105F00006E0290916F02019709F07AC082E090E0F2
:105F10000E945E7C88E090E09093240280932302AC
:105F200089E090E090932202809321028091B30B4C
:105F30009091B40B9093B20B8093B10B80911D02A2
:105F400090911E02A0911F02B0912002809319022D
:105F500090931A02A0931B02B0931C028091350209
:105F600090913602A0913702B091380280933902A5
:105F700090933A02A0933B02B0933C028091B00B05
:105F80008093AF0B8091AB0B9091AC0BA091AD0BBC
:105F9000B091AE0B8093A70B9093A80BA093A90B85
:105FA000B093AA0B8AE390E09093180280931702B3
:105FB0008091380C9091390CA0913A0CB0913B0C27
:105FC0008093E20B9093E30BA093E40BB093E50B6B
:105FD00080911502909116029093140280931302FF
:105FE0008091290290912A02A0912B02B0912C025B
:105FF00080932D0290932E02A0932F02B093300233
:1060000080916E0290916F02029709F07AC083E04E
:1060100090E00E945E7C8AE090E09093240280935E
:1060200023028BE090E090932202809321028091E2
:10603000A50B9091A60B9093B20B8093B10B80911E
:106040000F0290911002A0911102B0911202809360
:10605000190290931A02A0931B02B0931C02809124
:10606000310290913202A0913302B09134028093B8
:10607000390290933A02A0933B02B0933C02809184
:10608000A40B8093AF0B8091A00B9091A10BA091DA
:10609000A20BB091A30B8093A70B9093A80BA09396
:1060A000A90BB093AA0B8BE390E090931802809316
:1060B00017028091340C9091350CA091360CB09160
:1060C000370C8093E20B9093E30BA093E40BB09317
:1060D000E50B80910D0290910E0290931402809333
:1060E00013028091250290912602A0912702B0917F
:1060F000280280932D0290932E02A0932F02B0933A
:1061000030022F8D2335C1F41092B20B1092B10BD7
:106110008091B90B882371F068E275E0CE01019699
:106120000E94C375CE0101960E94E915CE01019629
:106130000E942475E12CFCC0C8010197029708F069
:1061400038C281E090E0A0E0B0E080931902909323
:106150001A02A0931B02B0931C02D30114968D91D6
:106160009C91029748F141E050E0B301CE010196C5
:106170000E949F19BE016F5F7F4FCE0149960E941A
:10618000EB74CE0101960E942475CE014996013030
:10619000110581F50E946A7320E030E040E251E48D
:1061A0000E940FAC0E9435AE6093190270931A02E0
:1061B00080931B0290931C02BF8D81E090E090932E
:1061C000B20B8093B10BB13401F58091B90B8823E8
:1061D00009F4B0CF6DE275E0CE0101960E94C3755F
:1061E000CE0101960E94E915CE0101960E94247508
:1061F000E12C6BC00E946A7320912D0230912E0217
:1062000040912F0250913002CBCFEF8DE63409F050
:1062100075C160E0809121020E940E7864E670E012
:1062200080E090E00E94817961E0809123020E94E9
:106230000E7864E670E080E090E00E94817960E092
:10624000809121020E940E7864E670E080E090E088
:106250000E94817961E0809123020E940E7864E6B9
:1062600070E080E090E00E94817902301105C1F475
:10627000CE0149960E946A739B01AC016091E20BCA
:106280007091E30B8091E40B9091E50B0E9456AD69
:106290006093E20B7093E30B8093E40B9093E50B18
:1062A0008091B90B882371F066E375E0CE01019609
:1062B0000E94C375CE0101960E940016CE01019680
:1062C0000E942475EE24E394F12C8091B90B88236D
:1062D00079F14091190250911A0260911B0270915C
:1062E0001C022AE0CE0101960E946275BE016F5F1A
:1062F0007F4FCE0107960E94BA756AE475E0CE0121
:1063000007960E942974BC01CE010D960E94BA75B1
:10631000CE010D960E94E915CE010D960E942475BE
:10632000CE0107960E942475CE0101960E94247525
:106330008091190290911A02A0911B02B0911C0247
:10634000181619061A061B060CF0E7C53F8D3634E1
:1063500009F4EFC4323509F4F0C460E08091210201
:106360000E940E7864E670E080E090E00E948179FF
:106370006E2D809123020E940E7864E670E080E02A
:1063800090E00E9481796091B10B809121020E947E
:106390000E7861E070E080E090E00E94817960E03A
:1063A000809121020E940E7868EC70E080E090E01D
:1063B0000E948179C12CD12C7601C394809119025D
:1063C00090911A02A0911B02B0911C02C816D90626
:1063D000EA06FB060CF0B3C46091B10B8091210278
:1063E0000E940E7861E070E080E090E00E94817988
:1063F00060E0809121020E940E78609139027091D4
:106400003A0280913B0290913C020E9481798091F6
:10641000390290913A02A0913B02B0913C020B9755
:10642000A105B1050CF464C060912D0270912E029B
:1064300080912F02909130029B01AC010E9457ADD8
:106440000E9435AE9B01AC01C701B6010E9415AD9B
:10645000672B682B692B09F04BC0023011050CF437
:1064600047C065EA75E088E99FE00E94AF74C70104
:10647000B6010E94B0AB20912D0230912E024091C6
:106480002F02509130020E94C3ADAB01BC0120E04D
:10649000CE0107960E942C7568E97FE0CE01019637
:1064A0000E94BA75BE01695F7F4FCE0101960E94BE
:1064B0003F746CE175E00E942974BC0188E99FE09B
:1064C0000E94D474CE0101960E942475CE010796D5
:1064D0000E94247568E97FE0CE0101960E94BA759A
:1064E000CE0101960E940721CE0101960E942475DB
:1064F0004FEFC41AD40AE40AF40A60CFFF8DF235D4
:1065000009F076CE60E0809121020E940E7864E668
:1065100070E080E090E00E94817960E08091230249
:106520000E940E7864E670E080E090E00E9481793D
:1065300060E0809121020E940E7864E670E080E0C5
:1065400090E00E94817960E0809123020E940E78A1
:1065500064E670E080E090E00E94817902301105ED
:10656000C1F4CE0149960E946A739B01AC0160910F
:10657000E20B7091E30B8091E40B9091E50B0E948C
:1065800057AD6093E20B7093E30B8093E40B909311
:10659000E50B8091B90B882309F4CCCD60E475E05C
:1065A000CE0101960E94C375CE0101960E9400168D
:1065B0001BCE0115110521F00330110509F0BACDEC
:1065C00080916E0290916F0220E137E240E050E04E
:1065D0008130910521F420E43CE940E050E02EA711
:1065E0003FA748AB59AB21E030E03093B20B20938A
:1065F000B10B30935D0220935C02029759F4033093
:10660000110541F480915F119091601190935D02AA
:1066100080935C0240915C0250915D025DA74CA7A3
:10662000551F5527551F5AAB81E090E090935D02AE
:1066300080935C0260E0809121020E940E7864E603
:1066400070E080E090E00E9481796AA98091230245
:106650000E940E7864E670E080E090E00E9481790C
:1066600060E0809121020E940E7864E670E080E094
:1066700090E00E9481796AA9809123020E940E789D
:1066800064E670E080E090E00E9481798FEF9FEFF8
:106690009093140280931302812C912C540118A61C
:1066A00019A61AA61BA61CA21DA21EA21FA218A2F2
:1066B00019A21AA21BA2212C312C21011FAA18AE4B
:1066C00019AE1AAE1BAA1CAA1DAA1EAA61E08091CF
:1066D00021020E940E7861E070E080E090E00E946C
:1066E000817960E0809121020E940E7861E070E083
:1066F00080E090E00E948179C501B40126E030E09D
:1067000040E050E00E9415AD672B682B692B09F023
:10671000F8C0A2E0B0E0BCAFABAFC12CD12C760189
:1067200080911702863308F0865320917B00982FC2
:106730009870277F922B90937B0087708064809362
:106740007C0080917A00806480937A0080917A0046
:1067500086FDFCCF8091780060917900762F682FBC
:10676000072E000C880B990B0E94B0AB9B01AC016B
:10677000C701B6010E9457AD6B017C0162E070E079
:1067800080E090E00E9481792BAD3CAD2130310555
:1067900009F0ADC020E030EC4FEF54E4C701B60182
:1067A0000E94C3AD6B017C018091B90B882399F1E4
:1067B0002DEC3CEC4CE45EE3C701B6010E946BAEED
:1067C00087FD29C022E0B701A601CE0107960E94ED
:1067D0002C7561E575E0CE0101960E94C375BE017E
:1067E000695F7F4FCE0101960E943F74BC01CE01CC
:1067F0000D960E94BA75CE010D960E94E915CE0144
:106800000D960E942475CE0101960E942475CE013A
:1068100007960E9424752AE939E949E95EE3C70130
:10682000B6010E946BAE87FD13C0211431044104F0
:10683000510411F4140125018CA19DA1AEA1BFA1A9
:10684000892B8A2B8B2B21F48CA29DA2AEA2BFA2F6
:106850002DEC3CEC4CE45EE3C701B6010E94A9AB11
:1068600018160CF449C0211431044104510409F4F0
:1068700048C028A139A14AA15BA1232B242B252B99
:1068800069F488A599A5AAA5BBA5892B8A2B8B2B72
:1068900009F401C188A299A2AAA2BBA228A139A188
:1068A0004AA15BA1221633064406550654F5809191
:1068B00013029091140297FFF3C0109214021092E9
:1068C0001302220E331E441E551ED201C101B5957E
:1068D000A795979587958FAB98AFA9AFBAAF18A238
:1068E00019A21AA21BA2212C312C21010AC0E1E01D
:1068F000F0E0FCAFEBAF14CF21143104410451049C
:1069000069F6E0901302F090140292E0E916F104A7
:1069100034F4F7FCE1C00330110509F0DDC08EA4AA
:106920009FA4A8A8B9A8AAE08A0E911CA11CB11C1A
:106930008EA59FA5A8A9B9A988169906AA06BB067F
:106940000CF4C4CEE2E0EE16F1040CF479C06BA9AD
:106950007CA98DA99EA92FA938AD49AD5AAD621B5E
:10696000730B840B950B0E94B0AB4B015C01B7011C
:10697000FF0C880B990B0E94B0AB9B01AC01C501C9
:10698000B4010E94C3AD20E030E044EB53E40E9428
:10699000C3AD6B017C01C0922D02D0922E02E09219
:1069A0002F02F092300220E030E040E85FE30E94E6
:1069B0006BAE87FDABC080916E0290916F0281300B
:1069C000910509F08FC0C0925711D0925811E092F2
:1069D0005911F0925A11C0922902D0922A02E092E3
:1069E0002B02F0922C0268EC75E0CE0101960E9419
:1069F000B175CE0101960E940016CE0101960E944B
:106A0000247540912D0250912E0260912F027091B9
:106A1000300225E0CE0101960E942C75CE01019630
:106A20000E94E915CE0101960E94247584EF91E041
:106A3000909367028093660269E370E10E94A40864
:106A40000330110531F03AA9E32E0115110509F0C3
:106A50006FCCC3010E946A736B017C01C092E20B90
:106A6000D092E30BE092E40BF092E50B20E030E0F3
:106A700044EB53E4C701B6010E946BAE87FD6AC0C8
:106A800020E030E044EB53E4C701B6010E9456AD6C
:106A90006B017C01EBCF88A699A6AAA6BBA6FACE6D
:106AA0000115110509F02DCF0196909314028093E2
:106AB000130228A139A14AA15BA1220E331E441E54
:106AC000551ED201C101B595A795979587958BABBA
:106AD0009CABADABBEAB03CFBFEF8B1A9B0AAB0A2F
:106AE000BB0A26CF029709F07ECFC0925B11D092ED
:106AF0005C11E0925D11F0925E11C0922502D0927D
:106B00002602E0922702F09228026DCF6CEA75E02F
:106B1000CE0101960E94B175CE0101960E94001629
:106B2000CE0101960E94247540912D0250912E02B3
:106B300060912F027091300225E0CE0101960E94F3
:106B40002C75CE0101960E94E915CE0101960E9496
:106B5000247576CF20E030E0A901C701B6010E947C
:106B6000A9AB87FF0BC020E030E044EB53E4C70142
:106B7000B6010E9457AD6B017C01ECCFC092A70B10
:106B8000D092A80BE092A90BF092AA0B48A459A4AA
:106B90006AA47BA48CA19DA1AEA1BFA1481A590AE9
:106BA0006A0A7B0A01151105D9F41092A70B1092FD
:106BB000A80B1092A90B1092AA0BACA5BDA5C12CD5
:106BC000D12C7601C394812C912C5401B7FF1CC0A9
:106BD000812C912C5401CC24CA94DC2C760114C055
:106BE000ECA5FDA5C12CD12C7601C394F7FF04C000
:106BF000CC24CA94DC2C76018090A70B9090A80B33
:106C0000A090A90BB090AA0B20912D0230912E02DA
:106C100040912F0250913002C501B4010E940FAC87
:106C20004B015C01A3019201C701B6010E94E3ACD4
:106C30000E94B0AB20E030E040E05FE30E940FAC88
:106C40009B01AC01C501B4010E9456AD0E9435AE56
:106C50006093190270931A0280931B0290931C0296
:106C60008091B90B882309F441C02AE048A559A5B1
:106C70006AA57BA5CE010D960E9462752AE04CA103
:106C80005DA16EA17FA1CE0107960E94627568E5A5
:106C900075E0CE0101960E94C375BE01695F7F4F0A
:106CA000CE0101960E943F746FEE75E00E94297438
:106CB000BE01635F7F4F0E943F74BC01CE014396CB
:106CC0000E94BA75CE0143960E94E915CE01439603
:106CD0000E942475CE0101960E942475CE0107966C
:106CE0000E942475CE010D960E9424758091190290
:106CF00090911A02A0911B02B0911C02B7FF15C01F
:106D0000B095A095909581959F4FAF4FBF4F8093C1
:106D1000190290931A02A0931B02B0931C02EE2456
:106D2000E394F12CF6E4FF8F03CBE12C22E52F8FC7
:106D3000FFCAEE24E394F12C10CBE12C0ECB0230F1
:106D4000110524F40115110509F0DFC061E080E0B0
:106D50000E94C57F0230110524F40115110509F0C8
:106D60009CC0C090E20BD090E30BE090E40BF0905D
:106D7000E50B20E030E044EB53E4C701B6010E948C
:106D80006BAE87FD0BC020E030E044EB53E4C7015D
:106D9000B6010E9456AD6B017C01EBCF20E030E0E4
:106DA000A901C701B6010E94A9AB87FF0BC020E073
:106DB00030E044EB53E4C701B6010E9457AD6B01CC
:106DC0007C01ECCFC092E20BD092E30BE092E40B9B
:106DD000F092E50B80916E0290916F020197B1F4F1
:106DE00061E175E088E99FE00E9407738091E20B02
:106DF0009091E30BA091E40BB091E50B8093380CDC
:106E00009093390CA0933A0CB0933B0C80916E0296
:106E100090916F020297B1F461E275E088E99FE01A
:106E20000E9407738091E20B9091E30BA091E40B19
:106E3000B091E50B8093340C9093350CA093360CF5
:106E4000B093370C4091E20B5091E30B6091E40B4F
:106E50007091E50B20E0CE0107960E942C7568E941
:106E60007FE0CE0101960E94BA75BE01695F7F4F37
:106E7000CE0101960E943F746DE175E00E94297475
:106E8000BC0188E99FE00E94D474CE0101960E9463
:106E90002475CE0107960E9424750130110539F53D
:106EA0004091190250911A0260911B0270911C02CC
:106EB00021E0CE0107960E94627560E675E0CE0182
:106EC00001960E94C375BE01695F7F4FCE01019696
:106ED0000E943F74BC0188E99FE00E94D474CE01F7
:106EE00001960E942475CE0107960E94247568E9D8
:106EF0007FE0CE0101960E94BA75CE0101960E94F4
:106F00000721CE0101960E94247510921902109259
:106F10001A0210921B0210921C0280916E02909134
:106F20006F028130910509F083C08091B10B90917F
:106F3000B20B9093B40B8093B30B80911902909194
:106F40001A02A0911B02B0911C0280931D02909323
:106F50001E02A0931F02B0932002809139029091EB
:106F60003A02A0913B02B0913C028093350290938B
:106F70003602A0933702B09338028091AF0B809312
:106F8000B00B8091A70B9091A80BA091A90BB09189
:106F9000AA0B8093AB0B9093AC0BA093AD0BB0936B
:106FA000AE0B8091E20B9091E30BA091E40BB091BA
:106FB000E50B8093380C9093390CA0933A0CB09366
:106FC0003B0C8091130290911402909316028093CF
:106FD0001502012B81F480912D0290912E02A09137
:106FE0002F02B09130028093290290932A02A0933D
:106FF0002B02B0932C02CE0149960E942475EC9688
:107000000FB6F894DEBF0FBECDBFDF91CF911F91B9
:107010000F91FF90EF90DF90CF90BF90AF909F9037
:107020008F907F906F905F904F903F902F9008953A
:10703000029709F78091B10B9091B20B9093A60B38
:107040008093A50B8091190290911A02A0911B02C6
:10705000B0911C0280930F0290931002A093110232
:10706000B09312028091390290913A02A0913B02B2
:10707000B0913C028093310290933202A09333028C
:10708000B09334028091AF0B8093A40B8091A70B37
:107090009091A80BA091A90BB091AA0B8093A00B83
:1070A0009093A10BA093A20BB093A30B8091E20B42
:1070B0009091E30BA091E40BB091E50B8093340C1D
:1070C0009093350CA093360CB093370C809113023B
:1070D0009091140290930E0280930D02012B09F0FF
:1070E0008ACF80912D0290912E02A0912F02B09113
:1070F00030028093250290932602A0932702B0933A
:10710000280279CF2F923F924F925F926F927F9297
:107110008F929F92AF92BF92CF92DF92EF92FF92A7
:107120000F931F93CF93DF93CDB7DEB7E3970FB6DF
:10713000F894DEBF0FBECDBF66EB7FE0CE018E962A
:107140000E94BA750EA51FA50115110571F0D80191
:107150008D918D01882349F0082E000C990B0E9417
:10716000C3B0F80131978083F2CF67E675E0CE01B6
:1071700001960E94C375BE016F5F7F4FCE018E9650
:107180000E940E74182FCE0101960E9424751123BF
:1071900009F401C145E050E066EB7FE0CE010196C5
:1071A0000E949F19BE016F5F7F4F82E99FE00E949E
:1071B000EB74CE0101960E94247582E99FE00E9443
:1071C000807360E082E99FE00E947C744091960F9A
:1071D0005091970F61E970E182E99FE00E945B7234
:1071E0006AE674E0CE0101960E94C375BE016F5F2E
:1071F0007F4F82E99FE00E940E74182FCE01019606
:107200000E94247564E574E0111102C069E574E020
:10721000CE0101960E94C37562E97FE0CE0101961E
:107220000E943F74BC0187E991E10E94D474CE01B1
:1072300001960E94247587E991E10E948073409134
:107240009B1150919C114150510967E971E1CE01A8
:1072500001960E949F19BE016F5F7F4F89E791E100
:107260000E94EB74CE0101960E94247589E791E19A
:107270000E9475730E94B0AB9B01AC010E9470AE7E
:10728000882309F448C060919B1170919C11625051
:10729000710987E991E10E94DD73682FCE010196A3
:1072A0000E948F75BE016F5F7F4F89E791E10E9459
:1072B000EB74CE0101960E9424756AE674E0CE015B
:1072C00001960E94C375BE016F5F7F4F89E791E110
:1072D0000E940E74182FCE0101960E94247511236E
:1072E000D1F060919B1170919C116350710987E9F5
:1072F00091E10E94DD73682FCE0101960E948F7587
:10730000BE016F5F7F4F89E791E10E94EB74CE0170
:1073100001960E94247584EF91E090936702809318
:10732000660269E370E10E94A40864E670E080E010
:1073300090E00E94817980913D02882371F066EB94
:107340007FE0CE0101960E94BA75CE0101960E949F
:10735000D51ACE0101960E942475CE018E960E9408
:10736000247581E0E3960FB6F894DEBF0FBECDBF63
:10737000DF91CF911F910F91FF90EF90DF90CF9011
:10738000BF90AF909F908F907F906F905F904F9045
:107390003F902F9008956DE675E0CE0101960E9412
:1073A000C375BE016F5F7F4FCE018E960E940E7433
:1073B000182FCE0101960E942475112309F447C0AD
:1073C00045E050E066EB7FE0CE0101960E949F19F8
:1073D000BE016F5F7F4F82E99FE00E94EB74CE0198
:1073E00001960E94247582E99FE00E94807360E00C
:1073F00082E99FE00E947C744091960F5091970F14
:1074000069E670E182E99FE00E945B7269E670E1E3
:10741000CE014C960E94C3756CE674E0CE010196D5
:107420000E94C375BE01645E7F4FCE0101960E942B
:107430003F74BC0181E991E10E94D474CE010196B0
:107440000E942475CE014C960E94247564CF63E798
:1074500075E0CE0101960E94C375BE016F5F7F4F3C
:10746000CE018E960E940E74182FCE0101960E94B6
:1074700024751123E1F043E050E066EB7FE0CE019C
:1074800001960E949F19BE016F5F7F4F82E99FE0C6
:107490000E94EB74CE0101960E94247562E97FE0A0
:1074A000CE0101960E94BA75CE010196CDCF67E755
:1074B00075E0CE0101960E94C375BE016F5F7F4FDC
:1074C000CE018E960E940E74182FCE0101960E9456
:1074D0002475112301F144E050E066EB7FE0CE011A
:1074E00001960E949F19BE016F5F7F4F82E99FE066
:1074F0000E94EB74CE0101960E94247582E99FE000
:107500000E9475737093F8106093F71070938F0258
:1075100060938E0200CF6CE775E0CE0101960E9469
:10752000C375BE016F5F7F4FCE018E960E940E74B1
:10753000182FCE0101960E942475112309F449C029
:1075400045E050E066EB7FE0CE0101960E949F1976
:10755000BE016F5F7F4F82E99FE00E94EB74CE0116
:1075600001960E94247582E99FE00E9475737093D2
:1075700054116093531184EF91E0909367028093CC
:10758000660269E370E10E94A40864E670E080E0AE
:1075900090E00E9481796BE777E0CE0101960E942E
:1075A000C37566EB7FE0CE0101960E943F74BC017B
:1075B000CE014C960E94BA75CE014C960E94E915F8
:1075C000CE014C960E942475CE0101960E9424752E
:1075D000B2CE62E875E0CE0101960E94C375BE018D
:1075E0006F5F7F4FCE018E960E940E74182FCE01D2
:1075F00001960E9424751123E1F044E050E066EB0F
:107600007FE0CE0101960E949F19BE016F5F7F4F00
:1076100082E99FE00E94EB74CE0101960E942475DE
:1076200082E99FE00E947573709356116093551123
:10763000A2CF67E875E0CE0101960E94C375BE0136
:107640006F5F7F4FCE018E960E940E74182FCE0171
:1076500001960E9424751123A1F044E050E066EBEE
:107660007FE0CE0101960E949F19BE016F5F7F4FA0
:1076700082E99FE00E94EB74CE0101960E9424757E
:1076800084CF6CE875E0CE0101960E94C375BE01FF
:107690006F5F7F4FCE018E960E940E74182FCE0121
:1076A00001960E9424751123A1F047E050E066EB9B
:1076B0007FE0CE0101960E949F19BE016F5F7F4F50
:1076C00082E99FE00E94EB74CE0101960E9424752E
:1076D0002CCE64E975E0CE0101960E94C375BE010F
:1076E0006F5F7F4FCE018E960E940E74182FCE01D1
:1076F00001960E9424751111D8CF6CE975E0CE0176
:1077000001960E94C375BE016F5F7F4FCE018E96BA
:107710000E940E74182FCE0101960E942475112329
:1077200021F081E00E94330800CE66EA75E0CE01C8
:1077300001960E94C375BE016F5F7F4FCE018E968A
:107740000E940E74182FCE0101960E9424751123F9
:1077500019F00E94E127E9CD61E879E0CE010196B8
:107760000E94B175BE016F5F7F4FCE018E960E9461
:107770000E74182FCE0101960E942475112309F46E
:1077800085C066E779E0CE0101960E94B175BE0121
:107790006F5F7F4FCE018E960E940E74182FCE0120
:1077A00001960E942475112309F454C04AE050E068
:1077B00066EB7FE0CE0101960E949F19BE016F5FCC
:1077C0007F4F82E99FE00E94EB74CE0101960E94F8
:1077D000247582E99FE00E9475730E94F37B0E94EA
:1077E000187C6093460C7093470C8093480C9093E0
:1077F000490C0E94187C6093400C7093410C80935C
:10780000420C9093430CCE014C960E94821B6DEA71
:1078100075E0CE0101960E94C375BE01645E7F4F84
:10782000CE0101960E943F74BC01CE0182960E9457
:10783000BA75CE0182960E94E915CE0182960E9409
:107840002475CE0101960E942475CE014C960E94AB
:10785000247571CD4BE050E066EB7FE0CE010196E0
:107860000E949F19BE016F5F7F4F82E99FE00E94D7
:10787000EB74CE0101960E94247582E99FE00E947C
:10788000757360587F488F4F9F4FA7CF63EF76E0A7
:10789000CE0101960E94C375BE016F5F7F4FCE017E
:1078A0008E960E940E74182FCE0101960E942475A8
:1078B000112309F46AC045E050E066EB7FE0CE0199
:1078C00001960E949F19BE016F5F7F4F82E99FE082
:1078D0000E94EB74CE0101960E9424750E94187CD0
:1078E0006093460C7093470C8093480C9093490C1E
:1078F00082E99FE00E947573609370027093710239
:1079000080937202909373026093391170933A11CD
:1079100080933B1190933C11209138112093580C87
:10792000672B682B692B11F41092580C84EF91E0AF
:10793000909367028093660269E370E10E94A40855
:1079400064E670E080E090E00E94817967E679E08B
:10795000CE0101960E94B175CE0101960E940016DB
:10796000CE0101960E9424754091700250917102DF
:107970006091720270917302CE0101960E943D7374
:10798000CE0101960E94E915DBC16EEB75E0CE01D8
:1079900001960E94C375BE016F5F7F4FCE018E9628
:1079A0000E940E74182FCE0101960E942475112397
:1079B000D9F14AE050E066EB7FE0CE0101960E94EB
:1079C0009F19BE016F5F7F4F82E99FE00E94EB74B9
:1079D000CE0101960E94247582E99FE00E94757392
:1079E000613071058105910519F481E080933811AA
:1079F00082E99FE00E947573672B682B692B11F455
:107A000010923811809138118093580C882309F412
:107A1000B2CD0E94187C6093460C7093470C809303
:107A2000480C9093490CA7CD69EC75E0CE01019606
:107A30000E94C375BE016F5F7F4FCE018E960E947C
:107A40000E74182FCE0101960E9424751123A1F007
:107A500048E050E066EB7FE0CE0101960E949F195E
:107A6000BE016F5F7F4F82E99FE00E94EB74CE0101
:107A700001960E9424758FCD62ED75E0CE010196CE
:107A80000E94C375BE016F5F7F4FCE018E960E942C
:107A90000E74182FCE0101960E942475112321F136
:107AA00045E050E066EB7FE0CE0101960E949F1911
:107AB000BE016F5F7F4F82E99FE00E94EB74CE01B1
:107AC00001960E94247582E99FE00E9475736130DF
:107AD000710521F481E08093590C2DCC672B09F0BE
:107AE0002ACC1092590C27CC68ED75E0CE01019696
:107AF0000E94C375BE016F5F7F4FCE018E960E94BC
:107B00000E74182FCE0101960E942475112351F195
:107B100063E070E086EB9FE00E94DD73682FCE018A
:107B200001960E948F75BE016F5F7F4F82E99FE0D3
:107B30000E94EB74CE0101960E94247582E99FE0B9
:107B40000E94807382E99FE00E9475739B0121501F
:107B500031092330310508F0EECB70936811609342
:107B60006711D9CB6CED75E0CE0101960E94C3750B
:107B7000BE016F5F7F4FCE018E960E940E74182F4C
:107B8000CE0101960E942475112309F46AC066E0B3
:107B900070E086EB9FE00E94DD73682FCE010196B6
:107BA0000E948F75BE016F5F7F4F82E99FE00E9448
:107BB000EB74CE0101960E94247582E99FE00E9439
:107BC000807360E082E99FE00E947C7482E99FE01C
:107BD0000E9475736B01CB010197039708F0ABCB43
:107BE00048E050E066EB7FE0CE0101960E949F19CD
:107BF000BE016F5F7F4F82E99FE00E94EB74CE0170
:107C000001960E94247582E99FE00E948073809112
:107C1000960F9091970F0997A8F028E030E050E078
:107C200040E062E97FE0CE0101960E94D875BE0176
:107C30006F5F7F4F82E99FE00E94EB74CE01019657
:107C40000E942475B60113E0660F771F1A95E1F7BD
:107C5000635B7F4E48E050E082E99FE00E945B72E8
:107C60005ACB6FE579E0CE0101960E94B175BE0155
:107C70006F5F7F4FCE018E960E940E74182FCE013B
:107C800001960E942475112309F486C063EC78E004
:107C9000CE0101960E94C37547E050E0BE01625DCF
:107CA0007F4FCE014C960E949F19BE01645E7F4FAC
:107CB000CE0101960E94EB74CE014C960E94247571
:107CC00064E075E0CE014C960E94C375BE01645E0F
:107CD0007F4FCE0101960E940E74182FCE014C9654
:107CE0000E942475112379F141E050E0BE016F5FDD
:107CF0007F4FCE014C960E949F19CE014C960E9458
:107D000075738B010A5C1F4FCE014C960E9424753F
:107D100010936A11009369111093910200939002DD
:107D200084EF91E0909367028093660269E370E1CB
:107D30000E94A40864E670E080E090E00E948179EF
:107D4000CE01019684CD6CE676E0CE014C960E9481
:107D5000C375BE01645E7F4FCE0101960E940E7412
:107D6000182FCE014C960E942475112379F041E022
:107D700050E0BE016F5F7F4FCE014C960E949F196D
:107D8000CE014C960E9475738B01BECFCE01019639
:107D90000E9475738B01BCCF68E579E0CE01019636
:107DA0000E94B175BE016F5F7F4FCE018E960E941B
:107DB0000E74182FCE0101960E942475112309F428
:107DC000AAC062EF75E0CE0101960E94C37546E03D
:107DD00050E0BE016F5F7F4FCE018E960E9482A160
:107DE0008C01CE0101960E942475980146E050E076
:107DF000BE01625D7F4FCE0101960E94D875CE0113
:107E000001960E9475736B01CE0101960E94247544
:107E100063EC78E0CE0101960E94C375A8014F5F24
:107E20005F4FBE01625D7F4FCE014C960E949F194D
:107E3000BE01645E7F4FCE0101960E94EB74CE01BD
:107E40004C960E94247564E075E0CE014C960E9429
:107E5000C375BE01645E7F4FCE0101960E940E7411
:107E6000182FCE014C960E942475112321F141E078
:107E700050E0BE016F5F7F4FCE014C960E949F196C
:107E8000CE014C960E9475738B010A5C1F4FCE0188
:107E90004C960E942475F6013196EE0FFF1FE75CA9
:107EA000FF4E11830083F601EE0FFF1FEA50F44FDF
:107EB0001183008335CF6CE676E0CE014C960E94AC
:107EC000C375BE01645E7F4FCE0101960E940E74A1
:107ED000182FCE014C960E942475112379F041E0B1
:107EE00050E0BE016F5F7F4FCE014C960E949F19FC
:107EF000CE014C960E9475738B01C9CFCE010196BD
:107F00000E9475730091F80B1091F90B0150110943
:107F1000060F171FC0CF69E374E0CE014C960E9494
:107F2000C375BE01645E7F4FCE018E960E940E74B3
:107F300011E0811115C063EE75E0CE0101960E943B
:107F4000C375BE016F5F7F4FCE018E960E940E7487
:107F500011E0811101C010E0CE0101960E9424754C
:107F6000CE014C960E942475112309F411C26FEEC4
:107F700075E0CE014C960E94C3756AEE75E0CE01A5
:107F800001960E94C375AE01445E5F4FBE016F5FF4
:107F90007F4FCE018E960E9489A0CE0101960E944D
:107FA0002475CE014C960E9424756FEE75E0CE01CB
:107FB0004C960E94C3756CEE75E0CE0101960E944E
:107FC000C375AE01445E5F4FBE016F5F7F4FCE0150
:107FD0008E960E9489A0CE0101960E942475CE0142
:107FE0004C960E9424756FEE75E0CE014C960E946F
:107FF000C3756EEE75E0CE0101960E94C375AE01A9
:10800000445E5F4FBE016F5F7F4FCE018E960E9430
:1080100089A0CE0101960E942475CE014C960E9443
:10802000247562EF75E0CE014C960E94C37561EF36
:1080300075E0CE0101960E94C375AE01445E5F4FAC
:10804000BE016F5F7F4FCE018E960E9489A0CE0148
:1080500001960E942475CE014C960E94247562EF11
:1080600075E0CE014C960E94C3756FE178E0CE01B9
:1080700001960E94C375AE01445E5F4FBE016F5F03
:108080007F4FCE018E960E9489A0CE0101960E945C
:108090002475CE014C960E942475CE018E960E94C6
:1080A00080730E94187C60934A0C70934B0C8093F1
:1080B0004C0C90934D0C56E0E52EF12C64E6462EC8
:1080C000512C612C712C22242394312C5701B3E0C4
:1080D000AB0EB11C8AA99BA90197A816B90608F096
:1080E0002AC9B701CE018E960E94DD73682FCE019A
:1080F0004C960E948F756701E2E0CE0ED11CFFEF17
:10810000EF1AFF0A9601A701BE01625D7F4FCE0103
:1081100001960E94D875CE0101960E9475738B015D
:10812000CE0101960E9424750130110521F40091C1
:108130005311109154110330110521F40091551180
:10814000109156116FEE75E0CE0101960E94C37535
:10815000A601BE016F5F7F4FCE018E960E9482A165
:108160006C01CE0101960E94247563EC78E0CE018B
:1081700001960E94C375480181E0881A91081C1479
:108180001D042CF59601A501BE01625D7F4FCE0155
:1081900082960E94D875BE016E5D7F4FCE0101961A
:1081A0000E94EB74CE0182960E94247593E089169A
:1081B000910420F17601AFEFEA1AFA0ACE01019696
:1081C0000E942475CE014C960E9424757FCFA50194
:1081D000BE01625D7F4FCE0182960E949F19BE0153
:1081E0006E5D7F4FCE0101960E94EB74CE018296A8
:1081F0000E942475B3E08B16910400F770E060E0F4
:10820000CE014C960E94DD73823509F061C0CE012B
:1082100001960E947573672B682B692BB1F4F801E6
:10822000EE0FFF1FE952FD4F11821082F801EE0F91
:10823000FF1FEE0FFF1FE154FD4F82E090E0A0E032
:10824000B0E080839183A283B383CE0101960E9424
:1082500075736130710581059105A9F5F801EE0F7F
:10826000FF1FE952FD4F31822082000F111F000FC6
:10827000111FF801E154FD4F80819181A281B381EA
:10828000181619061A061B0624F0408251826282D3
:108290007382CE0101960E9475736230710581056B
:1082A00091053CF0F801E154FD4F608371838283B6
:1082B00093830E94187C01521D4FD8016D937D93CA
:1082C0008D939C9313971C141D040CF473CF76CFDD
:1082D0008634E9F5CE0101960E947573672B682BF1
:1082E000692B39F4F801EE0FFF1FEC5AFD4F118294
:1082F0001082CE0101960E9475736130710581056F
:10830000910539F4F801EE0FFF1FEC5AFD4F318251
:108310002082000F111F000F111FF801E154FD4FC3
:1083200080819181A281B381181619061A061B0655
:1083300024F040825182628273820E94187C015232
:108340001D4FF8016083718382839383BCCF843493
:1083500061F4CE0101960E947573000F111F000F8A
:10836000111FF801EC5BFD4FA0CF843509F0ABCFB6
:10837000CE0101960E947573000F111F000F111F8F
:10838000F801E154FD4F6083718382839383D5CFDD
:1083900062E579E0CE0101960E94B175BE016F5F82
:1083A0007F4FCE018E960E940E74182FCE0101963B
:1083B0000E942475112309F49DC045E050E066EB4E
:1083C0007FE0CE0101960E949F19BE016F5F7F4F33
:1083D00082E99FE00E94EB74CE0101960E94247511
:1083E00082E99FE00E94807360E082E99FE00E9442
:1083F0007C746EEC78E0CE014C960E94C37562E905
:108400007FE0CE0101960E94BA75AE014E5D5F4FCE
:10841000BE01645E7F4FCE0101960E949EA1182F7F
:10842000CE0101960E942475CE014C960E942475BF
:10843000112311F40C949B398E010E5D1F4F53E6EE
:10844000A52E51E1B52E60E4C62E62E0D62EF12CA9
:10845000E12CD8016D918D01F50161935F01D60189
:108460006D936D01CE0101960E9411A0CE0101967F
:108470000E940016CE0101960E942475B3E0EB160F
:10848000F10471F06EEC78E0CE0101960E94C375A4
:10849000CE0101960E940016CE0101960E9424751D
:1084A000EFEFEE1AFE0AF4E0EF16F10491F663EC3A
:1084B00078E0CE0101960E94C375CE0101960E941C
:1084C000E915CE0101960E94247569E370E180915F
:1084D0006602909167020E94A40864E670E080E062
:1084E00090E00E9481796AE379E0CE0101960E94D2
:1084F000B17546CA65E379E0CE0101960E94B17577
:10850000BE016F5F7F4FCE018E960E940E74182FB2
:10851000CE0101960E942475112309F47CC044E029
:1085200050E066EB7FE0CE0101960E949F19BE01EC
:108530006F5F7F4F82E99FE00E94EB74CE0101964E
:108540000E94247582E99FE00E94807360E082E9C6
:108550009FE00E947C744091960F5091970F66EEB9
:108560007BE082E99FE00E945B726EEC78E0CE01D6
:108570004C960E94C37562E97FE0CE0101960E948D
:10858000BA75AE014E5D5F4FBE01645E7F4FCE0196
:1085900001960E949EA1182FCE0101960E9424757B
:1085A000CE014C960E942475112311F40C949B3932
:1085B0008E010E5D1F4F45E6E42E40E1F42E6E0164
:1085C00086E2C80ED11CD8016D918D01F70161932F
:1085D0007F01CE0101960E9411A0CE0101960E945A
:1085E000E915CE0101960E9424750C151D0559F759
:1085F00084EF91E0909367028093660269E370E1F3
:108600000E94A40864E670E080E090E00E94817916
:108610006AE279E06ACF63E279E0CE0101960E94D6
:10862000B175BE016F5F7F4FCE018E960E940E74B2
:10863000182FCE0101960E9424751123F1F146E016
:1086400050E066EB7FE0CE0101960E949F19BE01CB
:108650006F5F7F4F82E99FE00E94EB74CE0101962D
:108660000E94247582E99FE00E9480738091960F9A
:108670009091970F892B11F40C949B3982E99FE01C
:108680000E947573709362116093611170933F0241
:1086900060933E0284EF91E09093670280936602BC
:1086A00069E370E10E94A40864E670E080E090E075
:1086B0000E9481796FE079E018CF68E079E0CE011F
:1086C00001960E94B175BE016F5F7F4FCE018E96FD
:1086D0000E940E74182FCE0101960E94247511235A
:1086E000B9F06BEF78E0CE0101960E94B17544E6D7
:1086F00050E06FEF7FEFCE0101960E940909CE0195
:1087000001960E942475F0E0E0E019950C949B39E5
:1087100063EF78E0CE0101960E94B175BE016F5FF4
:108720007F4FCE018E960E940E74182FCE010196B7
:108730000E942475112301F164EF75E0CE010196CA
:108740000E94C3756FE771E1CE0101960E943F74EC
:10875000BC0188E99FE00E94D474CE0101960E947A
:10876000247568E97FE0CE0101960E94BA75CE01BA
:1087700001960E94E9158DC46CEE78E0CE01019659
:108780000E94B175BE016F5F7F4FCE018E960E9431
:108790000E74182FCE0101960E942475112369F0E2
:1087A0006DED78E088E99FE00E94AF7465E871E1C3
:1087B00088E99FE00E94A874D4CF6FEF75E0CE01E6
:1087C00001960E94C375BE016F5F7F4FCE018E96EA
:1087D0000E940E74182FCE0101960E942475112359
:1087E00031F00E94E92810923D020C949B3968E018
:1087F00076E0CE014C960E94C375BE01645E7F4F49
:1088000086EB9FE00E940E7411E0811115C06DE0AF
:1088100076E0CE0101960E94C375BE016F5F7F4F67
:1088200086EB9FE00E940E7411E0811101C010E000
:10883000CE0101960E942475CE014C960E942475AB
:10884000112309F441C062EF75E0CE0101960E9448
:10885000C3754091BA0F5091BB0F8D819E81481B0B
:10886000590BBE016F5F7F4F86EB9FE00E943BA0DC
:10887000AC014F5F5F4F66EB7FE0CE014C960E94EC
:108880009F19BE01645E7F4F82E99FE00E94EB74F6
:10889000CE014C960E942475CE0101960E9424754B
:1088A00082E99FE00E9475736115710531F481E0E2
:1088B0008093F0020E949D9396CF6130710509F07C
:1088C00092CF1092F002F6CF62E176E0CE010196EF
:1088D0000E94C375BE016F5F7F4FCE018E960E94CE
:1088E0000E74182FCE0101960E942475112309F4ED
:1088F0003BC143E050E066EB7FE0CE0101960E9471
:108900009F19BE016F5F7F4F82E99FE00E94EB7469
:10891000CE0101960E94247562E97FE0CE010196A6
:108920000E94BA75CE0101960E94D51ACE01019619
:108930000E94247584EF91E0909367028093660211
:1089400062E97FE0CE0101960E94BA7560E0CE0137
:1089500001960E949074BC018BE891E10E94D4744E
:10896000CE0101960E94247562E97FE0CE01019656
:108970000E94BA7560E0CE0101960E949074BC011D
:1089800085E891E10E94D474CE0101960E9424757D
:1089900040918F115091901169EF70E18BE891E156
:1089A0000E945B724091891150918A1164E071E1DB
:1089B00085E891E10E945B7269E370E18091660253
:1089C000909167020E94A40866E176E0CE010196CC
:1089D0000E94C37562E97FE0CE0101960E943F7458
:1089E000BC01CE0182960E94BA75CE0101960E940A
:1089F00024758091F5109091F610892B39F4BE0101
:108A00006E5D7F4F8FE99CE00E94FC7668EB7BE017
:108A100080E090E00E9481798091F5109091F610AD
:108A2000029709F087C062E97FE0CE0188960E9434
:108A3000BA756EE176E0CE0101960E94C375CE0153
:108A400001960E94C993CE0101960E94247564EF9D
:108A500071E080E090E00E94817961E276E0CE01F1
:108A600001960E94C375CE0101960E94C993CE0162
:108A700001960E9424756CED75E080E090E00E9404
:108A800081796AE276E0CE0101960E94C375CE013B
:108A900001960E94C993CE0101960E94247564EF4D
:108AA00071E080E090E00E94817968E376E0CE0199
:108AB00001960E94C375CE0101960E94C993CE0112
:108AC00001960E94247564EF71E080E090E00E94BE
:108AD000817966E176E0CE0101960E94C375BE0100
:108AE000685D7F4FCE0101960E943F74BC01CE01AC
:108AF0004C960E94BA75CE0101960E942475CE0153
:108B00004C960E948073BE01645E7F4FCE01019639
:108B10000E94BA75CE0101960E94C993CE010196BA
:108B20000E942475CE014C960E942475CE01889631
:108B30000E94247568EB7BE080E090E00E948179E0
:108B400069EF70E1CE0101960E94C375CE010196D6
:108B50000E94D51ACE0101960E94247510923D0202
:108B6000CE0182960C94273C66E476E0CE01019615
:108B70000E94C375BE016F5F7F4FCE018E960E942B
:108B80000E74182FCE0101960E942475112309F44A
:108B900086C044E050E066EB7FE0CE0101960E9483
:108BA0009F19BE016F5F7F4F82E99FE00E94EB74C7
:108BB000CE0101960E9424756BE476E0CE01019609
:108BC0000E94C37562E97FE0CE0101960E943F7466
:108BD000BC01CE014C960E94BA75CE0101960E944E
:108BE00024758091F5109091F610892B39F4BE010F
:108BF000645E7F4F8FE99CE00E94FC7668E873E139
:108C000080E090E00E9481798091F5109091F610BB
:108C1000029759F562E576E0CE0101960E94C37590
:108C20008091960F9091970F892B19F56BE576E05F
:108C3000CE0101960E940773BE01645E7F4FCE0194
:108C400082960E94BA75CE0182960E94C993CE0187
:108C500082960E94247568E873E180E090E00E94AB
:108C60008179CE0101960E94247510923D020C94E8
:108C7000253CBE016F5F7F4FCE0182960E94BA7580
:108C8000CE0182960E94C993CE0182960E942475DD
:108C900060E777E180E090E00E948179CDCF64E6E3
:108CA00076E0CE0101960E94C375BE016F5F7F4FD3
:108CB000CE018E960E940E74182FCE0101960E944E
:108CC0002475112309F475C066EB7FE082E99FE00B
:108CD0000E94D47481E080933D0266EB7FE0CE0178
:108CE00001960E94BA75CE0101960E94D51ACE0156
:108CF00001960E9424758091F5109091F6100297CC
:108D000009F162E97FE08FE99CE00E94FC7668EB64
:108D10007BE080E090E00E948179CE0101960E9484
:108D20006294BE016F5F7F4F86EB9FE00E94EB7401
:108D3000CE0101960E94247560ED77E080E090E01E
:108D40000E9481798091F5109091F610029771F44C
:108D500062E97FE0CE0101960E94BA75CE010196CC
:108D60000E94C993CE0101960E9424758091BA0F8A
:108D70009091BB0F892B09F436CD6BE777E0CE01DC
:108D800001960E94C37566EB7FE0CE0101960E94BA
:108D90003F74BC01CE014C960E94BA75CE014C9630
:108DA0000E94E915CE014C960E942475CE010196D1
:108DB00050C268E676E0CE0101960E94C375BE01FE
:108DC0006F5F7F4FCE018E960E940E74182FCE01DA
:108DD00001960E942475112309F495C18091F51024
:108DE0009091F610019709F0FECC6EE676E0CE0188
:108DF00088960E94C375BE01685D7F4F8FE99CE035
:108E00000E94FC766CE271E080E090E00E94817943
:108E1000CE0182960E94629464E670E080E090E069
:108E20000E94817910E000E025E0C22ED12C3AE0CA
:108E3000A32EB12C69E776E0CE0101960E94C3759E
:108E400050E040E0BE016F5F7F4FCE0182960E94EE
:108E500082A17C01CE0101960E942475A7014F5F7B
:108E60005F4FBE016E5D7F4FCE0101960E949F193C
:108E7000BE016F5F7F4FCE0188960E94EB74CE01DA
:108E800001960E9424758CA59DA5892B09F170E09F
:108E900060E0CE0188960E94DD73082E000C990BCD
:108EA000C0970A97A8F46BE776E0CE0101960E947E
:108EB000C375BE016F5F7F4FCE0188960E940E740E
:108EC000E82ECE0101960E942475FF24F394E11050
:108ED000F12C6CE777E0CE0101960E94B17564E158
:108EE00070E0CE0101960E9458A2CE0101960E9428
:108EF00024750F5F1F4F62E370E080E090E00E94F6
:108F00008179C801B6010E9481AE0197C1F4CE01FA
:108F100001960E946E1C8D819E81892B09F4BEC032
:108F2000BE016F5F7F4F86EB9FE00E94D4740E946A
:108F30008238FF24F394CE0101960E942475CE015D
:108F400001960E946294BE016F5F7F4FCE018296B0
:108F50000E94EB74CE0101960E94247562E370E0DA
:108F600080E090E00E9481790436110519F0FF201D
:108F700009F460CF8091B90B8823F1F06BE777E0BB
:108F8000CE014C960E94C375BE01685D7F4FCE0135
:108F90004C960E943F74BC01CE0101960E94BA75A6
:108FA000CE0101960E94E915CE0101960E9424751A
:108FB000CE014C960E9424758CA59DA5892B69F045
:108FC00070E060E0CE0188960E94DD73082E000CF0
:108FD000990BC0970A9708F47AC063E876E0CE014F
:108FE00001960E94C375CE0182960E942475CE011F
:108FF00088960E9424758D819E81009709F449C04E
:10900000E981FA812081222309F443C0079708F4FB
:1090100040C064ED78E0CE014C960E94B17568ECDA
:1090200070E0CE014C960E9458A2CE014C960E9450
:109030002475BE016F5F7F4FCE014C960E94BA75BA
:1090400040ED57E06FEF7FEFCE014C960E9409098B
:10905000CE014C960E9424756FE876E0CE014C96C6
:109060000E94C37566EB7FE0CE014C960E943F7470
:10907000BC01CE0182960E94BA75CE0182960E94F2
:10908000E915CE0182960E942475CE014C960E946D
:109090002475CE0101960E942475A5CB04311105DB
:1090A0000CF449CFC801B5010E9481AE892B09F0AB
:1090B00042CFBE01685D7F4F8FE99CE00E94FC7645
:1090C00068EC70E080E090E00E94817934CF6BE73B
:1090D00076E0CE0101960E94C375BE016F5F7F4F9F
:1090E000CE0188960E940E74182FCE0101960E9420
:1090F0002475111172CFBE01685D7F4FCE010196BC
:109100000E94A87570CF6DE976E0CE0101960E94AD
:10911000C375BE016F5F7F4FCE018E960E940E74A5
:10912000182FCE0101960E942475112309F4EAC07C
:1091300025E030E044E050E066EB7FE0CE010196B0
:109140000E94D875BE016F5F7F4F82E99FE00E9449
:10915000EB74CE0101960E94247566EB7FE0CE0190
:1091600001960E94BA75CE0101960E94D51ACE01D1
:1091700001960E94247582E99FE00E947573613018
:10918000710509F069C07093F6106093F5106BEAF1
:1091900077E0CE0101960E94B175CE0101960E9442
:1091A000D51ACE0101960E94247562EA76E0CE01BE
:1091B0004C960E94C37565E871E1CE014C960E9401
:1091C0003F74BC01CE0101960E94BA7548EC50E094
:1091D0006FEF7FEFCE0101960E943220CE01019603
:1091E0000E942475CE014C960E9424750E94F49F23
:1091F00040E052EC61E070E08FE99CE00E94217158
:1092000084EF91E0909367028093660269E370E1D6
:109210000E94A40861EB76E0CE014C960E94C375D3
:109220006FE771E1CE014C960E943F74BC01CE0104
:1092300001960E94BA7540ED57E06FEF7FEFCE01C7
:1092400001960E940909CE0101960E942475CE0163
:109250004C960E942475C7CA61157105D1F510920C
:10926000F6101092F5106DE977E0CE0101960E949C
:10927000B175CE0101960E94D51ACE0101960E94C9
:10928000247568EA76E0CE014C960E94C37565E8C5
:1092900071E1CE014C960E943F74BC01CE01019653
:1092A0000E94BA7548EC50E06FEF7FEFCE01019657
:1092B0000E943220CE0101960E942475CE014C9668
:1092C0000E9424750E94F49F40E855E260E070E03F
:1092D00093CF6230710509F086CA7093F6106093DF
:1092E000F5106CE877E0CE0101960E94B175CE01D1
:1092F00001960E94D51ACE0101960E9424756CEA4F
:1093000076E0C1CF66EB76E0CE0101960E94C37590
:10931000BE016F5F7F4FCE018E960E940E74182F94
:10932000CE0101960E942475112309F441C047E043
:1093300050E066EB7FE0CE0101960E949F19BE01CE
:109340006F5F7F4F82E99FE00E94EB74CE01019630
:109350000E94247561E876E0CE0101960E94C375F3
:10936000BE016F5F7F4F82E99FE00E940E74182F4D
:10937000CE0101960E94247511111092570C68EDD0
:1093800074E0CE0101960E94C375BE016F5F7F4FEE
:1093900082E99FE00E940E74182FCE0101960E9470
:1093A0002475112309F4E9CC81E08093570CE5CCB6
:1093B0006EEB76E0CE0101960E94C375BE016F5F31
:1093C0007F4FCE018E960E940E74182FCE0101960B
:1093D0000E942475112381F146E050E066EB7FE0A6
:1093E000CE0101960E949F19BE016F5F7F4F82E9F7
:1093F0009FE00E94EB74CE0101960E94247582E9E1
:109400009FE00E946A7360933D1170933E118093B8
:109410003F119093401184EF91E090936702809305
:10942000660269E370E10E94A40864E670E080E0EF
:1094300090E00E948179A1CC65EC76E0CE010196A6
:109440000E94C375BE016F5F7F4FCE018E960E9452
:109450000E74182FCE0101960E942475112301F17C
:1094600048E050E066EB7FE0CE0101960E949F1934
:10947000BE016F5F7F4F82E99FE00E94EB74CE01D7
:1094800001960E94247582E99FE00E946A736093AE
:109490004311709344118093451190934611BBCFB3
:1094A0006EEC76E0CE0101960E94C375BE016F5F3F
:1094B0007F4FCE018E960E940E74182FCE0101961A
:1094C0000E942475112301F149E050E066EB7FE032
:1094D000CE0101960E949F19BE016F5F7F4F82E906
:1094E0009FE00E94EB74CE0101960E94247582E9F0
:1094F0009FE00E946A7360934711709348118093B4
:10950000491190934A1187CF68ED76E0CE0101961C
:109510000E94C375BE016F5F7F4FCE018E960E9481
:109520000E74182FCE0101960E9424751123F1F0BC
:1095300049E050E066EB7FE0CE0101960E949F1962
:10954000BE016F5F7F4F82E99FE00E94EB74CE0106
:1095500001960E94247582E99FE00E946A730E942E
:1095600035AE70934E1160934D1155CF62EE76E09B
:10957000CE0101960E94C375BE016F5F7F4FCE0181
:109580008E960E940E74182FCE0101960E942475AB
:109590001123F1F04AE050E066EB7FE0CE01019646
:1095A0000E949F19BE016F5F7F4F82E99FE00E947A
:1095B000EB74CE0101960E94247582E99FE00E941F
:1095C0006A730E9435AE70934C1160934B1123CF98
:1095D0006DEE76E0CE0101960E94C375BE016F5F0D
:1095E0007F4FCE018E960E940E74182FCE010196E9
:1095F0000E942475112311F14BE050E066EB7FE0EF
:10960000CE0101960E949F19BE016F5F7F4F82E9D4
:109610009FE00E94EB74CE0101960E94247582E9BE
:109620009FE00E946A730E9435AE60934F11709361
:1096300050118093511190935211EDCE69EF76E065
:10964000CE0101960E94C375BE016F5F7F4FCE01B0
:109650008E960E940E74182FCE0101960E942475DA
:109660001123E1F045E050E066EB7FE0CE0101968A
:109670000E949F19BE016F5F7F4F82E99FE00E94A9
:10968000EB74CE0101960E94247582E99FE00E944E
:1096900075737093421160934111BDCE6FEF76E008
:1096A000CE0101960E94C375BE016F5F7F4FCE0150
:1096B0008E960E940E74182FCE0101960E9424757A
:1096C000112359F00E94187C60934A0C70934B0C44
:1096D00080934C0C90934D0C86C865E077E0CE01EA
:1096E00001960E94C375BE016F5F7F4FCE018E96BB
:1096F0000E940E74182FCE0101960E94247511232A
:1097000089F143E050E0BE01625D7F4FCE010196DA
:109710000E949F19BE016F5F7F4F82E99FE00E9408
:10972000EB74CE0101960E9424758091960F909162
:10973000970F892B41F082E99FE00E947573709327
:109740006F0260936E0280916E0290916F0201979A
:10975000029708F412CB81E090E090936F0280931F
:109760006E020BCB66EE76E0CE014C960E94C3757E
:10977000BE01645E7F4FCE018E960E940E7411E092
:10978000811115C060E577E0CE0101960E94C37596
:10979000BE016F5F7F4FCE018E960E940E7411E066
:1097A000811101C010E0CE0101960E942475CE0106
:1097B0004C960E942475112309F468C066EE76E089
:1097C000CE0101960E94C375BE016F5F7F4FCE012F
:1097D0008E960E940E74182FCE0101960E94247559
:1097E0001123A1F046E050E0BE01625D7F4FCE0143
:1097F00001960E949F19BE016F5F7F4F82E99FE033
:109800000E94EB74CE0101960E94247560E577E01A
:10981000CE0101960E94C375BE016F5F7F4FCE01DE
:109820008E960E940E74182FCE0101960E94247508
:109830001123A1F042E050E0BE01625D7F4FCE01F6
:1098400001960E949F19BE016F5F7F4F82E99FE0E2
:109850000E94EB74CE0101960E9424758091960FB0
:109860009091970F892B09F488CA62E97FE0CE01B5
:1098700001960E94BA7561E070E0CE0101960E94E7
:10988000582FCE0101960E94247577CA62E177E0D5
:10989000CE0182960E94C375BE016E5D7F4FCE01E0
:1098A0008E960E940E7411E0811129C069E077E064
:1098B000CE014C960E94C375BE01645E7F4FCE01FF
:1098C0008E960E940E7411E0811115C061E177E05F
:1098D000CE0101960E94C375BE016F5F7F4FCE011E
:1098E0008E960E940E7411E0811101C010E0CE012D
:1098F00001960E942475CE014C960E942475CE01DB
:1099000082960E942475112309F4E6C062E177E093
:10991000CE0101960E94C375BE016F5F7F4FCE01DD
:109920008E960E940E74182FCE0101960E94247507
:10993000112309F466C046E050E0BE01625D7F4F2E
:10994000CE0101960E949F19BE016F5F7F4F82E991
:109950009FE00E94EB74CE0101960E94247582E97B
:109960009FE00E946A736B017C0120E030E0A90156
:109970000E946BAE18160CF08EC0A701960160E035
:1099800070E08AE794E40E94C3AD0E9435AE609314
:10999000390270933A0280933B0290933C0280918B
:1099A000390290913A02A0913B02B0913C02181604
:1099B00019061A061B0664F081E090E0A0E0B0E012
:1099C0008093390290933A02A0933B02B0933C02F9
:1099D00080916E0290916F028130910509F068C00C
:1099E0008091390290913A02A0913B02B0913C02E1
:1099F0008093350290933602A0933702B0933802D9
:109A0000BCC947E050E0BE01625D7F4FCE010196C8
:109A10000E949F19BE016F5F7F4F82E99FE00E9405
:109A2000EB74CE0101960E94247560E874E0CE01CB
:109A300001960E94C375BE016F5F7F4FCE018E9667
:109A40000E940E74182FCE0101960E9424751123D6
:109A500031F081E090E090936F0280936E026FE1AD
:109A600076E0CE0101960E94C375BE016F5F7F4F05
:109A7000CE018E960E940E74182FCE0101960E9480
:109A80002475112309F46BCF82E090E090936F026C
:109A900080936E0264CF81E090E0A0E0B0E080931C
:109AA000390290933A02A0933B02B0933C0277CFE5
:109AB000029709F062C98091390290913A02A0910F
:109AC0003B02B0913C028093310290933202A0930A
:109AD0003302B093340251C969E177E0CE014C966C
:109AE0000E94C375BE01645E7F4FCE018E960E94B8
:109AF000EE7311E0811115C06EE177E0CE010196A1
:109B00000E94C375BE016F5F7F4FCE018E960E948B
:109B10000E7411E0811101C010E0CE0101960E9487
:109B20002475CE014C960E942475112309F48DC230
:109B30006BEA77E0CE0101960E94C375BE016F5FAC
:109B40007F4FCE018E960E940E74182FCE01019683
:109B50000E942475112309F4FBC001E010E010936A
:109B60006F0200936E0210935D0200935C0265E247
:109B700077E082E99FE00E94077310935D020093F3
:109B80005C0281E090E0A0E0B0E080933902909325
:109B90003A02A0933B02B0933C028093350290932B
:109BA0003602A0933702B093380262E97FE0CE011B
:109BB00001960E94BA7562E070E0CE0101960E94A3
:109BC000582FCE0101960E94247563EC78E0CE01F7
:109BD00001960E94B175CE0101960E94E915CE0151
:109BE00001960E94247563EB78E0CE0101960E94F5
:109BF000B175CE0101960E940721CE0101960E9407
:109C0000247561E876E082E99FE00E94077362E9CB
:109C10007FE0CE0101960E94BA7563E070E0CE014C
:109C200001960E94582FCE0101960E94247582E071
:109C300090E090936F0280936E0262EA78E0CE012A
:109C400001960E94B175CE0101960E94E915CE01E0
:109C500001960E94247566E978E0CE0101960E9483
:109C6000B175CE0101960E940721CE0101960E9496
:109C7000247565E277E082E99FE00E940773809196
:109C80005F119091601197FF06C069E277E082E969
:109C90009FE00E94077362E97FE0CE0101960E9477
:109CA000BA7562E070E0CE0101960E94582FCE0195
:109CB00001960E94247561E876E082E99FE00E94A7
:109CC000077382E090E090936F0280936E0262E9E6
:109CD0007FE0CE0101960E94BA7563E070E0CE018C
:109CE00001960E94582FCE0101960E94247584EFA0
:109CF00091E0909367028093660269E370E10E94AD
:109D0000A40864E670E080E090E00E94817981E040
:109D100090E090936F0280936E021092DA0210929C
:109D2000D90282E090E0A0E0B0E08093C30290937B
:109D3000C402A093C502B093C6020E94187C60932F
:109D4000E3027093E4028093E5029093E60215C863
:109D500069E177E0CE0101960E94C375BE016F5F95
:109D60007F4FCE018E960E940E74182FCE01019661
:109D70000E94247511110C94BD4660E874E0CE0178
:109D800001960E94C375BE016F5F7F4FCE018E9614
:109D90000E940E74182FCE0101960E942475112383
:109DA00031F081E090E090936F0280936E026FE15A
:109DB00076E0CE0101960E94C375BE016F5F7F4FB2
:109DC000CE018E960E940E74182FCE0101960E942D
:109DD0002475112331F082E090E090936F0280931C
:109DE0006E0281E090E0A0E0B0E0809339029093B1
:109DF0003A02A0933B02B0933C0280916E02909194
:109E00006F028130910509F099C090935D028093B3
:109E10005C026EE177E0CE0101960E94C375BE013F
:109E20006F5F7F4FCE018E960E940E74182FCE0169
:109E300001960E942475112319F146E050E0BE01FD
:109E4000625D7F4FCE014C960E949F196DE277E0D4
:109E5000CE0101960E94C375BE01645E7F4FCE01A4
:109E600001960E943F74BC0182E99FE00E94D47475
:109E7000CE0101960E942475CE014C960E94247555
:109E80008091390290913A02A0913B02B0913C023C
:109E90008093350290933602A0933702B093380234
:109EA00065E277E082E99FE00E94077362E97FE064
:109EB000CE0101960E94BA7562E070E0CE01019673
:109EC0000E94582FCE0101960E94247565E878E023
:109ED000CE0101960E94B175CE0101960E94E9154E
:109EE000CE0101960E94247581E090E090935D027E
:109EF00080935C0261E876E082E99FE00E9407734C
:109F000062E97FE0CE0101960E94BA7563E070E0DD
:109F1000CE0101960E94582FCE0101960E94247511
:109F200065E778E0CE0101960E94B175CE010196F9
:109F30000E940721CE0101960E94247580916E0235
:109F400090916F02029711F00C94BD4665E277E0A4
:109F500082E99FE00E94077380915F1190916011E8
:109F600097FF06C069E277E082E99FE00E940773ED
:109F700001E010E010935D0200935C0262E97FE073
:109F8000CE0101960E94BA7562E070E0CE010196A2
:109F90000E94582FCE0101960E94247561E876E058
:109FA00082E99FE00E94077364E678E0CE010196A3
:109FB0000E94B175CE0101960E94E915CE0101966D
:109FC0000E94247562E97FE0CE0101960E94BA7575
:109FD00063E070E0CE0101960E94582FCE010196F9
:109FE0000E94247568E578E0CE0101960E94B17563
:109FF000CE0101960E940721CE0101960E94247590
:10A0000080915F1190916011919581959109909344
:10A01000601180935F1110935D0200935C0284EFE6
:10A0200091E0909367028093660269E370E10E9479
:10A03000A40864E670E080E090E00E9481791093CB
:10A040006F0200936E020C94BD466FE277E0CE0182
:10A0500088960E94C375BE01685D7F4FCE018E96C3
:10A060000E940E7401E081113DC060E877E0CE01EE
:10A0700082960E94C375BE016E5D7F4FCE018E96A3
:10A080000E940E7401E0811129C06FE777E0CE01D4
:10A090004C960E94C375BE01645E7F4FCE018E96C2
:10A0A0000E940E7401E0811115C066E377E0CE01D5
:10A0B00001960E94C375BE016F5F7F4FCE018E96E1
:10A0C0000E940E7401E0811101C000E0CE010196F2
:10A0D0000E942475CE014C960E942475CE01829672
:10A0E0000E942475CE0188960E942475002309F4ED
:10A0F0001FC26FE277E0CE0101960E94C375BE01D8
:10A100006F5F7F4FCE018E960E940E74082FCE0196
:10A1100001960E94247546E050E0011117C060E8E6
:10A1200077E0CE0101960E94C375BE016F5F7F4F3D
:10A13000CE018E960E940E74082FCE0101960E94C9
:10A140002475002309F48BC042E050E0BE01625D3B
:10A150007F4FCE0101960E949F19BE016F5F7F4F16
:10A1600082E99FE00E94EB74CE0101960E94247563
:10A170008091960F9091970F892B11F40C94BD4606
:10A180006DE277E0CE014C960E94C375BE01645E1D
:10A190007F4F82E99FE00E940E74811114C06FE628
:10A1A00078E0CE0101960E94C375BE016F5F7F4FBC
:10A1B00082E99FE00E940E7411E0811110E0CE014F
:10A1C00001960E942475CE014C960E942475C12CE4
:10A1D000D12C7601112309F46AC182E99FE00E9423
:10A1E0006A736B017C0180916E0290916F020197FE
:10A1F00009F09FC082E99FE00E946A739B01AC0155
:10A200006091E20B7091E30B8091E40B9091E50B70
:10A210000E9457AD6093E20B7093E30B8093E40BC5
:10A220009093E50B8090E20B9090E30BA090E40BF1
:10A23000B090E50B20E030E044EB53E4C501B401FD
:10A240000E946BAE87FD86C020E030E044EB53E413
:10A25000C501B4010E9456AD4B015C01EBCF43E058
:10A2600050E0BE01625D7F4FCE0101960E949F19B2
:10A27000BE016F5F7F4F82E99FE00E94EB74CE01C9
:10A2800001960E94247560E874E0CE0101960E9458
:10A29000C375BE016F5F7F4FCE018E960E940E7414
:10A2A000082FCE0101960E9424750023B1F081E0B1
:10A2B00090E090936F0280936E028091380C9091A1
:10A2C000390CA0913A0CB0913B0C8093E20B909327
:10A2D000E30BA093E40BB093E50B6FE176E0CE01C6
:10A2E00001960E94C375BE016F5F7F4FCE018E96AF
:10A2F0000E940E74082FCE0101960E94247500233F
:10A3000009F436CF82E090E090936F0280936E0262
:10A310008091340C9091350CA091360CB091370C93
:10A320008093E20B9093E30BA093E40BB093E50BC7
:10A330001FCF82E99FE00E946A739B01AC0160918C
:10A34000E20B7091E30B8091E40B9091E50B0E947E
:10A3500056AD60CF20E030E0A901C501B4010E94F4
:10A36000A9AB87FF0BC020E030E044EB53E4C5010C
:10A37000B4010E9457AD4B015C01ECCF8092E20B1F
:10A380009092E30BA092E40BB092E50B20E030E05A
:10A39000A901C701B6010E946BAE87FD15C06FE62B
:10A3A00078E0CE0101960E94C37562E97FE0CE019C
:10A3B00001960E943F74BC0182E99FE00E94D47420
:10A3C000CE0101960E94247520E030E0A901C7016A
:10A3D000B6010E94A9AB87FF6AC080916E0290917E
:10A3E0006F02019799F520E030E0A901C701B6019D
:10A3F0000E946BAE18160CF092C020E030E040E2F4
:10A4000051E4C701B6010E9457AD22E0AB01BC0187
:10A41000CE014C960E942C756DE277E0CE0101963C
:10A420000E94C375BE01645E7F4FCE0101960E94FB
:10A430003F74BC0182E99FE00E94D474CE01019672
:10A440000E942475CE014C960E94247580916E0264
:10A4500090916F02019759F120E030E0A901C70106
:10A46000B6010E946BAEB701A60118160CF0705829
:10A4700022E0CE014C960E942C756DE277E0CE0171
:10A4800001960E94C375BE01645E7F4FCE010196A6
:10A490000E943F74BC0182E99FE00E94D474CE0107
:10A4A00001960E942475CE014C960E94247581E08D
:10A4B00090E090935D0280935C0262E97FE0CE01C0
:10A4C00001960E94BA7562E070E0CE0101960E948A
:10A4D000582FCE0101960E94247520E030E0A9019A
:10A4E000C701B6010E94A9AB87FD02C00C94BD460E
:10A4F00080916E0290916F02019711F00C94BD460D
:10A500006AE377E082E99FE00E94077362E97FE0F7
:10A51000CE0101960E94BA7562E070E0AEC9A70153
:10A52000960160E070E080E291E40E9456AD6DCF4C
:10A530006FE377E0CE0182960E94C375BE016E5D27
:10A540007F4FCE018E960E940E7411E0811129C0BA
:10A550006EE377E0CE014C960E94C375BE01645E47
:10A560007F4FCE018E960E940E7411E0811115C0AE
:10A5700065E477E0CE0101960E94C375BE016F5F6E
:10A580007F4FCE018E960E940E7411E0811101C0A2
:10A5900010E0CE0101960E942475CE014C960E94D7
:10A5A0002475CE0182960E942475112309F49BC064
:10A5B000CE018E960E94807365E277E082E99FE08B
:10A5C0000E94077360E874E0CE0101960E94C37593
:10A5D000BE016F5F7F4FCE018E960E940E74182FC2
:10A5E000CE0101960E942475112331F081E090E0A4
:10A5F00090936F0280936E026FE176E0CE01019638
:10A600000E94C375BE016F5F7F4FCE018E960E9480
:10A610000E74182FCE0101960E942475112391F01B
:10A6200082E090E090936F0280936E0280915F11C0
:10A630009091601197FF06C069E277E082E99FE0A0
:10A640000E94077381E090E090935D0280935C022A
:10A6500062E97FE0CE0101960E94BA7562E070E087
:10A66000CE0101960E94582FCE0101960E942475BA
:10A670006FE377E0CE0101960E94C375BE016F5F64
:10A680007F4FCE018E960E940E74182FCE01019638
:10A690000E94247545E050E0111102C046E050E0F0
:10A6A000BE01625D7F4FCE0101960E949F19BE01DF
:10A6B0006F5F7F4F82E99FE00E94EB74CE010196AD
:10A6C0000E9424758091960F9091970F892B11F419
:10A6D0000C94BD4662E97FE0CE0101960E94BA75F6
:10A6E00063E070E0CAC86DE477E0CE0182960E9414
:10A6F000C375BE016E5D7F4FCE018E960E940E74B3
:10A7000011E0811129C06CE477E0CE014C960E94E3
:10A71000C375BE01645E7F4FCE018E960E940E749B
:10A7200011E0811115C063E577E0CE0101960E942A
:10A73000C375BE016F5F7F4FCE018E960E940E746F
:10A7400011E0811101C010E0CE0101960E94247534
:10A75000CE014C960E942475CE0182960E942475EB
:10A76000112309F426C16DE477E0CE0101960E9421
:10A77000C375BE016F5F7F4FCE018E960E940E742F
:10A78000182FCE0101960E942475112309F443C0AD
:10A7900045E050E0BE01625D7F4FCE0101960E9410
:10A7A0009F19BE016F5F7F4F82E99FE00E94EB74AB
:10A7B000CE0101960E9424758091960F9091970F7B
:10A7C000892B61F082E99FE00E946A736093E20B3B
:10A7D0007093E30B8093E40B9093E50BC090E20B36
:10A7E000D090E30BE090E40BF090E50B20E030E03C
:10A7F00044EB53E4C701B6010E946BAE87FD55C020
:10A8000020E030E044EB53E4C701B6010E9456ADAE
:10A810006B017C01EBCF46E050E0BE01625D7F4FF3
:10A82000CE0101960E949F19BE016F5F7F4F82E9A2
:10A830009FE00E94EB74CE0101960E94247560E8AF
:10A8400074E0CE0101960E94C375BE016F5F7F4F19
:10A85000CE018E960E940E74182FCE0101960E9492
:10A860002475112331F081E090E090936F02809382
:10A870006E026FE176E0CE0101960E94C375BE01C3
:10A880006F5F7F4FCE018E960E940E74182FCE01FF
:10A8900001960E942475112309F48ECF82E090E086
:10A8A00090936F0280936E0287CF20E030E0A90181
:10A8B000C701B6010E94A9AB87FF0BC020E030E0C2
:10A8C00044EB53E4C701B6010E9457AD6B017C0114
:10A8D000ECCFC092E20BD092E30BE092E40BF0924B
:10A8E000E50B80916E0290916F02019771F4C09216
:10A8F000380CD092390CE0923A0CF0923B0C61E1AA
:10A9000075E088E99FE00E9407738091E20B9091C7
:10A91000E30BA091E40BB091E50B20916E02309116
:10A920006F022230310571F48093340C9093350C12
:10A93000A093360CB093370C61E275E088E99FE094
:10A940000E9407734091E20B5091E30B6091E40B7E
:10A950007091E50B21E0CE014C960E942C7568E9C0
:10A960007FE0CE0101960E94BA75BE01645E7F4F02
:10A97000CE0101960E943F746CE175E00E9429743B
:10A98000BC0188E99FE00E94D474CE0101960E9428
:10A990002475CE014C960E94247568E97FE0CE01B3
:10A9A00001960E94BA75CE0101960E9407210C946F
:10A9B000414C6BE577E0CE0182960E94C375BE01E3
:10A9C0006E5D7F4FCE018E960E940E7411E0811154
:10A9D00029C06AE577E0CE014C960E94C375BE019E
:10A9E000645E7F4FCE018E960E940E7411E081113D
:10A9F00015C060E677E0CE0101960E94C375BE01E6
:10AA00006F5F7F4FCE018E960E940E7411E0811110
:10AA100001C010E0CE0101960E942475CE014C9633
:10AA20000E942475CE0182960E942475112309F498
:10AA300012C2C0903902D0903A02E0903B02F090EE
:10AA40003C0266E677E0CE0101960E94C375BE0126
:10AA50006F5F7F4FCE018E960E940E74182FCE012D
:10AA600001960E942475112309F465C044E050E06A
:10AA7000BE01625D7F4FCE0101960E949F19BE010B
:10AA80006F5F7F4F82E99FE00E94EB74CE010196D9
:10AA90000E94247580916E0290916F028130910521
:10AAA00009F093C0C0903502D0903602E090370292
:10AAB000F090380281E090E0A0E0B0E080933502B1
:10AAC00090933602A0933702B09338028091960F8C
:10AAD0009091970F892B09F090C06BE677E082E99F
:10AAE0009FE00E9407738091960F9091970F892B9A
:10AAF00081F062E97FE0CE0101960E94BA7570E0B4
:10AB000060E0CE0101960E94582FCE0101960E946E
:10AB1000247580916E0290916F028130910509F049
:10AB20008CC1C0923502D0923602E0923702F09288
:10AB300038020C94BD4645E050E0BE01625D7F4F97
:10AB4000CE0101960E949F19BE016F5F7F4F82E97F
:10AB50009FE00E94EB74CE0101960E94247560E88C
:10AB600074E0CE0101960E94C375BE016F5F7F4FF6
:10AB7000CE018E960E940E74182FCE0101960E946F
:10AB80002475112331F081E090E090936F0280935F
:10AB90006E026FE176E0CE0101960E94C375BE01A0
:10ABA0006F5F7F4FCE018E960E940E74182FCE01DC
:10ABB00001960E942475112309F46CCF82E090E085
:10ABC00090936F0280936E0265CF029709F07ECF5B
:10ABD000C0903102D0903202E0903302F090340203
:10ABE00081E090E0A0E0B0E08093310290933202E7
:10ABF000A0933302B093340269CF61E777E0CE01CE
:10AC000001960E94C375BE016F5F7F4F82E99FE08E
:10AC10000E94EE73182FCE0101960E942475112315
:10AC200009F477CF82E99FE00E946A7320E030E068
:10AC3000A9010E94A9AB811128C080916E02909158
:10AC40006F02019731F464E777E082E99FE00E94A8
:10AC5000077380916E0290916F02029731F46BE658
:10AC600077E082E99FE00E9407738091960F9091B0
:10AC7000970F892B09F44DCF62E97FE0CE01019651
:10AC80000E94BA7561E070E03CCF62EF75E0CE01E2
:10AC900001960E94C375BE016F5F7F4F82E99FE0FE
:10ACA0000E94EE73182FCE0101960E942475112385
:10ACB00009F42FCF41E050E062E97FE0CE01019638
:10ACC0000E949F19CE0101960E946A734B015C019C
:10ACD000CE0101960E94247520E030E0A901C50153
:10ACE000B4010E94A9AB181634F0812C912C90E885
:10ACF000A92E9FE3B92E00916E0210916F020130D0
:10AD0000110509F075C0A501940160E070E48CE9BB
:10AD100095E40E94C3AD60932D0270932E02809340
:10AD20002F029093300260935711709358118093C3
:10AD3000591190935A116093290270932A028093BB
:10AD40002B0290932C02B801CE014C960E941173F5
:10AD500069E777E0CE0101960E94C375BE01645E8B
:10AD60007F4FCE0101960E943F74BC01CE018296B6
:10AD70000E94BA75CE0182960E940016CE0182967C
:10AD80000E942475CE0101960E942475CE014C9636
:10AD90000E94247566E478E0CE0101960E94B175A8
:10ADA000CE0101960E940016CE0101960E942475E4
:10ADB00040912D0250912E0260912F02709130022D
:10ADC00025E0CE0101960E942C75CE0101960E94CD
:10ADD000E915CE0101960E94247584EF91E09093CD
:10ADE00067028093660269E370E10E94A40891CE35
:10ADF0000230110509F0A7CFA501940160E070E4CD
:10AE00008CE196E40E94C3AD60932D0270932E02F4
:10AE100080932F029093300260935B1170935C11CA
:10AE200080935D1190935E116093250270932602CA
:10AE3000809327029093280286CF029711F00C94FA
:10AE4000BD46C0923102D0923202E0923302F092BB
:10AE500034020C94BD466EE777E0CE0182960E94E4
:10AE6000C375BE016E5D7F4FCE018E960E940E743B
:10AE700011E0811129C06DE777E0CE014C960E9468
:10AE8000C375BE01645E7F4FCE018E960E940E7424
:10AE900011E0811115C063E877E0CE0101960E94B0
:10AEA000C375BE016F5F7F4FCE018E960E940E74F8
:10AEB00011E0811101C010E0CE0101960E942475BD
:10AEC000CE014C960E942475CE0182960E94247574
:10AED000112309F429C18AA99BA9059710F40C94A0
:10AEE000BD4644E050E0BE01625D7F4FCE01019659
:10AEF0000E949F19BE016F5F7F4F82E99FE00E9411
:10AF0000EB74CE0101960E9424756EE777E0CE01C6
:10AF100001960E94C375BE016F5F7F4FCE018E9672
:10AF20000E940E74182FCE0101960E9424751123E1
:10AF300009F49BC044E050E0BE01625D7F4FCE014A
:10AF400001960E949F19BE016F5F7F4F82E99FE0CB
:10AF50000E94EB74CE0101960E94247582E99FE065
:10AF60000E946A7320E030E0A9010E946BAE1816BF
:10AF700014F00C94BD4682E99FE00E946A736093CE
:10AF80002D0270932E0280932F0290933002209115
:10AF90006E0230916F022130310509F0B0C060932C
:10AFA0005711709358118093591190935A116093CF
:10AFB000290270932A0280932B0290932C02B901EC
:10AFC000CE014C960E94117369E777E0CE0101969D
:10AFD0000E94C375BE01645E7F4FCE0101960E9440
:10AFE0003F74BC01CE0182960E94BA75CE01829652
:10AFF0000E940016CE0182960E942475CE01019611
:10B000000E942475CE014C960E94247564E378E07A
:10B01000CE0101960E94B175CE0101960E940016E4
:10B02000CE0101960E94247540912D0250912E026E
:10B0300060912F027091300225E0CE0101960E94AE
:10B040002C75CE0101960E94E915CE0101960E9451
:10B05000247584EF91E0909367028093660269E320
:10B0600070E10E94A4080C94BD4645E050E0BE018A
:10B07000625D7F4FCE0101960E949F19BE016F5FF6
:10B080007F4F82E99FE00E94EB74CE0101960E94FF
:10B09000247560E874E0CE0101960E94C375BE017C
:10B0A0006F5F7F4FCE018E960E940E74182FCE01D7
:10B0B00001960E942475112331F081E090E0909375
:10B0C0006F0280936E026FE176E0CE0101960E94DE
:10B0D000C375BE016F5F7F4FCE018E960E940E74C6
:10B0E000182FCE0101960E942475112309F436CF42
:10B0F00082E090E090936F0280936E022FCF223017
:10B10000310509F05CCF60935B1170935C11809303
:10B110005D1190935E1160932502709326028093D7
:10B120002702909328024BCF64E875E0CE014C963D
:10B130000E94C375BE01645E7F4FCE018E960E9451
:10B140000E7411E0811115C069E877E0CE01019617
:10B150000E94C375BE016F5F7F4FCE018E960E9425
:10B160000E7411E0811101C010E0CE0101960E9421
:10B170002475CE014C960E942475112309F463C0F6
:10B1800064E875E0CE0101960E94C375BE016F5F51
:10B190007F4FCE018E960E940E74182FCE0101961D
:10B1A0000E942475112399F042E050E066EB7FE0A5
:10B1B000CE0101960E949F19BE016F5F7F4F82E909
:10B1C0009FE00E94EB74CE0101960E94247569E80D
:10B1D00077E0CE0101960E94C375BE016F5F7F4F7D
:10B1E000CE018E960E940E74182FCE0101960E94F9
:10B1F0002475112399F043E050E066EB7FE0CE0127
:10B2000001960E949F19BE016F5F7F4F82E99FE008
:10B210000E94EB74CE0101960E94247582E99FE0A2
:10B220000E947573653B710510F40C94BD4661E294
:10B2300078E0CE0101960E94B175CE0101960E9480
:10B2400000160C94414C6DE877E0CE0101960E9407
:10B25000C375BE016F5F7F4FCE018E960E940E7444
:10B26000182FCE0101960E942475112309F474C091
:10B2700026E030E044E050E066EB7FE0CE0101964E
:10B280000E94D875BE016F5F7F4F82E99FE00E94E8
:10B29000EB74CE0101960E94247562EF75E0CE0139
:10B2A00001960E94C3754091BA0F5091BB0F8D81DA
:10B2B0009E81481B590BBE016F5F7F4F86EB9FE05D
:10B2C0000E943BA0AC014F5F5F4F66EB7FE0CE0179
:10B2D0004C960E949F19BE01645E7F4F82E99FE0F9
:10B2E0000E94EB74CE014C960E942475CE0101960B
:10B2F0000E94247582E99FE00E946A7388E2EAEB6B
:10B30000FBE0A0E1B1E101900D928A95E1F784EFB5
:10B3100091E0909367028093660269E370E10E9476
:10B32000A40860E078E088E99FE00E94AF7444E000
:10B3300050E066EB7FE0CE0101960E949F19BE01AE
:10B340006F5F7F4F88E99FE00E94A874CE0101964D
:10B350000E9424750C94B14361E977E0CE01019617
:10B360000E94C375BE016F5F7F4FCE018E960E9413
:10B370000E74182FCE0101960E94247511110C94A1
:10B38000974969E977E0CE0101960E94C375BE0135
:10B390006F5F7F4FCE018E960E940E74182FCE01E4
:10B3A00001960E942475112371F141E068E972E071
:10B3B000CE0101960E94EB8DBE016F5F7F4F8DE93C
:10B3C00091E10E9410198DE991E10E94988D8111FF
:10B3D00004C064EB77E00C9475428DE991E10E9422
:10B3E0003270892B51F08DE991E10E94F888682F25
:10B3F0008CE39DE00E945B6EF0CF8DE991E10E94AD
:10B40000A48D0C949B3960EA77E0CE0101960E94EE
:10B41000C375BE016F5F7F4FCE018E960E940E7482
:10B42000182FCE0101960E9424751123E9F08DB7E3
:10B430009EB7825391400FB6F8949EBF0FBE8DBF4A
:10B44000ADB7BEB7119682E391E0E9E3F0E1019078
:10B450000D920197E1F70E940A2B0FB6F894DEBF18
:10B460000FBECDBF0C949B3969EA77E0CE010196FF
:10B470000E94C375BE016F5F7F4FCE018E960E9402
:10B480000E74182FCE0101960E942475112309F421
:10B4900057C0EDB7FEB7E253F1400FB6F894FEBFC8
:10B4A0000FBEEDBFADB7BEB7119682E391E0E9E301
:10B4B000F0E101900D920197E1F70E9489240FB607
:10B4C000F894DEBF0FBECDBF6FEE77E0CE010196E0
:10B4D0000E94B175ADB7BEB7A253B1400FB6F89494
:10B4E000BEBF0FBEADBF119682E391E0E9E3F0E18C
:10B4F00001900D920197E1F70E94B91D0FB6F894E3
:10B50000DEBF0FBECDBF8DB79EB7825391400FB641
:10B51000F8949EBF0FBE8DBFADB7BEB7119682E344
:10B5200091E0E9E3F0E101900D920197E1F70E94CB
:10B530000A2B0FB6F894DEBF0FBECDBF0C94A03E11
:10B540006BEA77E0CE0101960E94C375BE016F5F82
:10B550007F4FCE018E960E940E74182FCE01019659
:10B560000E9424751123F9F06DED77E0CE0101966C
:10B570000E94B175BE016F5F7F4FCE014C960E9455
:10B58000BA75CE014C960E94E915CE014C960E94E8
:10B590002475EDB7FEB7E253F1400FB6F894FEBF45
:10B5A0000FBEEDBFB9CF6FEA77E0CE0101960E94E2
:10B5B000C375BE016F5F7F4FCE018E960E940E74E1
:10B5C000182FCE0101960E942475112309F4F5C0AD
:10B5D00061EC77E0CE0182960E94B175BE016E5D8E
:10B5E0007F4FCE0101960E94BA75AE014F5F5F4F4B
:10B5F00062E070E081E892E00E943C26182FCE01C4
:10B6000001960E942475111122C0BE016E5D7F4F0C
:10B61000CE014C960E94BA7563EB77E0CE014C9652
:10B620000E94297469EE7FE00E943F74BC01CE0144
:10B6300001960E94BA75CE0101960E94E915CE01CD
:10B6400001960E942475CE014C960E94247568EEE6
:10B6500073E080E090E00E948179BE016E5D7F4FD3
:10B66000CE0101960E94BA75AE014F5F5F4F63E055
:10B6700070E084E792E00E943C26182FCE010196EC
:10B680000E942475111122C0BE016E5D7F4FCE0154
:10B690004C960E94BA7563EC77E0CE014C960E94FE
:10B6A000297469EE7FE00E943F74BC01CE010196CF
:10B6B0000E94BA75CE0101960E94E915CE0101964D
:10B6C0000E942475CE014C960E94247568EE73E0AA
:10B6D00080E090E00E9481796DED7FE0CE010196DF
:10B6E0000E94BA75AE014F5F5F4F61E070E082EB80
:10B6F00092E00E943C26182FCE0101960E942475EC
:10B70000111121C06DED7FE0CE014C960E94BA75FB
:10B7100063EC77E0CE014C960E94297469EE7FE0DD
:10B720000E943F74BC01CE0101960E94BA75CE0101
:10B7300001960E94E915CE0101960E942475CE0162
:10B740004C960E94247568EE73E080E090E00E94C1
:10B7500081798091570C882311F40C94B04543E112
:10B7600062EB72E0CE0101960E94EB8DBE016F5F2D
:10B770007F4F83ED91E10E94101983ED91E10E94CA
:10B78000988D882311F40C94B0456DED7FE083ED26
:10B7900091E10E940A7766E970E080E090E00E9403
:10B7A000817983ED91E10E94A48D62E370E080E0F5
:10B7B00090E00E9481790C94B0456FEC77E0CE0167
:10B7C00001960E94C375BE016F5F7F4FCE018E96BA
:10B7D0000E940E74182FCE0101960E942475112329
:10B7E000A9F008EF1BE0D8018C910E5F1F4F60E0BD
:10B7F0000E940E786CE271E080E090E00E94817916
:10B80000BBE00E3F1B0779F70C949B3963ED77E0A3
:10B81000CE0101960E94C375BE016F5F7F4FCE01BE
:10B820008E960E940E74182FCE0101960E942475E8
:10B830001123C1F008EF1BE08EEFE82E8BE0F82E0D
:10B84000F80180810E5F1F4F61E00E940E786CE26C
:10B8500071E080E090E00E948179E016F10681F7C6
:10B860000C949B3968ED77E0CE0101960E94C37578
:10B87000BE016F5F7F4FCE018E960E940E74182F0F
:10B88000CE0101960E942475112311F40C949B396A
:10B8900027E030E046E050E066EB7FE0CE01019625
:10B8A0000E94D875BE016F5F7F4F82E99FE00E94C2
:10B8B000EB74CE0101960E94247582E99FE00E94FC
:10B8C0007573672B71F41092B90B66EB7FE0CE01B4
:10B8D00001960E94BA75CE0101960E94D51A0C9469
:10B8E000494881E08093B90BF0CF2F923F924F925D
:10B8F0005F926F927F928F929F92AF92BF92CF9200
:10B90000DF92EF92FF920F931F93CF93DF9300D0BC
:10B9100000D01F921F92CDB7DEB760919002709158
:10B92000910280918E0290918F020E94171684E1FD
:10B93000482E512C612C712C312C212C8FEF281A80
:10B94000380AC301B2010E9481796091900270911E
:10B95000910280918E0290918F020E9417168C01A5
:10B9600083E02816310434F08EE12816310444F4C3
:10B97000012B51F084E1480E511C611C711CDECF7B
:10B980000115110509F0A6C080918E0290918F02D9
:10B990008B30910509F086C080906F1190907011E6
:10B9A000A0907111B0907211C0906B11D0906C1179
:10B9B000E0906D11F0906E1164E670E080E090E030
:10B9C0000E9481796DE075E0CE0101960E94B1750B
:10B9D000CE0101960E940721CE0101960E94247596
:10B9E00061E082E00E94C57F21E0B501A401CE01A3
:10B9F00001960E942C75BE016F5F7F4F8FEE91E123
:10BA00000E94FC76CE0101960E9424756FED8FEEA8
:10BA100091E10E94F27F68E075E08FEE91E10E9473
:10BA20001E7720E0B701A601CE0101960E942C7579
:10BA3000BE016F5F7F4F8FEE91E10E94FC76CE01D9
:10BA400001960E9424756FED77E08FEE91E10E94E0
:10BA5000F47689829A82AB82BC82CD82DE82EF82CA
:10BA6000F88629813A814B815C816D817E818F814D
:10BA7000988528960FB6F894DEBF0FBECDBFDF9134
:10BA8000CF911F910F91FF90EF90DF90CF90BF90DB
:10BA9000AF909F908F907F906F905F904F903F906E
:10BAA0002F9008958631910509F476CF0C9709F00F
:10BAB00083CF8090DE0A9090DF0AA090E00AB090D9
:10BAC000E10AC090DA0AD090DB0AE090DC0AF0903C
:10BAD000DD0A72CF0F3F8FEF1807CCF06AEF74E0EA
:10BAE000CE0101960E94B1754AE050E070E060E03E
:10BAF000CE0101960E943220CE0101960E9424754B
:10BB000067ED74E088E99FE00E94AF7432C00E3F99
:10BB10008FEF1807B9F169EC74E0CE0101960E942D
:10BB2000B1754AE050E070E060E0CE0101960E94FD
:10BB30003220CE0101960E9424756AEB74E088E9F8
:10BB40009FE00E94AF74B801CE0101960E9411736C
:10BB5000BE016F5F7F4F88E99FE00E94A874CE010D
:10BB600001960E94247564EA74E088E99FE00E94CF
:10BB7000527419821A821B821C821D821E821F82AD
:10BB800018866FCF69E974E0CE0101960E94B17505
:10BB90004AE050E070E060E0CE0101960E94322061
:10BBA000CE0101960E94247569E774E0ABCF2F9215
:10BBB0003F924F925F926F927F928F929F92AF923D
:10BBC000BF92CF92DF92EF92FF920F931F93CF938A
:10BBD000DF93CDB7DEB7AC970FB6F894DEBF0FBEDC
:10BBE000CDBF8C017B018091320C9091330C01967A
:10BBF0009093330C8093320C20914F0C222341F010
:10BC00006AE070E00E9481AE181619060CF4C0C2FA
:10BC100081E080934F0C1092330C1092320C50E064
:10BC200040E060E274E0C8010E945A1982E0E81620
:10BC3000F10409F4C6C263EC78E087ED9FE00E944E
:10BC40000773609190027091910280918E029091A1
:10BC50008F020E9417161C016FEF7AE0C8010E9444
:10BC6000411961EE77E0C8010E94F47669E771E15D
:10BC7000CE0101960E94BA75BE016F5F7F4FC80169
:10BC80000E94FC76CE0101960E9424756AEE77E050
:10BC9000C8010E94F47664E076E0C8010E941E7735
:10BCA0006FE771E1CE0101960E94BA75BE016F5F28
:10BCB0007F4FC8010E94FC766AEF75E0C8010E94C0
:10BCC0001E7761E970E1CE0109960E94C375BE013D
:10BCD000675F7F4FC8010E94FC766DEE75E0C8017A
:10BCE0000E941E7769EF70E1CE010F960E94C37526
:10BCF000BE01615F7F4FC8010E94FC7666EE75E071
:10BD0000C8010E941E77CE010F960E942475CE01B5
:10BD100009960E942475CE0101960E9424750E9406
:10BD20003F7A28EE33E040E050E00E94F3AC290176
:10BD30003A016CED75E0C8010E941E77CE010196B4
:10BD40000E94821BBE016F5F7F4FC8010E94FC767C
:10BD5000CE0101960E942475C301B20120E13EE0AC
:10BD600040E050E00E9415AD4B015C01B901CE01ED
:10BD700087960E94AB194CE3C42ED12CE12CF12CF8
:10BD8000C501B401A70196010E9415ADB901CE010C
:10BD900001960E94AB196FEA76E0CE0109960E94E7
:10BDA000C375BE016F5F7F4FCE0109960E943F743D
:10BDB000BC01CE0187960E94A874CE0109960E940C
:10BDC0002475CE0101960E942475C301B201A7011A
:10BDD00096010E9415ADCE0101960E94AB196FEA43
:10BDE00076E0CE0109960E94C375BE016F5F7F4F5A
:10BDF000CE0109960E943F74BC01CE0187960E9435
:10BE0000A874CE0109960E942475CE0101960E9465
:10BE1000247560EF77E0CE0109960E94C375BE01DC
:10BE2000695D7F4FCE0109960E943F7463EF77E012
:10BE30000E942974BC01CE0101960E94BA75BE0110
:10BE40006F5F7F4FC8010E94FC76CE0101960E9471
:10BE50002475CE0109960E94247561E078E0C8013E
:10BE60000E94F476CE0101960E943D72B801CE0187
:10BE700001960E9496766CEF77E0C8010E94E0760A
:10BE80000E94755C29833A834B835C836D837E8338
:10BE90008F83988749815A816B817C8121E0CE0113
:10BEA0000F960E942C75BE01615F7F4FCE010996EF
:10BEB0000E94BA7569E078E0CE0109960E94297463
:10BEC000BC0187ED9FE00E94D474CE0109960E94C8
:10BED0002475CE010F960E94247560E178E0CE01B2
:10BEE0000F960E94C37567ED7FE0CE010F960E940A
:10BEF0003F74BC01CE0109960E94BA75BE01675F0E
:10BF00007F4FC8010E94FC76CE0109960E942475DD
:10BF1000CE010F960E9424754D815E816F817885D8
:10BF200021E0CE0109960E942C75BE01675F7F4F0C
:10BF300087ED9FE00E94EB74CE0109960E94247564
:10BF400062E278E0CE010F960E94C37567ED7FE054
:10BF5000CE010F960E943F7463E378E00E9429743B
:10BF6000BC01CE0109960E94BA75BE01675F7F4F82
:10BF7000C8010E94FC76CE0109960E942475CE016C
:10BF80000F960E9424754091380C5091390C6091A5
:10BF90003A0C70913B0C22E0CE010F960E942C755A
:10BFA0006AE378E0CE0145960E94C375BE01615FE9
:10BFB0007F4FCE0145960E943F746CE478E00E946A
:10BFC0002974BC01CE0109960E94BA75BE01675F53
:10BFD0007F4FC8010E94FC76CE0109960E9424750D
:10BFE000CE0145960E942475CE010F960E942475BD
:10BFF0004091340C5091350C6091360C7091370C97
:10C0000022E0CE010F960E942C7565E578E0CE0106
:10C0100045960E94C375BE01615F7F4FCE01459674
:10C020000E943F746CE478E00E942974BC01CE0148
:10C0300009960E94BA75BE01675F7F4FC8010E94D2
:10C04000FC76CE0109960E942475CE0145960E9489
:10C050002475CE010F960E942475E6EF2E16EFEFA1
:10C060003E062CF46AEF7BE0C8010E94411967ED9F
:10C070007AE0C8010E94411999E3E92E90E1F92E76
:10C0800027EDA22E22E0B22ECC24C394D12C47015E
:10C09000F8E08F0E911C82E0A80EB11C809139103F
:10C0A00090913A108C159D050CF464C0B601CE0138
:10C0B0000F960E9411736BE777E0CE0145960E94C0
:10C0C000C375BE01615F7F4FCE0145960E943F74EC
:10C0D0006FEE75E00E942974BC01CE0109960E94A2
:10C0E000BA75BE01675F7F4FC8010E94FC76B70139
:10C0F000645E7F4FCE014B960E94C375BE01655EA4
:10C100007F4FC8010E94FC7663E678E0C8010E9478
:10C11000F476F50160817181660F771F660F771FD6
:10C120006B5B7F4ECE0181960E94C375BE016F5D31
:10C130007F4FC8010E94FC7668E678E0C8010E9443
:10C14000F476CE0181960E942475CE014B960E9412
:10C150002475CE0109960E942475CE0145960E9451
:10C160002475CE010F960E942475FFEFCF1ADF0AC7
:10C1700074018DCFCE0187960E94247581E0809353
:10C180005A0C68EB7BE0C8010E94411910924F0CD9
:10C19000AC960FB6F894DEBF0FBECDBFDF91CF9146
:10C1A0001F910F91FF90EF90DF90CF90BF90AF90D5
:10C1B0009F908F907F906F905F904F903F902F90C7
:10C1C00008956AEF7BE0C8010E944119DACF8F928F
:10C1D0009F92AF92BF92CF92DF92EF92FF920F9316
:10C1E0001F93CF93DF93CDB7DEB7A0970FB6F89428
:10C1F000DEBF0FBECDBF63EC78E081E090E10E942E
:10C20000077363EC78E085EF9FE00E94077348E4D2
:10C21000842E42E0942E59E3A52E50E1B52E6FEC0A
:10C22000E62E62E0F62E77EDC72E72E0D72E01E003
:10C2300010E0F40181919191A191B1914F01892B6D
:10C240008A2B8B2B19F5F60182819381F7012281CC
:10C25000338182179307D1F0880F991FFC01EB54AB
:10C26000F44FD801AA0FBB1FAA50B44F60818C9124
:10C270000E940E78F60182819381F7019383828375
:10C2800064E670E080E090E00E948179F7016281CD
:10C2900073818091391090913A10801791070CF4B6
:10C2A000E5C2CE0145960E941173B801CE010F96EA
:10C2B0000E941173B501645E7F4FCE0109960E9402
:10C2C000C3756FEE75E0CE0101960E94C375BE0185
:10C2D000675F7F4FCE0101960E943F746EE678E063
:10C2E0000E942974BE01615F7F4F0E943F7462EF1C
:10C2F00075E00E942974BE016B5E7F4F0E943F74FF
:10C30000BC0181E090E10E94A874CE0101960E94D8
:10C310002475CE0109960E942475CE010F960E94C5
:10C320002475CE0145960E9424750F5F1F4FF8E0DB
:10C33000AF0EB11C22E0E20EF11C82E0C80ED11C4F
:10C340000430110509F075CFE0915311F0915411AB
:10C35000EE0FFF1FE153FD4F60817181CE01019609
:10C360000E94117346E050E0BE016F5F7F4FCE0127
:10C3700009960E94271CBE01675F7F4F85EF9FE0F3
:10C380000E94A874CE0109960E942475CE010196E0
:10C390000E942475E0915511F0915611EE0FFF1F88
:10C3A000E153FD4F60817181CE0101960E941173AE
:10C3B00046E050E0BE016F5F7F4FCE0109960E94BC
:10C3C000271CBE01675F7F4F85EF9FE00E94A87426
:10C3D000CE0109960E942475CE0101960E94247513
:10C3E0006FEE75E0CE0145960E94C3750E943F7ABC
:10C3F00028EE33E040E050E00E94F3AC69017A019E
:10C4000063EC78E0CE014B960E94C37563EC78E054
:10C4100087E090E10E940773CE0101960E94821B83
:10C4200044E150E0BE016F5F7F4FCE0109960E944C
:10C43000271CBE01675F7F4F87E090E10E94EB748D
:10C44000CE0109960E942475CE0101960E942475A2
:10C450002AE0B701A601CE0109960E94627548E064
:10C4600050E0BE01675F7F4FCE010F960E94271CF0
:10C4700067E070E1CE0101960E94BA75BE01615F6E
:10C480007F4FCE0101960E943F74BC018BEF9FE06D
:10C490000E94D474CE0101960E942475CE010F969D
:10C4A0000E942475CE0109960E9424752AE0B701E6
:10C4B000A601CE0109960E94627561E778E0CE017F
:10C4C00001960E94C375BE01675F7F4FCE01019642
:10C4D0000E943F74BE016B5E7F4F0E943F74BC019F
:10C4E00087E090E10E94A874CE0101960E94247515
:10C4F000CE0109960E9424754091380C5091390C58
:10C5000060913A0C70913B0C21E0CE0101960E94A3
:10C510002C75BE016F5F7F4FCE014B960E94EB746E
:10C52000CE0101960E94247568E778E0CE0101965D
:10C530000E94C375BE01655E7F4FCE0101960E94C9
:10C540003F74BE016B5E7F4F0E943F74BC0187E069
:10C5500090E10E94A874CE0101960E942475BE014C
:10C56000655E7F4FCE0101960E94BA7546E050E0AD
:10C57000BE016F5F7F4FCE0109960E94271CBE014E
:10C58000675F7F4F8BEF9FE00E94A874CE010996F2
:10C590000E942475CE0101960E9424754091340CAE
:10C5A0005091350C6091360C7091370C21E0CE0122
:10C5B00001960E942C75BE016F5F7F4FCE014B9696
:10C5C0000E94EB74CE0101960E94247566E878E023
:10C5D000CE0101960E94C375BE01655E7F4FCE01FC
:10C5E00001960E943F74BE016B5E7F4F0E943F74B4
:10C5F000BC0187E090E10E94A874CE0101960E94E0
:10C600002475BE01655E7F4FCE0101960E94BA750A
:10C6100046E050E0BE016F5F7F4FCE0109960E9459
:10C62000271CBE01675F7F4F8BEF9FE00E94A874BD
:10C63000CE0109960E942475CE0101960E942475B0
:10C64000609190027091910280918E0290918F0280
:10C650000E9417169093450C8093440C892B71F01F
:10C66000609190027091910280918E0290918F0260
:10C670000E9417169093450C8093440C8091440CB3
:10C680009091450C8C3F9F4F0CF410C10E94755C3B
:10C6900029833A834B835C836D837E838F83988762
:10C6A00049815A816B817C8121E0CE0109960E94EB
:10C6B0002C75BE01675F7F4FCE014B960E94EB74D5
:10C6C000CE0109960E94247560E978E0CE010996B2
:10C6D0000E94C375BE01655E7F4FCE0109960E9420
:10C6E0003F74BE016B5E7F4F0E943F74BC0187E0C8
:10C6F00090E10E94A874CE0109960E942475BE01A3
:10C70000655E7F4FCE0109960E94BA7546E050E003
:10C71000BE01675F7F4FCE010F960E94271CBE01AE
:10C72000615F7F4F8BEF9FE00E94A874CE010F9650
:10C730000E942475CE0109960E9424754D815E8168
:10C740006F81788521E0CE0109960E942C75BE018B
:10C75000675F7F4FCE014B960E94EB74CE01099626
:10C760000E9424756BE978E0CE0109960E94C3759A
:10C77000BE01655E7F4FCE0109960E943F74BE01E7
:10C780006B5E7F4F0E943F74BC0187E090E10E9486
:10C79000A874CE0109960E942475BE01655E7F4F84
:10C7A000CE0109960E94BA7546E050E0BE01675F6F
:10C7B0007F4FCE010F960E94271CBE01615F7F4F05
:10C7C0008BEF9FE00E94A874CE010F960E94247503
:10C7D000CE0109960E94247561E070E187E090E146
:10C7E0000E94A8746FEE75E0CE0101960E94C37599
:10C7F00065EF7FE0CE0101960E943F74BC018BEF94
:10C800009FE00E94A874CE0101960E9424756BEFF0
:10C810007FE0CE0101960E94BA75CE0101960E947A
:10C82000E915CE0101960E9424756AE070E080E06F
:10C8300090E00E948179CE014B960E942475CE0132
:10C8400045960E942475A0960FB6F894DEBF0FBEE1
:10C85000CDBFDF91CF911F910F91FF90EF90DF90AF
:10C86000CF90BF90AF909F908F900895CE01459646
:10C870000E941173B801CE010F960E941173B50189
:10C880006C5E7F4FCE0109960E94C3756FEE75E016
:10C89000CE0101960E94C375BE01675F7F4FCE0136
:10C8A00001960E943F746DE678E01ACD61EA78E067
:10C8B00087E090E10E949E7460EB78E08BEF9FE050
:10C8C0000E949E7467EB78E087E090E10E949E747E
:10C8D00060EB78E08BEF9FE00E949E747DCFBF926B
:10C8E000CF92DF92EF92FF920F931F93CF93DF933C
:10C8F000CDB7DEB7C455D1090FB6F894DEBF0FBE71
:10C90000CDBF6C018B0165965FAF4EAF659780918F
:10C91000320C9091330C01969093330C8093320C2F
:10C9200080914F0C81113CC0BB24B394B0924F0C4A
:10C930001092330C1092320C63EC78E0CE01895BDC
:10C940009F4F0E94C37563EC78E0CE01835B9F4FDD
:10C950000E94C37550E040E060E274E0C6010E94AE
:10C960005A190130110509F0A6C063EC78E087E0A0
:10C9700090E10E9407736596EEADFFAD65978081EB
:10C98000811124C00E94E760B0925A0CCE01835BF3
:10C990009F4F0E942475CE01895B9F4F0E94247592
:10C9A0000FB6F894DEBF0FBECDBFCC5ADF4F0FB627
:10C9B000F894DEBF0FBECDBFDF91CF911F910F91D5
:10C9C000FF90EF90DF90CF90BF9008956596EEAD09
:10C9D000FFAD65978081882309F467C000E210E00D
:10C9E0009E012F5F3F4F40E250E0BE016F5D7F4FE1
:10C9F000CE018D5A9F4F0E946571049739F3BE0195
:10CA00006F5D7F4FCE018F5B9F4F0E94C375BE014C
:10CA10006F5B7F4FCE01895B9F4F0E94EB74CE010D
:10CA20008F5B9F4F0E942475BE016F5F7F4FCE01C9
:10CA30008F5B9F4F0E94C375BE016F5B7F4FCE011E
:10CA4000835B9F4F0E94EB74CE018F5B9F4F0E94D0
:10CA50002475BE01695B7F4F87E090E10E94A87456
:10CA600063968EAD9FAD6397892B09F4AFCF62EFCC
:10CA700075E0CE018F5B9F4F0E94C375BE01635B63
:10CA80007F4FCE018F5B9F4F0E943F746FEE75E02A
:10CA90000E942974BC0187E090E10E94A874CE0135
:10CAA0008F5B9F4F0E94247591CF67E070E183EE0A
:10CAB0009FE00E94D47410924F0C68CF2F923F9247
:10CAC0004F925F926F927F928F929F92AF92BF929E
:10CAD000CF92DF92EF92FF920F931F93CF93DF934A
:10CAE000CDB7DEB7C258D1090FB6F894DEBF0FBE7E
:10CAF000CDBF6C015B0188EE482E83E0582E612C7F
:10CB0000712C09EF13E09BE5892E912C8C0E9D1E54
:10CB10008CE0880E911C1B019FEF291A390AD6015F
:10CB20005996ED90FC90F7018581823008F493C00E
:10CB300082859385A485B5858F719927AA27BB2700
:10CB4000892B8A2B8B2B09F086C040E250E0BE0176
:10CB50006F5F7F4FC7010E94DA87803209F07BC088
:10CB60008981882309F477C0853E79F38E3269F391
:10CB70008C8583FDEACF22961FAE1EAE229785E8F4
:10CB800093E09FAF8EAF24961FAE2497BE016F5FD8
:10CB90007F4FE0E080E04EE2DB019D91BD019032ED
:10CBA000A1F0883049F426E730E02C0F3D1F2E0F0E
:10CBB000311DD9014C93EF5F26E730E02C0F3D1F6C
:10CBC0002E0F311DD9019C93EF5F8F5F8B3021F7C2
:10CBD00086E790E08C0F9D1F8E0F911DFC01108247
:10CBE000D60159966D917C9121E0AE014A585F4F74
:10CBF000CE01CE960E94E189882369F1BE01625C74
:10CC00007F4FCE0181960E94488DAE014A585F4FFA
:10CC1000BE016F5D7F4FCE01855A9F4F0E94B68D3A
:10CC2000CE01855A9F4F0E94988D882309F4ACC08D
:10CC3000F12CFA141B042CF569E0CE0101960E9438
:10CC40008F75CE0101960E940016CE0101960E94BA
:10CC50002475F394EECF6F961FAE1EAE6F97A3961A
:10CC60004CAE5DAE6EAE7FAEA3976D961FAF0EAFAE
:10CC70006D97E6961FAE1EAEE697A8961FAEA897D4
:10CC8000CFCFB401CE0101960E94C375CE010196AB
:10CC90000E940016CE0101960E942475E696EEAD24
:10CCA000FFADE697309709F447C08581823008F4DC
:10CCB00043C06AE674E0CE0101960E94C375CE01BE
:10CCC00001960E94E915CE0101960E9424756F9687
:10CCD0008EAD9FAD6F979C838B83A3968CAD9DADDE
:10CCE000AEADBFADA3978D839E83AF83B887A79664
:10CCF0008CAD9DADAEADBFADA79789879A87AB8749
:10CD0000BC871A8309838DE0F401DE011D96019032
:10CD10000D928A95E1F7E6968EAD9FADE6979B8FD3
:10CD20008A8FB101CE0101960E945E65CE01855ABF
:10CD30009F4F0E94A48DF3CE61EC78E0CE01019666
:10CD40000E94C375CE0101960E940016CE01019685
:10CD50000E942475E696EEADFFADE69740E050E008
:10CD6000BA01309721F04389548965897689CE01CB
:10CD700001960E943D73CE0101960E94E915CE01F5
:10CD800001960E942475D2CFCE57DF4F0FB6F8948C
:10CD9000DEBF0FBECDBFDF91CF911F910F91FF90EE
:10CDA000EF90DF90CF90BF90AF909F908F907F904B
:10CDB0006F905F904F903F902F9008956F927F9269
:10CDC0008F929F92AF92BF92CF92DF92EF92FF929B
:10CDD0000F931F93CF93DF93CDB7DEB7C456D1091E
:10CDE0000FB6F894DEBF0FBECDBF40E052EC61E05D
:10CDF00070E08CE39DE00E94217140E855E260E024
:10CE000070E08FE99CE00E94217161E088E00E945F
:10CE10002B7961E089E00E942B7960E08AE30E942F
:10CE20002B7961E088E00E940E7860E089E00E9442
:10CE30000E7861E08AE00E942B7961E08BE00E942D
:10CE40002B7960E08BE30E942B7961E08AE00E94FD
:10CE50000E7860E08BE00E940E780E94147984EFD7
:10CE600091E0909367028093660264EC7AE08CE331
:10CE70009DE00E941E7763EC79E08CE39DE00E94C8
:10CE8000247660ED77E080E090E00E9481798CE389
:10CE90009DE00E94F76D982E2EE1E22EF12C91106C
:10CEA0000BC08CE39DE00E94F76D982E6EE170E060
:10CEB00080E090E00E94817921E0E21AF10879F7A0
:10CEC000809166029091670209E310E1FC01E95349
:10CED000F0416F01C601800F911F0E94CDACF80197
:10CEE00081938F01F1E10B361F07A1F76091531178
:10CEF00070915411072E000C880B990B0E94B0AB57
:10CF00009B01AC010E9470AE882331F081E090E07B
:10CF10009093541180935311609155117091561153
:10CF2000072E000C880B990B0E94B0AB9B01AC0143
:10CF30000E9470AE882331F082E090E09093561109
:10CF40008093551125E79216B1F060914F117091C1
:10CF5000501180915111909152110E94B0AB9B01E0
:10CF6000AC010E9470AE811106C080913910909181
:10CF70003A108197E8F08DB79EB7825391400FB673
:10CF8000F8949EBF0FBE8DBFADB7BEB7119682E3BA
:10CF900091E0E9E3F0E101900D920197E1F70E9441
:10CFA00089240FB6F894DEBF0FBECDBF95E7992E4A
:10CFB0002DB73EB7225331400FB6F8943EBF0FBE97
:10CFC0002DBFADB7BEB7119682E391E0E9E3F0E182
:10CFD00001900D920197E1F70E94B91D0FB6F894E8
:10CFE000DEBF0FBECDBF95E7991619F0E3E79E129D
:10CFF0001BC02DB73EB7225331400FB6F8943EBF49
:10D000000FBE2DBFADB7BEB7119682E391E0E9E345
:10D01000F0E101900D920197E1F70E940A2B0FB603
:10D02000F894DEBF0FBECDBF62EB7AE08FEE9FE0DB
:10D030000E94AF746CE97AE089EE9FE00E94AF74C1
:10D040000E94147964EC78E08CE39DE00E94E07625
:10D05000D12CC12C17E201E000939B0C10939D0C86
:10D0600010929C0C10929E0C81E00E94977E811180
:10D07000AEC160ED78E08CE39DE00E94F476812FF4
:10D080000E947F761093F3116CEE78E08CE39DE0C4
:10D090000E94F476812F0E947F769FEFC91AD90AE9
:10D0A0001F5F1034C9F661E279E0CD2811F067E323
:10D0B00079E08CE39DE00E94E0760E941479109262
:10D0C000F4118091F811823018F098E09093F411E7
:10D0D0009091F911992339F0813029F48091F4115C
:10D0E00084608093F41162E370E080E090E00E943D
:10D0F00081796091FA118FEE91E10E94877F68EE4D
:10D1000073E080E090E00E94817960E38FEE91E12E
:10D110000E949B7F0BE416E4C8010197F1F760E3DE
:10D120008FEE91E10E949B7FC8010197F1F760E3C8
:10D130008FEE91E10E949B7F83E592E00197F1F7EA
:10D1400060E28FEE91E10E949B7F8091F4118062FA
:10D150000E94B47F84E08093F5118CE00E94B47F3C
:10D1600081E00E94B47F0BE31FE1C8010197F1F752
:10D1700082E08093F61186E00E94B47F82E00E94F4
:10D18000B47FC8010197F1F780E40E94B47F0EE5F7
:10D1900012E086E6C82E82E0D82EF80161918F0158
:10D1A0008FEE91E10E94F27FC016D106B1F70E9486
:10D1B000E5080E94D50864E670E080E090E00E94F7
:10D1C000817964E87AE0CE0101960E94B175CE01C2
:10D1D00001960E94E915CE0101960E94247561E036
:10D1E00085E30E942B7961E085E30E940E7861E07F
:10D1F0008AE00E942B7961E08AE00E940E7861E06B
:10D2000089E30E942B798091D10E803308F052C0BF
:10D2100061E089E30E942B798091D10E282F30E0C4
:10D22000F901EE0FFF1FE20FF31FE25CF14F908157
:10D23000907C996390831092D20E1092D30E2CE0C2
:10D24000622F0E9475AE829FB00111249B012E0DAA
:10D250003F1DF901EE0FFF1FE20FF31FE25CF14FDC
:10D26000908196FD19C0FFEFEF1AFF0A2CE0E2163D
:10D27000F10461F7813009F0B7C01092800082E0BC
:10D28000809381001092850010928400B19A809161
:10D290006F00826080936F00E091D10E8E2F90E03E
:10D2A000FC01EE0FFF1FE80FF91FE25CF14F8081D8
:10D2B0008064808368EC70E080E090E00E94817977
:10D2C00068EE73E080E090E00E94817963E77AE0A5
:10D2D000CE0101960E94B1754AE050E06FEF7FEFFA
:10D2E000CE0101960E943220CE0101960E94247543
:10D2F0001092F20D1092F00D1092ED0D1092EC0DB7
:10D3000084E08093EB0D0E943F7A8B0161E0809175
:10D31000EB0D0E942B7961E08091EB0D0E940E785D
:10D320000E94C71482E58093E50D1092E60D80916E
:10D33000E50D9091E60D0E94E509AAE0FA2E8FEF27
:10D340000E947709FA94F110FACF87EE9DE00E94CF
:10D35000658120E030E0A90160E087EE9DE00E9459
:10D36000A781F82E8093F10D31E0831709F468C08E
:10D370000E943F7A601B710B613D774050F381E062
:10D380008093EC0D87EE9DE00E947B8165E67AE05C
:10D39000CE0101960E94B175CE0101960E94E91559
:10D3A000CE0101960E94247564E57AE0CE010196D3
:10D3B0000E94B1754AE050E06FEF7FEFCE01019619
:10D3C0000E940909CE0101960E9424754BC1843048
:10D3D00009F066CE66E079E08CE39DE00E94F47689
:10D3E000812F0E947F765CCE823061F41092900093
:10D3F00080939100109295001092940088BB8093C6
:10D4000071004ACF833069F41092A00082E08093CB
:10D41000A1001092A5001092A40089BB8093720015
:10D420003BCF811139CF1092200182E080932101FE
:10D4300010922501109224018ABB809373002CCF97
:10D440002AEA31E040E050E068E087EE9DE00E948B
:10D45000A78182FF2AC0F092F20D8091F20DC12CBB
:10D46000D12CE12CE0E4FE2E823019F0C12CD12C1D
:10D47000760120E030E0A90167E387EE9DE00E949D
:10D48000A781A701960169E287EE9DE00E94A7812E
:10D490008093F10D8823D1F00E943F7A601B710BBD
:10D4A000613D774030F388E06BCFF4E0FF2E0E94BF
:10D4B00089818093F10DFA94F110F9CF8A3A11F035
:10D4C00082E05ECF82E08093F20DC7CF8091F20DB3
:10D4D0008230D1F420E030E0A9016AE387EE9DE0DC
:10D4E0000E94A781882311F086E04ACF0E9489819B
:10D4F000807C803C19F483E08093F20D0E94898146
:10D500000E9489810E94898187EE9DE00E947B8133
:10D5100080E58093E50D1092E60D81E00E949583F1
:10D52000882309F49BC28091160E81112FCF809120
:10D530000A0E803109F099C282E08093160E109293
:10D54000280E1092290E10922A0E10922B0E809106
:10D550000B0E90910C0EB0E0A0E075E0880F991FC3
:10D56000AA1FBB1F7A95D1F78093240E9093250EA6
:10D57000A093260EB093270E83EF9DE090932D0E7F
:10D5800080932C0E81E08093150E1092170E10924E
:10D59000180E1092190E10921A0E10921B0E109265
:10D5A0001C0E10921D0E10921E0E10921F0E109245
:10D5B000200E1092210E1092220E1092230E68E47B
:10D5C0007AE0CE0101960E94B175CE0101960E94CB
:10D5D000E915CE0101960E94247541E06AE674E0E7
:10D5E000CE0101960E94EB8DBE016F5F7F4F88EBED
:10D5F00091E10E9410198091BA119091BB119C8306
:10D600008B838091BC119091BD11A091BE11B091FE
:10D61000BF118D839E83AF83B8878091C011909195
:10D62000C111A091C211B091C31189879A87AB87AC
:10D63000BC8789EF93E09A8389838DE0E4ECF1E184
:10D64000DE011D9601900D928A95E1F78091D1112E
:10D650009091D2119B8F8A8F70E060E0CE0101968D
:10D660000E945E6568EE73E080E090E00E94817940
:10D6700043E162EB72E0CE0101960E94EB8DBE01A8
:10D680006F5F7F4F83ED91E10E9410196FE07AE0A8
:10D690008DED9FE00E94AF7464E07AE08DED9FE035
:10D6A0000E94527483ED91E10E94988D882309F4C1
:10D6B0000DC21EAE1DAE85E893E09CAF8BAF2196E8
:10D6C0001FAE219719A218A29F8F8E8F1BA2812CAB
:10D6D000712C7E01EBE3EE0EF11C01E11EE05C011A
:10D6E000882D972DFC01EE54FD4F20812F3209F437
:10D6F0000196DC01AE54BD4FFE01E85AFF4F30E009
:10D7000020E06F014D914F3249F0442339F00196EA
:10D710002F5F3F4F41932C303105A1F72C0D3D1D5C
:10D72000F9011082FC01EE54FD4F20812F3209F4E3
:10D730000196882E792E8E549D4FFC0160801C82AC
:10D740001B82BA82A9821E8221E0A601B801CE0105
:10D7500001960E94E189882309F4D5C1CE01019682
:10D760000E94CD896110A0C12EE00131120719F08D
:10D77000C8010E94CD8983ED91E10E94A48D66E9E4
:10D7800070E080E090E00E9481791092560C04E6EF
:10D7900010E091100BC08CE39DE00E94F76D982E75
:10D7A00064E170E080E090E00E948179015011090D
:10D7B00081F76FED79E0CE0101960E94B17548ECDA
:10D7C00050E070E060E0CE0101960E940909CE01B0
:10D7D00001960E94247532E781E0931280E00E9456
:10D7E000330882E090E00E945E7C6CE271E080E0B1
:10D7F00090E00E94817983E090E00E945E7C6CE280
:10D8000071E080E090E00E94817901E010E01093E7
:10D810006F0200936E0210935D0200935C0265E25A
:10D8200077E082E99FE00E94077362E97FE0CE0122
:10D8300001960E94BA7562E070E0CE0101960E94E6
:10D84000582FCE0101960E9424756EEC79E0CE012E
:10D8500001960E94B175CE0101960E94E915CE0194
:10D8600001960E9424756EEB79E0CE0101960E942C
:10D87000B17548EC50E070E060E0CE0101960E9486
:10D880003220CE0101960E94247561E876E082E99B
:10D890009FE00E94077362E97FE0CE0101960E943B
:10D8A000BA7563E070E0CE0101960E94582FCE0158
:10D8B00001960E94247510936F0200936E0268EA2D
:10D8C00079E0CE0101960E94B175CE0101960E94C9
:10D8D000E915CE0101960E9424756DE979E0CE012B
:10D8E00001960E94B1754AE050E06FEF7FEFCE01E4
:10D8F00001960E943220CE0101960E94247568EEA6
:10D9000073E080E090E00E9481790E94E1270E940C
:10D91000E9288DB79EB7825391400FB6F8949EBF09
:10D920000FBE8DBFADB7BEB7119682E391E0E9E3BC
:10D93000F0E101900D920197E1F70E940A2B1092FD
:10D940004E0C87ED9DE59093470F8093460F2091F5
:10D95000680F0FB6F894DEBF0FBECDBF2830D8F4E5
:10D96000822F90E0FC01EE0FFF1FEE0FFF1FE85B20
:10D97000F04F40E559E0518340832F5F2093680FBB
:10D98000880F991F880F991FFC01E65BF04F81EE0D
:10D9900099E1918380832091680F2830D8F4822FF9
:10D9A00090E0FC01EE0FFF1FEE0FFF1FE85BF04F52
:10D9B00046E559E0518340832F5F2093680F880F1D
:10D9C000991F880F991FFC01E65BF04F8FE694E6E4
:10D9D0009183808388ED9EE00E94ED116BE879E0F1
:10D9E000CE0101960E94B175CE0101960E94E91503
:10D9F000CE0101960E94247510924F0C0E94187C53
:10DA00006093500C7093510C8093520C9093530C74
:10DA1000809138118093580C882351F00E94187C13
:10DA20006093460C7093470C8093480C9093490C7C
:10DA3000CC59DF4F0FB6F894DEBF0FBECDBFDF91DC
:10DA4000CF911F910F91FF90EF90DF90CF90BF90FB
:10DA5000AF909F908F907F906F90089580E00E948C
:10DA60009583882309F492CC5ECD803209F08ECC68
:10DA700083E08093160E40910D0E50910E0E609132
:10DA80000F0E7091100E4093280E5093290E609344
:10DA90002A0E70932B0E24E23EE083EF9DE00E945D
:10DAA000E185811169CD72CC21E0A601B801C701E1
:10DAB0000E94E189D82EFEE001311F0709F44DC014
:10DAC000C8010E94CD89D1104DC024C06FEE79E00D
:10DAD000CE0101960E94B175CE0101960E940016FA
:10DAE000CE0101960E94247562EB72E0CE01019690
:10DAF0000E94C375CE0101960E94E915CE010196E0
:10DB00000E94247542CEFEE001311F0719F0C801C2
:10DB10000E94CD896EE379E0CE0101960E94C37523
:10DB2000CE0101960E940016CE0101960E94247536
:10DB300062EB72E0CE0101960E94C375CE010196A0
:10DB40000E94E915CE0101960E9424756DED7FE0DB
:10DB500083ED91E10E940A770ECE8823D9F28E01DF
:10DB6000025E1F4F902F812F8701E92EF82EB8CD2E
:10DB7000089508950895AF92BF92CF92DF92EF92E9
:10DB8000FF920F931F93CF93DF936C017B018B0167
:10DB9000040F151FEB015E01AE18BF08C017D107B7
:10DBA00059F06991D601ED91FC910190F081E02D41
:10DBB000C6011995892B79F7C501DF91CF911F9186
:10DBC0000F91FF90EF90DF90CF90BF90AF900895AE
:10DBD000FC01538D448D252F30E0842F90E0821B73
:10DBE000930B541710F0CF96089501970895FC01F8
:10DBF000918D828D981761F0A28DAE0FBF2FB11D50
:10DC00005D968C91928D9F5F9F73928F90E00895A7
:10DC10008FEF9FEF0895FC01918D828D981731F061
:10DC2000828DE80FF11D858D90E008958FEF9FEFB5
:10DC30000895FC01918D228D892F90E0805C9F4F8B
:10DC4000821B91098F73992708958FE99CE00E94A8
:10DC5000196E21E0892B09F420E0822F08958CE3CE
:10DC60009DE00E94196E21E0892B09F420E0822FAB
:10DC70000895FC01A48DA80FB92FB11DA35ABF4F61
:10DC80002C91848D90E001968F739927848FA689BB
:10DC9000B7892C93A089B1898C91837080648C930F
:10DCA000938D848D981306C00288F389E02D8081BE
:10DCB0008F7D80830895EF92FF920F931F93CF93F0
:10DCC000DF93EC0181E0888F9B8D8C8D98131AC0B7
:10DCD000E889F989808185FF15C09FB7F894EE899E
:10DCE000FF896083E889F9898081837080648083FB
:10DCF0009FBF81E090E0DF91CF911F910F91FF9046
:10DD0000EF900895F62E0B8D10E00F5F1F4F0F73ED
:10DD10001127E02E8C8D8E110CC00FB607FCFACFA8
:10DD2000E889F989808185FFF5CFCE010E94396E9F
:10DD3000F1CFEB8DEC0FFD2FF11DE35AFF4FF08279
:10DD40009FB7F8940B8FEA89FB8980818062CFCFDF
:10DD5000CF93DF93EC01888D8823B9F0AA89BB8922
:10DD6000E889F9898C9185FD03C0808186FD0DC00D
:10DD70000FB607FCF7CF8C9185FFF2CF808185FF2E
:10DD8000EDCFCE010E94396EE9CFDF91CF9108959A
:10DD900080E090E0892B29F00E942F6E81110E9473
:10DDA000000080E090E0892B49F080E090E0892B32
:10DDB00029F00E94000081110E94000080E090E0A4
:10DDC000892B49F080E090E0892B29F00E94000027
:10DDD00081110E94000080E090E0892B29F00E94D0
:10DDE000256E81110C94000008958150823108F055
:10DDF0005AC0E82FF0E08827EF5FF0498F4F0C946E
:10DE000095AE216F256F136F196F1D6F536F286FBC
:10DE10002E6F326F386F3C6F406F466F4A6F536F93
:10DE20004E6F546F586F809180008F778093800081
:10DE30000895809180008F7DF9CF80918000877F49
:10DE4000F5CF84B58F7784BD089584B58F7DFBCFE2
:10DE50008091B0008F778093B00008958091B000DA
:10DE60008F7DF9CF809190008F77809390000895F7
:10DE7000809190008F7DF9CF80919000877FF5CFC2
:10DE80008091A0008F778093A00008958091A000DA
:10DE90008F7DF9CF8091A000877FF5CF8091200101
:10DEA0008F77809320010895809120018F7DF9CF95
:10DEB00080912001877FF5CFCF93DF93282F30E02B
:10DEC000F901E75FF24F8491F901ED53F34FD491DB
:10DED000F901E358F34FC491CC23A1F081110E94C2
:10DEE000F56EEC2FF0E0EE0FFF1FED59F34FA5910B
:10DEF000B491EC91ED2381E090E009F480E0DF91B2
:10DF0000CF91089580E090E0FACF20912812260F5B
:10DF10003327331F21323105ECF42091950CFC019D
:10DF200090E080E0243069F082E00895A09128120A
:10DF30002191AC01485F5D4EA40FB52FB11D2C930C
:10DF40000196861798F380912812680F6093281223
:10DF500080E0089581E008950895E091550C809146
:10DF6000540CE81730F4F0E0EF5FF34F808190E05D
:10DF700008958FEF9FEF08959091550C8091540C68
:10DF80002FEF3FEF981748F4E92FF0E0EF5FF34FE2
:10DF9000208130E09F5F9093550CC90108958091D6
:10DFA000540C9091550C891B990B0895CF92DF92D8
:10DFB000EF92FF920F931F93CF93DF937C01CB01DE
:10DFC0008A0120919B0C222389F0EB016B01C40E86
:10DFD000D51ECC15DD0569F06991D701ED91FC9155
:10DFE0000190F081E02DC7011995F3CF642F0E94B5
:10DFF000856FC801DF91CF911F910F91FF90EF9036
:10E00000DF90CF900895CF93DF931F92CDB7DEB707
:10E01000698320919B0C2223F9F020919E0C2032E1
:10E0200058F021E030E0FC013383228390E080E06F
:10E030000F90DF91CF91089580919C0CE82FF0E034
:10E04000E155FA4E998190838F5F80939C0C809369
:10E050009E0C81E090E0ECCF61E0CE0101960E9441
:10E06000856FF7CFDC015996ED91FC913097B9F0AF
:10E0700083899489A589B689428553856485758588
:10E08000841B950BA60BB70B811520E89207A10501
:10E09000B10538F08FEF9FE7A0E0B0E0089590E081
:10E0A00080E00895CF93DF931F92CDB7DEB76983E9
:10E0B000DC01ED91FC910280F381E02D41E050E024
:10E0C000BE016F5F7F4F19950F90DF91CF9108953B
:10E0D0000E94BEB00F931F93CF93DF93EC01888112
:10E0E0009981009759F02A813B812617370730F034
:10E0F00081E0DF91CF911F910F9108958B016F5FA8
:10E100007F4F0E94DDAF009759F0998388831B836E
:10E110000A832C813D81232B59F7FC011082E8CF23
:10E1200080E0E7CFEF92FF920F931F93CF93DF939F
:10E130006115710541F480E0DF91CF911F910F913E
:10E14000FF90EF90089541155105B1F07B01EC016E
:10E150000C811D81040F151FB8010E946A7088236D
:10E1600051F3288139818C819D81B701820F931FE2
:10E170000E940EB11D830C8381E0DECFCF93DF932D
:10E18000EC0188819981009711F00E9454AF1982A7
:10E1900018821D821C821B821A82DF91CF91089502
:10E1A000EF92FF920F931F93CF93DF93EC017B01CC
:10E1B0008A01BA010E946A7081110BC0CE010E94CF
:10E1C000BE70CE01DF91CF911F910F91FF90EF9024
:10E1D00008951D830C83B701888199810E940EB137
:10E1E000F0CFCF92DF92EF92FF920F931F93CF93D6
:10E1F000DF93EC017A018B016C01C40ED51ECC15A6
:10E20000DD05A9F00E9475098FE00E9477098D2F26
:10E210000E9477098C2F0E947709219680E00E9446
:10E220007709F80181938F010E947309E8CFC70134
:10E23000DF91CF911F910F91FF90EF90DF90CF90E2
:10E240000895CF93DF93EC019A01AB01E889F98936
:10E2500082E08083211581EE38074105510581F167
:10E2600060E079E08DE390E00E94F3AC2150310949
:10E27000410951095695479537952795EC85FD85B8
:10E280001082EE85FF852083188EEC89FD8986E05B
:10E290008083EA89FB89808180618083EA89FB89A8
:10E2A000808188608083EA89FB898081806880839F
:10E2B000EA89FB8980818F7D8083DF91CF910895EA
:10E2C000E889F989108220E1D9CF2F923F924F92AD
:10E2D0005F926F927F928F929F92AF92BF92CF92F6
:10E2E000DF92EF92FF920F931F93CF93DF9300D0B3
:10E2F000CDB7DEB71C013B014A0129015801FC01E1
:10E30000C080D18070E060E0C3010E94F3B0A8013A
:10E3100070E060E0C2010E94F3B0F601808110E07D
:10E3200000E0811162C004E010E004C07601F10158
:10E33000F182E082C8010F900F900F90DF91CF9192
:10E340001F910F91FF90EF90DF90CF90BF90AF9013
:10E350009F908F907F906F905F904F903F902F9005
:10E3600008956B3209F482C06D3309F04EC081818B
:10E370008823E9F2F7018FEFE81AF80A6081653225
:10E3800009F452C00CF048C0662309F456C082E07C
:10E39000A816B1040CF061C0012B09F46BC003E0B6
:10E3A00010E0E8CF81818983882309F282818A8302
:10E3B0007601811104C0F2E0EF0EF11CB8CF83E0CA
:10E3C000E80EF11C1B8240E150E070E060E0CE01FD
:10E3D00001960E946CA319C0F3016083F1E08F1ACB
:10E3E0009108C30101963C0167017601FFEFEF1A26
:10E3F000FF0AF6016081663209F499CF0CF0B1CFC3
:10E40000662309F493CF653269F2F2E08F16910426
:10E410001CF701E010E0E8CF663209F488CF6B32D8
:10E4200009F0B5CF60E2B3CF81818983882301F100
:10E4300082818A83811103C032967F0178CF7F0168
:10E4400093E0E90EF11C1B8240E150E070E060E0D7
:10E45000CE0101960E946CA39ACFF2016083F1E095
:10E46000AF1AB108C20101962C0184CF60E2CDCF72
:10E47000F701E3CF02E010E07DCFCF93DF93EC0113
:10E4800087E194E0998388831A821B821C821D8213
:10E4900080E590E00E94E509BE016E5F7F4F44E099
:10E4A00050E08FE090E00E94F1700E94E409CE01FC
:10E4B000DF91CF9108950F931F93CF93DF93411571
:10E4C000510541F0FC01048115810115110539F454
:10E4D000FB011082DF91CF911F910F910895415060
:10E4E00051094017510708F48A01EB01FC016081D2
:10E4F0007181A801CE010E9423B1C00FD11F1882E3
:10E50000E9CFCF93C82F462F61E070E00E947E09CB
:10E5100061E070E08C2F0E9499098111F9CFCF91B1
:10E520000895FF920F931F93CF93DF93F82E10E07F
:10E5300000E08F2D0E94CA09EC01892B21F08F2D5C
:10E540000E94CA098C01C017D10799F7CE01DF914B
:10E55000CF911F910F91FF900895AF92BF92CF92EC
:10E56000DF92EF92FF920F931F93CF93DF931F924F
:10E570001F92CDB7DEB77A836983BA01A901E98119
:10E58000FA81F770082F10E0000F111F0D59134F7B
:10E59000D8018D919C918E0F9F1F9F01240F351FD5
:10E5A00021303840A0F05A016B0160E078E07B0137
:10E5B000EE1AFF0AA701B6010E94F170A5014E19DB
:10E5C0005F09B6016E0D7F1DF801808191810F906A
:10E5D0000F90DF91CF911F910F91FF90EF90DF90FF
:10E5E000CF90BF90AF900C94F17020E3FC0120839A
:10E5F0003296862F82958F706F706A3030F4605D2E
:10E600006293682F8111F5CF0895695CF9CFFB0102
:10E6100001900020E9F73197AF01461B570B0C948E
:10E62000D0700F931F93CF93DF93CDB7DEB7629770
:10E630000FB6F894DEBF0FBECDBF8C01CB01F80141
:10E640001182108213821282158214824AE0BE0166
:10E650006F5F7F4F0E94B3A4BE016F5F7F4FC80101
:10E660000E94077362960FB6F894DEBF0FBECDBF4F
:10E67000DF91CF911F910F9108950F931F93CF9327
:10E68000DF93CDB7DEB7A1970FB6F894DEBF0FBE0C
:10E69000CDBF8C01CB01BA01F80111821082138227
:10E6A0001282158214822AE0AE014F5F5F4F0E94F2
:10E6B000EDA4BE016F5F7F4FC8010E940773A19652
:10E6C0000FB6F894DEBF0FBECDBFDF91CF911F9183
:10E6D0000F910895FC0180819181009711F00C94B5
:10E6E0006FA460E070E0CB010895FC01808191810E
:10E6F000009711F00C9473A460E070E0CB010895D2
:10E70000AF92BF92CF92DF92EF92FF920F931F933F
:10E71000CF93DF93DC01CD90DC901197C114D1042D
:10E7200039F01496CD91DC918C017601209761F43B
:10E73000DF91CF911F910F91FF90EF90DF90CF90DD
:10E74000BF90AF90089575015701BFEFAB1ABB0A98
:10E75000F7018081082E000C990B0E949AA4892B46
:10E7600091F72197CC0DDD1D8881082E000C990BA7
:10E770000E949AA4892B29F0CE15DF0510F021976D
:10E78000F3CFAE014F5F5F4F4E195F09D801159669
:10E790005C934E931497CE14DF0420F4B701C601A6
:10E7A0000E94D8B0D801ED91FC91119714968D91EB
:10E7B0009C91E80FF91F1082BBCFFC0124813581A9
:10E7C0006217730748F480819181009729F0860FC2
:10E7D000971FFC018081089580E00895FC01248149
:10E7E0003581FB014481558124173507A0F0FC01D8
:10E7F00080819181009779F0FB01608171816115C1
:10E80000710549F0241B350B820F931F0E9405B13F
:10E8100021E0892B09F020E0822F0895FB0144813B
:10E820005581FC01248135812417350778F08081DA
:10E830009181009759F0FB0160817181611571052B
:10E8400029F00E9415B121E0892B09F020E0822FE8
:10E850000895CF93DF93EC01FB0101900020E9F7CD
:10E860003197AF01461B570B0E949270811103C074
:10E87000CE010E94BE70CE01DF91CF910895CF935B
:10E88000DF93EC01FB0144815581608171810E941D
:10E890009270811103C0CE010E94BE70CE01DF9143
:10E8A000CF910895EF92FF920F931F93CF93DF9331
:10E8B000EC017B01CB010E94AAA40097A9F00C8176
:10E8C0001D81080F191FB801CE010E946A708823AC
:10E8D00061F0288139818C819D81B701820F931F5E
:10E8E0000E94A3A41D830C8381E0DF91CF911F912F
:10E8F0000F91FF90EF900895CF93DF931F921F9297
:10E90000CDB7DEB769831A8241E050E0BE016F5F88
:10E910007F4F0E9492700F900F90DF91CF910895DA
:10E92000CF93DF93EC010E947C74811103C0CE0170
:10E930000E94BE70CE01DF91CF910895FB0101903E
:10E940000020E9F73197AF01461B570B0C949270EA
:10E95000FB0144815581608171810C949270EF922A
:10E96000FF920F931F93CF93DF93EC018B01CB01A9
:10E970000E94AAA47C01BC01CE010E946A70811190
:10E980000BC0CE010E94BE70CE01DF91CF911F91CE
:10E990000F91FF90EF900895FD82EC82B80188817D
:10E9A00099810E94A3A4F0CFCF93DF93EC01FB01E8
:10E9B0008617970749F0608171816115710541F0F3
:10E9C000448155810E94D070CE01DF91CF9108958E
:10E9D0000E94BE70F9CF0F931F93CF93DF938C01EA
:10E9E000EB01FC01808191810097E1F068817981E0
:10E9F00061157105A9F0428153812C813D81421737
:10EA0000530770F00E940EB18C819D81F8019583AF
:10EA100084831D821C82DF91CF911F910F910895F5
:10EA20000E9454AF88819981F801918380838A8103
:10EA30009B81938382838C819D81958384831982BA
:10EA400018821B821A82E5CFFC0180819181009798
:10EA500011F00C9454AF0895EF92FF920F931F930F
:10EA6000CF93DF93CDB7DEB7A1970FB6F894DEBF93
:10EA70000FBECDBF7C01CB01BA01F701118210821C
:10EA8000138212821582148242E0420F8E010F5FC0
:10EA90001F4F0E94AAA2009789F0BC01C7010E94E3
:10EAA0000773A1960FB6F894DEBF0FBECDBFDF91FE
:10EAB000CF911F910F91FF90EF900895C7010E9491
:10EAC000BE70EFCF0F931F93CF93DF93CDB7DEB719
:10EAD000A2970FB6F894DEBF0FBECDBF8C01CB015D
:10EAE000BA01F801118210821382128215821482F7
:10EAF00030E0AE014F5F5F4F0E94BEA4BE016F5F6A
:10EB00007F4FC8010E940773A2960FB6F894DEBF2C
:10EB10000FBECDBFDF91CF911F910F910895CF937D
:10EB2000DF931F921F92CDB7DEB7FC0111821082D6
:10EB3000138212821582148269831A82BE016F5F6A
:10EB40007F4F0E9407730F900F90DF91CF91089530
:10EB5000FC011182108213821282158214820C949D
:10EB6000EB74FC01118210821382128215821482CE
:10EB70000C94AF74FC0111821082138212821582F0
:10EB800014820C94D474FC011182108213821282BC
:10EB9000158214826115710551F0FB01019000206E
:10EBA000E9F73197AF01461B570B0C94D0700895CD
:10EBB000AF92BF92CF92DF92EF92FF920F931F938B
:10EBC000CF93DF936C015B017A018901241735072C
:10EBD00020F48F2D7901042F182F63EC78E0C60103
:10EBE0000E94C375D5011496CD91DC91EC16FD06FB
:10EBF000E0F40C171D0708F4E801D501ED91FC9134
:10EC00001197EC0FFD1F108110826D917C916E0D9C
:10EC10007F1DC60161157105A1F00E940773F50102
:10EC200080819181C80FD91F1883C601DF91CF91D0
:10EC30001F910F91FF90EF90DF90CF90BF90AF901A
:10EC400008950E94BE70EBCFFB0101900020E9F710
:10EC50003197AF01461B570BDC01ED91FC9102800F
:10EC6000F381E02D19948F929F92AF92BF92EF9211
:10EC7000FF920F931F93CF93DF93CDB7DEB7A1978A
:10EC80000FB6F894DEBF0FBECDBF7C01FA01CB01F9
:10EC900019A2223008F42AE08E010F5D1F4F822E48
:10ECA000912CB12CA12CBF01A50194010E94F3ACC1
:10ECB000F901CA016A300CF5605DD8016E938D01CF
:10ECC000232B242B252B79F790E080E0109721F05F
:10ECD000BD01C7010E942476A1960FB6F894DEBF4D
:10ECE0000FBECDBFDF91CF911F910F91FF90EF909D
:10ECF000BF90AF909F908F900895695CDECFCF93C7
:10ED0000DF93482F50E070E060E020E18CE39DE06D
:10ED10000E943376EC0163EC79E08CE39DE00E9485
:10ED200024768C0F9D1FDF91CF9108958F929F9233
:10ED3000AF92BF92CF92DF92EF92FF920F931F9309
:10ED4000CF93DF937C01EB016C0182E0C80ED11CF4
:10ED50004701E5E08E0E911C10E000E0F6014191C4
:10ED60006F0150E070E060E02AE0CE010E9433764F
:10ED70005C01E881F9810190F081E02D6EE2CE0125
:10ED800019958A0D9B1D080F191FC814D90431F756
:10ED9000F701458150E070E060E02AE0CE010E947A
:10EDA0003376800F911FDF91CF911F910F91FF90CC
:10EDB000EF90DF90CF90BF90AF909F908F9008958D
:10EDC0000F931F93CF93DF93EC010E9424768C0165
:10EDD00063EC79E0CE010E942476800F911FDF91D1
:10EDE000CF911F910F9108956115710511F00C9449
:10EDF000247690E080E00895DB0114964D915C91BB
:10EE000015976D917C91DC01ED91FC910280F3816D
:10EE1000E02D19940F931F93CF93DF93EC010E9481
:10EE2000FC768C0163EC79E0CE010E942476800FA1
:10EE3000911FDF91CF911F910F910895EF92FF9253
:10EE40000F931F93CF93DF938C017B01D0E0C0E041
:10EE5000F701EC0FFD1F6491662361F0D801ED917D
:10EE6000FC910190F081E02DC8011995892B11F0DA
:10EE70002196EECFCE01DF91CF911F910F91FF90A0
:10EE8000EF900895DC0187E194E08D939D9384E0F9
:10EE9000FB0101900D928A95E1F708951F920F9260
:10EEA0000FB60F9211240BB60F922F933F934F93EF
:10EEB0005F936F937F938F939F93AF93BF93EF93E2
:10EEC000FF938FE99CE00E94396EFF91EF91BF9113
:10EED000AF919F918F917F916F915F914F913F91F2
:10EEE0002F910F900BBE0F900FBE0F901F90189593
:10EEF0001F920F920FB60F9211240BB60F922F9301
:10EF00008F939F93EF93FF93E091AF0CF091B00C30
:10EF10008081E091B50CF091B60C82FD1DC090810E
:10EF20008091B80C8F5F8F732091B90C821741F0DC
:10EF3000E091B80CF0E0E156F34F958F8093B80C58
:10EF4000FF91EF919F918F912F910F900BBE0F909A
:10EF50000FBE0F901F9018958081F2CF1F920F92D5
:10EF60000FB60F9211240BB60F922F933F934F932E
:10EF70005F936F937F938F939F93AF93BF93EF9321
:10EF8000FF938CE39DE00E94396EFF91EF91BF915A
:10EF9000AF919F918F917F916F915F914F913F9131
:10EFA0002F910F900BBE0F900FBE0F901F901895D2
:10EFB0001F920F920FB60F9211240BB60F922F9340
:10EFC0008F939F93EF93FF93E0914C0DF0914D0D34
:10EFD0008081E091520DF091530D82FD1DC0908112
:10EFE0008091550D8F5F8F732091560D821741F0E0
:10EFF000E091550DF0E0E45CF24F958F8093550D54
:10F00000FF91EF919F918F912F910F900BBE0F90D9
:10F010000FBE0F901F9018958081F2CF1F93CF9352
:10F02000DF93282F30E0F901E75FF24F8491F90177
:10F03000ED53F34FD491F901E358F34FC491CC232E
:10F04000A9F0162F81110E94F56EEC2FF0E0EE0F63
:10F05000FF1FE75BF34FA591B4918FB7F894EC9144
:10F06000111108C0D095DE23DC938FBFDF91CF91C3
:10F070001F910895DE2BF8CFAF92BF92CF92DF920F
:10F08000EF92FF920F931F93CF93DF936B017A015F
:10F09000EC01C25DDC4E28813CE0389F8001399F45
:10F0A000100D1124A090ED15B12C27FF1FC0FB01FE
:10F0B0001182108288818F5F888388819801280F50
:10F0C000311D87FD3A95F6012A153B051CF4888110
:10F0D0008C30C4F180819181049680349C4908F47D
:10F0E00073C0F60180819181049670C08881980177
:10F0F000280F311D87FD3A952A153B05DCF68881DE
:10F10000A801480F511D87FD5A95FA01EE0FFF1F08
:10F11000E40FF51FE25CF14F808186FFCBCF888141
:10F12000F801E80FF11D87FDFA95CF01EE0FFF1FE3
:10F13000E80FF91FE25CF14F808160E08F730E945D
:10F140000E78B8CF808191812881A801420F511D8E
:10F1500027FD5A959A01FA01EE0FFF1FE20FF31FE8
:10F16000E25CF14F21813281820F931FF70191837D
:10F17000808388819801280F311D87FD3A95F90118
:10F18000EE0FFF1FE20FF31FE25CF14F808186FF5D
:10F1900022C08881080F111D87FD1A95F801EE0F16
:10F1A000FF1FE00FF11FE25CF14F808161E08F7380
:10F1B000DF91CF911F910F91FF90EF90DF90CF9053
:10F1C000BF90AF900C940E7880E49CE9F701918396
:10F1D00080838FEF8883DF91CF911F910F91FF90F4
:10F1E000EF90DF90CF90BF90AF9008951092950C64
:10F1F00081E08093940C10926F0C61E084E10E9496
:10F200000E7861E085E10E940E78E9EBF0E0808104
:10F210008E7F808380818D7F808388E48093B80097
:10F2200085E48093BC0008951092550C1092540C04
:10F2300010929C0C10929E0C0E94F67888EB9DE632
:10F24000909344138093431389EB9DE6909342136C
:10F25000809341130895CF93DF9390E0FC01ED5329
:10F26000F34F24918358934FFC0184918823D1F06C
:10F2700090E0880F991FFC01E15DF34FA591B491D7
:10F28000FC01E75BF34FC591D49161110EC09FB7AC
:10F29000F8948C91E22FE0958E238C932881E223C1
:10F2A000E8839FBFDF91CF9108958FB7F894EC91D9
:10F2B000E22BEC938FBFF6CF3FB7F89480913713D2
:10F2C00090913813A0913913B0913A1326B5A89BA9
:10F2D00005C02F3F19F00196A11DB11D3FBFBA2FE8
:10F2E000A92F982F8827BC01CD01620F711D811DA8
:10F2F000911D42E0660F771F881F991F4A95D1F72D
:10F3000008958F929F92AF92BF92CF92DF92EF9229
:10F31000FF926B017C010E945C794B015C01C1147E
:10F32000D104E104F104B9F00E945C79681979090B
:10F330008A099B09683E73408105910580F321E0AD
:10F34000C21AD108E108F10888EE880E83E0981E01
:10F35000A11CB11CE4CFFF90EF90DF90CF90BF9045
:10F36000AF909F908F900895AF92BF92CF92DF920F
:10F37000EF92FF920F931F93CF93DF93C82FD62F57
:10F3800010927311109274111092751110927611DF
:10F390001092771161E00E942B7960E08C2F0E941F
:10F3A0000E786D2F70E090E080E00E94817960E03F
:10F3B0008C2F0E942B798BE990E00197F1F700E9FF
:10F3C00011E08C2F0E945C6F892B81F40150110990
:10F3D000C1F78EEF9FEFDF91CF911F910F91FF90BB
:10F3E000EF90DF90CF90BF90AF90089500E911E0CB
:10F3F0008C2F0E945C6F019721F401501109C1F715
:10F40000E8CF18E2D0E800E090E9E92EFF24F39479
:10F410008C2F0E945C6F892B29F481E0E81AF10897
:10F42000B9F7D7CF0E945C796B017C0180E9A82EE7
:10F43000BB24B3948C2F0E945C6F019729F481E068
:10F44000A81AB108B9F7C5CF0E945C796C197D097B
:10F450008E099F09693271058105910538F0E02F09
:10F46000F0E0E559FE4E80858D2B8087D69511F40E
:10F470000F5FD0E8115041F690E080E0ACCF2FB79D
:10F48000F8946091331370913413809135139091F7
:10F4900036132FBF0895CF92DF92EF92FF92CF9352
:10F4A000DF938091EA0E843051F4CFEFDFEFCE018D
:10F4B000DF91CF91FF90EF90DF90CF900895E09192
:10F4C0000D0FE1113EC00E943F7A6B017C0128EED6
:10F4D000C20E23E0D21EE11CF11C8EED9EE00E94C4
:10F4E000AE0C882311F38091430F882331F0809173
:10F4F0000E0F90910F0F892BC1F28EED9EE00E94AE
:10F500007F0BEC01CF3FDC0771F08091430F882324
:10F5100071F280910E0F90910F0F019790930F0F42
:10F5200080930E0FC4CF0E943F7AC616D706E80616
:10F53000F90698F610920D0F8EED9EE00E9459127A
:10F54000B6CFE150E0930D0FF0E0EC52F14FC18DDA
:10F55000D0E0ADCF0F931F93CF93DF93EC018C01DD
:10F56000F80181918F018823A1F10E944B7AF80163
:10F570002291022E000C330B8217930789F38F3FE1
:10F58000980781F0A0910D0F91E09A0F90930D0FC5
:10F59000B0E0AC52B14F59968C93903219F48FE190
:10F5A00080930D0F2FE1EC17FD07C9F092919F3F5B
:10F5B000D1F3A0910D0F81E08A0F80930D0FB0E081
:10F5C000AC52B14F59969C93803269F720930D0F3E
:10F5D000EACF81E0DF91CF911F910F91089580E0F4
:10F5E000F9CF1F920F920FB60F9211242F933F93D2
:10F5F0008F939F93AF93BF93809133139091341364
:10F60000A0913513B09136133091321323E0230FBC
:10F610002D3758F50196A11DB11D2093321380930B
:10F62000331390933413A0933513B0933613809112
:10F63000371390913813A0913913B0913A13019672
:10F64000A11DB11D8093371390933813A0933913E4
:10F65000B0933A13BF91AF919F918F913F912F91AA
:10F660000F900FBE0F901F90189526E8230F02965B
:10F67000A11DB11DD2CF1F920F920FB60F92112470
:10F680000BB60F922F933F934F935F936F937F939C
:10F690008F939F93AF93BF93EF93FF9348E251E013
:10F6A00064E271E090E080E00E943C78FF91EF918D
:10F6B000BF91AF919F918F917F916F915F914F918A
:10F6C0003F912F910F900BBE0F900FBE0F901F9088
:10F6D00018951F920F920FB60F9211240BB60F922E
:10F6E0002F933F934F935F936F937F938F939F934A
:10F6F000AF93BF93EF93FF9348EA50E064EA70E062
:10F7000083E090E00E943C78FF91EF91BF91AF9130
:10F710009F918F917F916F915F914F913F912F9129
:10F720000F900BBE0F900FBE0F901F9018951F9259
:10F730000F920FB60F9211240BB60F922F933F9397
:10F740004F935F936F937F938F939F93AF93BF93E9
:10F75000EF93FF9348E950E064E970E082E090E0C5
:10F760000E943C78FF91EF91BF91AF919F918F9153
:10F770007F916F915F914F913F912F910F900BBEB1
:10F780000F900FBE0F901F9018951F920F920FB6FB
:10F790000F9211240BB60F922F933F934F935F93C9
:10F7A0006F937F938F939F93AF93BF93EF93FF9349
:10F7B00048E850E064E870E081E090E00E943C7826
:10F7C000FF91EF91BF91AF919F918F917F916F9139
:10F7D0005F914F913F912F910F900BBE0F900FBEF5
:10F7E0000F901F90189560932A1370932B1380939A
:10F7F0002C1390932D13645D7E4F8F4F9F4F60931A
:10F80000261370932713809328139093291382E073
:10F8100090E090932513809324130E943F7A609385
:10F820002013709321138093221390932313089530
:10F83000CF92DF92EF92FF920F931F930E943F7A35
:10F840008B019C01C0902013D0902113E0902213D3
:10F85000F090231360912A1370912B1380912C1335
:10F8600090912D130C191D092E093F09083E1340D4
:10F8700021053105E0F0DC01CB010196A11DB11D90
:10F8800080932A1390932B13A0932C13B0932D13D2
:10F89000B701A60148515C4F6F4F7F4F4093201333
:10F8A000509321136093221370932313C7CF1F919A
:10F8B0000F91FF90EF90DF90CF900895CF93DF935B
:10F8C000EC010E94187C9E01220F331F220F331F70
:10F8D000F901E152FD4F6083718382839383CE01EE
:10F8E000880F991FFC01E952FD4F40815181141688
:10F8F000150644F4FC01E153FD4F4081518114167B
:10F90000150614F1FC01E952FD4F41E050E051832E
:10F91000408381539D4FFC015183408321543D4FCF
:10F9200088E097E0A0E0B0E0F90180839183A283B2
:10F93000B383CE010E94FD1464EF71E080E090E09B
:10F94000DF91CF910C948179DF91CF9108954F92FF
:10F950005F926F927F928F929F92AF92BF92CF925F
:10F96000DF92EF92FF920F931F93CF93DF934B01A0
:10F970005C0180911C1390911D13A0911E13B091F6
:10F980001F1388159905AA05BB0509F4C6C08CE3A9
:10F99000C82ED12CE12CF12CC501A70196010E94A3
:10F9A000F3AC6093210CCA01B901A70196010E9432
:10F9B000F3AC6093220CC501B40120E13EE040E0CD
:10F9C00050E00E94F3ACCA01B90128E130E040E008
:10F9D00050E00E94F3AC6093230CC501B40120E811
:10F9E00031E541E050E00E94F3AC69017A01CA01BF
:10F9F000B9016C5F7F4F8F4F9F4F27E030E040E0B1
:10FA000050E00E94F3AC6F5F6093240C412C512CAA
:10FA1000320140E004E610E0C0E9D1E0242F30E0FC
:10FA20002E54384FF901E370FF273097F9F4C901DC
:10FA3000B8010E9481AE892B31F4C901BE010E9438
:10FA400081AE892B99F48EE691E0A0E0B0E0480EFB
:10FA5000591E6A1E7B1ED301C201AA27BB27C816E6
:10FA6000D906EA06FB0638F04F5FD8CF8DE691E065
:10FA7000A0E0B0E0ECCF4093270CC90164E670E051
:10FA80000E9481AEEC01C90160E971E00E9481AE83
:10FA9000309721F42097D9F40097C9F04DE651E052
:10FAA00060E070E0441A550A660A770AC418D5085F
:10FAB000E608F708A5E3B3E020E0213069F43097C9
:10FAC000E9F5209711F40097C9F54DE106C04EE61F
:10FAD00051E060E070E0E6CF4C9150E070E060E013
:10FAE00031E0320FC416D506E606F70640F0C41A18
:10FAF000D50AE60AF70A1196232F3C30F1F62F5F5C
:10FB00002093260CC394C092250C80921C139092D3
:10FB10001D13A0921E13B0921F13DF91CF911F915E
:10FB20000F91FF90EF90DF90CF90BF90AF909F909C
:10FB30008F907F906F905F904F9008954CE1CDCF64
:10FB40000E94187C0E94A77C8091270C90E08E5424
:10FB5000984F08950E94187C0E94A77C8091260CE3
:10FB600090E008950E94187C0E94A77C8091250C4B
:10FB700090E008950E94187C0E94A77C8091220C3E
:10FB800090E008950E94187C0E94A77C8091230C2D
:10FB900090E008951F920F920FB60F9211240BB6AA
:10FBA0000F922F933F934F935F936F937F938F9316
:10FBB0009F93AF93BF93EF93FF9380914C120E945A
:10FBC0005C6F20914F12309150122F5F3F4F309356
:10FBD000501220934F1290914E12953618F096E0E5
:10FBE00090934B1290914B12943009F46EC0F8F43C
:10FBF000923031F1933009F44CC090914D12992319
:10FC000019F0811171C02F9AFF91EF91BF91AF91BF
:10FC10009F918F917F916F915F914F913F912F9124
:10FC20000F900BBE0F900FBE0F901F901895953040
:10FC300009F457C0963009F791E090931B134FC019
:10FC40008111DBCF20914F123091501224363105B3
:10FC500028F41092501210924F12CFCF10921B1313
:10FC600010924E12E0914E1291E09E0F90934E1220
:10FC7000F0E020914F1230915012EE0FFF1FEF5A1B
:10FC8000FD4E318320831092501210924F1293E058
:10FC900019C0813009F0B1CFE0914E1291E09E0F72
:10FCA00090934E12F0E020914F1230915012EE0FCF
:10FCB000FF1FEF5AFD4E3183208310925012109295
:10FCC0004F1294E090934B1298CF882359F22091D1
:10FCD0004F12309150122536310508F48ECF95E041
:10FCE000F1CF81118ACFB5CF2F988ECFCF93DF93ED
:10FCF00091E0909307128823B9F0C091B800D09199
:10FD0000BA008091BC008A7B8093BC0060E084E1F3
:10FD10000E940E7860E085E10E940E780E94F678DD
:10FD2000D093BA00C093B800DF91CF9108958F921D
:10FD30009F92AF92BF92CF92DF92EF92FF920F937A
:10FD40001F93CF93DF93D0919E0CD13208F0D7C090
:10FD5000182FC0919D0C0E945C796B017C018091F1
:10FD6000950C81116BC082E08093950C1093940CDC
:10FD70008FEF8093930C1092920CD093910CAFEA7A
:10FD8000B5E1E1E7FCE080E0D81391C01092700C7F
:10FD90008091700CCC0FC82BC093700C80916F0CAD
:10FDA000813009F088C010926F0C0E945C796B0161
:10FDB0007C018091700C8093BB008091970C909196
:10FDC000980CA091990CB0919A0C892B8A2B8B2BB3
:10FDD000A1F00E945C790091970C1091980C2091F1
:10FDE000990C30919A0C6C197D098E099F090617A0
:10FDF00017072807390708F442C08091BC0083FD2B
:10FE0000D8CF85EC8093BC000E945C796B017C01AB
:10FE10008091950C823009F450C08091930C8F3FF3
:10FE200009F46FC08091930C803209F46CC080910A
:10FE3000930C803309F469C084E026C08091970C4C
:10FE40009091980CA091990CB0919A0C892B8A2BC7
:10FE50008B2B09F484CF0E945C798090970C909052
:10FE6000980CA090990CB0909A0C6C197D098E0991
:10FE70009F0986169706A806B90608F070CF8091EC
:10FE8000960C0E94767E85E010929C0C10929E0C3F
:10FE900010929B0CDF91CF911F910F91FF90EF90EB
:10FEA000DF90CF90BF90AF909F908F9008959D91DD
:10FEB00091938F5F69CF85EEA5CF8091970C90913C
:10FEC000980CA091990CB0919A0C892B8A2B8B2BB2
:10FED00009F49ECF0E945C790091970C1091980CC8
:10FEE0002091990C30919A0C6C197D098E099F090B
:10FEF000061717072807390708F08ACFC0CF81E017
:10FF0000C3CF80E0C1CF82E0BFCF83E0BDCFFC0193
:10FF1000248131E030939B0C20939D0C10929C0C1B
:10FF200010929E0C8385682B89ED9DE00E940370E2
:10FF300081E00C94977E0F931F93CF938C01C62F73
:10FF40000E94877F6C2F6460C8010E94877F6C2F9E
:10FF50006B7FC8010E94877F83EC90E00197F1F7E7
:10FF6000CF911F910F910895CF93C82F682F607F75
:10FF70008FEE91E10E949B7F80E1C89FB001112428
:10FF80008FEE91E1CF910C949B7FCF93DF9300D0C4
:10FF900000D01F921F92CDB7DEB798E0EBE2F3E0FE
:10FFA000DE01119601900D929A95E1F79091F8116A
:10FFB000961708F46FEF70E0660F771F21E030E0CE
:10FFC0002C0F3D1F620F731FFB019081890F80680A
:10FFD00028960FB6F894DEBF0FBECDBFDF91CF914C
:10FFE0000C94B47F0F931F93CF938C01C62F607F27
:10FFF00061600E949B7F80E1C89FB0011124616015
:020000021000EC
:10000000C8010E949B7F81E090E0CF911F910F91EA
:10001000089585ED8093BC008091970C9091980C89
:10002000A091990CB0919A0C0796A11DB11D23E0E7
:10003000B695A795979587952A95D1F72091BC00FD
:1000400024FD03C01092950C08954091970C509197
:10005000980C6091990C70919A0C452B462B472B6C
:1000600069F30097A105B10541F025E32A95F1F761
:1000700000000197A109B109E1CF8091960C0C9481
:10008000767E1F920F920FB60F9211240BB60F922D
:100090002F933F934F935F936F937F938F939F9390
:1000A000AF93BF93EF93FF938091B900887F803621
:1000B00009F44DC008F040C0883209F4A9C028F501
:1000C000803109F49DC0C8F4882309F4FBC088304E
:1000D00009F496C0FF91EF91BF91AF919F918F91DD
:1000E0007F916F915F914F913F912F910F900BBE38
:1000F0000F900FBE0F901F901895883109F488C09B
:10010000803241F78093930C14C0803409F49DC071
:1001100040F48033B9F38833E9F68093930C85EC8F
:10012000B0C0803509F485C0883509F496C088349C
:1001300089F60E940980CECF883909F48CC038F541
:10014000883729F050F4883611F0803719F683E0AB
:100150008093950C10924A1257C0883809F47BC0DE
:10016000803919F0803809F0B5CF80914A12803279
:1001700008F071C0E0914A1281E08E0F80934A121C
:100180008091BB00F0E0E65DFD4E80833DC0803B8A
:1001900039F0E0F4803A09F479C0883A09F09ACF4E
:1001A00084E08093950C1092291210922812E0910D
:1001B0004313F091441319958091281281110FC0B7
:1001C00081E0809328121092081209C0803C09F443
:1001D000A6CF883C09F4A3CF883B09F07BCFE09100
:1001E000291281E08E0F80932912F0E0E85FFD4E26
:1001F00080818093BB00909129128091281229C0A0
:100200008091700C8093BB0085EC8093BC0062CF22
:100210009091920C8091910C981758F5E091920C66
:1002200081E08E0F8093920CF0E0EF58F34F8081C5
:10023000E9CFE091920C81E08E0F8093920C809137
:10024000BB00F0E0EF58F34F80839091920C8091C7
:10025000910C9817C8F285E8D8CFE091920C81E014
:100260008E0F8093920C8091BB00F0E0EF58F34F1B
:1002700080838091940C81115CCF81E080936F0C1E
:1002800084EA8093BC001092950C24CF85EC809377
:10029000BC001092950C80914A12803230F4E091AB
:1002A0004A12F0E0E65DFD4E108260914A1270E065
:1002B000E0914113F09142138AE292E11995109274
:1002C0004A1208CF1092930C34CFCF93DF93EC01F6
:1002D00080910112811109C081E080930112809107
:1002E000E50D9091E60D0E94E50960E08C81DF91BB
:1002F000CF910C940E7861E0FC0184810E940E780D
:1003000080910112882321F0109201120C94E409CB
:1003100008958FEF0C9477090F931F93CF93DF937A
:10032000EC010E943F7A8B010E9489818F3F69F026
:100330000E943F7A601B710B6C177D07A8F380E069
:10034000DF91CF911F910F91089581E0F9CF8F92A6
:100350009F92AF92BF92FF920F931F93CF93DF9321
:10036000EC01F62E49015A018E81882389F08F8194
:1003700098859C012F5F3F4F38872F8382309240B2
:1003800018F40E948981F3CFCE010E947B811E82E6
:10039000CE010E9465818CE291E00E948C818F2DBC
:1003A00080640E94770908E110E0D501C401002EA5
:1003B00004C0B695A795979587950A94D2F70E94A1
:1003C000770908501109083F8FEF180771F785E981
:1003D000FF2021F028E087E8F2128FEF0E947709D2
:1003E00010E00E9489818A8787FF04C01F3F11F0B7
:1003F0001F5FF7CFDF91CF911F910F91FF90BF90BB
:10040000AF909F908F900895AF92BF92CF92DF925E
:10041000EF92FF920F931F93CF93DF93EC0169014B
:10042000C801820F931F8130924050F58E8188233E
:1004300079F088819981AA81BB8184179507A607E5
:10044000B70731F48F819885C816D90608F042C0E5
:10045000488359836A837B838B85833039F089E0B5
:10046000440F551F661F771F8A95D1F79A01AB017C
:1004700061E1CE010E94A781882389F083E08D830A
:10048000CE010E947B8180E0DF91CF911F910F917F
:10049000FF90EF90DF90CF90BF90AF9008950E94B3
:1004A0003F7A5B010E9489818A878F3F69F40E94AD
:1004B0003F7A6A197B096D327140A0F38FE08D831A
:1004C000CE010E947B81DCCF8E3F89F418861F828B
:1004D00081E08E838F8198858C159D0550F40E9454
:1004E00089818F819885019698878F83F3CF8DE0DE
:1004F000E6CF6701E00EF11E0E948981F60181932B
:100500006F01EE15FF05C1F78F819885080F191F40
:1005100018870F838985882319F001151240A0F0F0
:100520008E81882389F08F8198859C012F5F3F4FB2
:1005300038872F838230924018F40E948981F3CF4C
:10054000CE010E947B811E8281E09ECFEF92FF92BE
:100550000F931F93CF93DF93EC01790182E1411553
:1005600051056105710599F08B85833039F089E07B
:10057000440F551F661F771F8A95D1F79A01AB016B
:1005800068E1CE010E94A781882319F084E08D8361
:1005900030C08EEF0E94770987018EEFF81AF801BC
:1005A00081918F010E9477090E151F05C1F78FEF0A
:1005B0000E9477098FEF0E9477090E9489818A87BC
:1005C0008F71853089F488E592E00E948C818823C0
:1005D000A9F020E030E0A9016DE0CE010E94A781E2
:1005E000882371F084E1D3CF81E18D83CE010E9415
:1005F0007B81CE010E947B8180E00AC085E1C7CF6C
:100600000E9489818111EECFCE010E947B8181E021
:10061000DF91CF911F910F91FF90EF900895CF93AD
:10062000DF93809102128823A9F1C0914515D091E2
:10063000461540916A0250916B0260916C02709174
:100640006D0225E433E1CE010E94A682811104C02F
:1006500080E0DF91CF9108954091031250910412F0
:1006600060910512709106124115510561057105E1
:1006700079F025E433E1CE010E94A682882341F37C
:100680001092031210920412109205121092061288
:100690001092021281E0DDCF8F929F92AF92BF92B3
:1006A000EF92FF920F931F93CF934B015C01C42FE6
:1006B00080916A0290916B02A0916C02B0916D02E0
:1006C00088159905AA05BB0549F10E940F83811180
:1006D0000BC080E0CF911F910F91FF90EF90BF90E2
:1006E000AF909F908F90089585E4E82E83E1F82ED7
:1006F00000E012E030E020E0B501A4018091451552
:10070000909146150E940482882319F380926A0210
:1007100090926B02A0926C02B0926D024091021214
:100720004C2B4093021281E0D5CF8F929F92AF92D3
:10073000BF92CF92DF92EF92FF92CF9327EE3DE0F0
:100740003093461520934515882309F46DC040E089
:1007500060E070E0CB010E944C8381110BC080E00F
:10076000CF91FF90EF90DF90CF90BF90AF909F9090
:100770008F900895809103158F7789F780910F15D9
:1007800090911015A0911115B09112158436910514
:10079000A105B10520F3C0900B15D0900C15E09089
:1007A0000D15F0900E15C114D104E104F104B9F255
:1007B00040E0C701B6010E944C83882381F28091FA
:1007C0005013909151138115924049F6A091551301
:1007D000AA2329F260915313709154136115710586
:1007E00009F4BDCF20915213222309F4B8CFA0936E
:1007F000050E2093F70D90E080E030E0E1E0F0E0BE
:10080000C82FAF01082E02C0440F551F0A94E2F70B
:100810002417350769F041E0480F019689309105AA
:1008200079F74093000E9BCFC12CD12C7601C0CF1D
:100830008093000E20915B1330915C1350E040E0F8
:100840002115310541F42091691330916A134091CB
:100850006B1350916C132093F80D3093F90D409366
:10086000FA0D5093FB0D46015701860E971EA11CF1
:10087000B11C8092060E9092070EA092080EB092C4
:10088000090EE0915613F0915713F0930C0EE0937C
:100890000B0EB0E00E9434ADDC01CB01880D991D38
:1008A000AA1DBB1D80930D0E90930E0EA0930F0EEC
:1008B000B093100E25E0EE0FFF1F2A95E1F7E150EF
:1008C000FE4FEF2FFF27E6958E0F9F1FA11DB11D35
:1008D0008093010E9093020EA093030EB093040E2A
:1008E0008090581390905913B12CA12C811491042D
:1008F00041F48090651390906613A0906713B090B8
:100900006813C81AD90AEA0AFB0AC80CD91CEA1CDF
:10091000FB1C04C0F694E794D794C794CA95D2F709
:10092000C092FC0DD092FD0DE092FE0DF092FF0DF5
:1009300085EFC8168FE0D806E104F10428F48CE0B6
:1009400080930A0E81E00CCF80E125EFC2162FEFD5
:10095000D206E104F104A0F3809171139091721317
:10096000A0917313B091741380930D0E90930E0E9B
:10097000A0930F0EB093100E80E2E2CF4F925F92E1
:100980006F927F928F929F92AF92BF92CF92DF929F
:10099000EF92FF920F931F93CF93DF93EC014230BE
:1009A00051056105710590F480E0DF91CF911F91B1
:1009B0000F91FF90EF90DF90CF90BF90AF909F90FE
:1009C0008F907F906F905F904F90089589859A8562
:1009D000AB85BC850196A11DB11D84179507A6079F
:1009E000B70710F3CB88DC88ED88FE888F898031CB
:1009F00009F042C0BB27A72F962F852F4801590128
:100A00002A013B01C80ED91EEA1EFB1E80916A0214
:100A100090916B02A0916C02B0916D02C816D9063C
:100A2000EA06FB0699F58F898031C1F5B301A20171
:100A3000552766277727440F551F4B5B5C4EFA01FD
:100A400091828082809102128160809302128A8951
:100A5000823080F08D819E81AF81B8858C0D9D1D87
:100A6000AE1DBF1D8093031290930412A093051234
:100A7000B093061281E099CFDB01CA01E7E0B69599
:100A8000A79597958795EA95D1F7B8CF40E0C7012C
:100A9000B6010E944C838111C6CF86CFB301A2015B
:100AA0004F77552766277727440F551F440F551F4B
:100AB0004B5B5C4EFA0180829182A282B382C2CFEC
:100AC0008F929F92AF92BF92CF92DF92EF92FF925E
:100AD0000F931F93CF93DF93FC0181859285A385AC
:100AE000B4850196A11DB11D84179507A607B70708
:100AF00070F480E0DF91CF911F910F91FF90EF9004
:100B0000DF90CF90BF90AF909F908F900895838893
:100B10009488A588B6888789803189F5BB27A72F57
:100B2000962F852FE9016A017B018F01BC01CD0160
:100B3000680D791D8A1D9B1D80906A0290906B0242
:100B4000A0906C02B0906D0286169706A806B906B2
:100B500001F5F8018789803111F5DD24EE24FF24A9
:100B6000F601EE0FFF1FEB5BFC4E80819181B0E040
:100B7000A0E088839983AA83BB8381E0BBCFDB019C
:100B8000CA01C7E0B695A79597958795CA95D1F7FD
:100B9000C9CF40E00E944C838111DBCFAACFE894FB
:100BA000C7F8DD24EE24FF24F601EE0FFF1FEE0F41
:100BB000FF1FEB5BFC4E80819181A281B381BF70EE
:100BC000D8CF4F925F926F927F92AF92BF92CF92A7
:100BD000DF92EF92FF920F931F93CF93DF9300D09A
:100BE0001F92CDB7DEB78C0149835A836B837C8318
:100BF0005901C12CD12C7601412C82E0582E612C58
:100C0000712C49815A816B817C819E012F5F3F4FFE
:100C1000C8010E946085882339F1F8018585A30108
:100C2000920104C0220F331F441F551F8A95D2F72B
:100C3000DA01C901C80ED91EEA1EFB1E49815A817C
:100C40006B817C818789803111F188EF9FEFAFEF55
:100C5000BFE0481759076A077B0798F2F501C08281
:100C6000D182E282F38281E00F900F900F900F907B
:100C7000DF91CF911F910F91FF90EF90DF90CF9078
:100C8000BF90AF907F906F905F904F90089588EFE6
:100C90009FEFA0E0B0E0DDCF8F929F92AF92BF9226
:100CA000CF92DF92EF92FF920F931F93CF93DF9338
:100CB000EC018D8181110EC080E0DF91CF911F91F9
:100CC0000F91FF90EF90DF90CF90BF90AF909F90EB
:100CD0008F9008950B891C892D893E89041715076B
:100CE0002607370748F34A015B01823031F48A86D0
:100CF0009B86AC86BD8681E0E0CF81149104A1047F
:100D0000B10449F41E821F82188619861A861B8632
:100D10001C861D86F0CF0A851B852C853D85EB8DB5
:100D2000FC8D858590E00996B901A80141505109D3
:100D300061097109082E04C0769567955795479506
:100D40000A94D2F775016401E1E0CE1AD108E108F6
:100D5000F10804C0F694E794D794C7948A95D2F723
:100D6000C416D506E606F70620F0012B022B032B4E
:100D700011F58F89988DA98DBA8D8E839F83A88751
:100D8000B9878E010A5F1F4FC114D104E104F10439
:100D900009F4ADCF4E815F816885798598018B8D8F
:100DA0009C8D0E94608591E0C91AD108E108F10884
:100DB0008111EACF81CFC41AD50AE60AF70AE1CF3A
:100DC0003F924F925F926F927F928F929F92AF92DB
:100DD000BF92CF92DF92EF92FF920F931F93CF9328
:100DE000DF93CDB7DEB72C970FB6F894DEBF0FBEFA
:100DF000CDBF5C01DC015B968D909C905C97169654
:100E00004D905D906D907C90199741145104610450
:100E1000710409F468C0BFEF4B1A5B0A6B0A7B0AC6
:100E2000312CF40181859285A385B4859C01AD01A7
:100E30002F5F3F4F4F4F5F4F29873A874B875C8724
:100E4000730162011D821E821F821886F401818552
:100E50009285A385B4852D813E814F8158852817C1
:100E600039074A075B0708F056C089859A85AB8524
:100E7000BC858C159D05AE05BF0550F482E0C82EDB
:100E8000D12CE12CF12C92E0492E512C612C712CAB
:100E90009E012F5F3F4FB701A601C4010E946085EC
:100EA0008823C9F189819A81AB81BC81892B8A2BE6
:100EB0008B2B09F1260137019FEF491A590A690A5C
:100EC000790A2D813E814F8158852F5F3F4F4F4FCB
:100ED0005F4F2D833E834F8358873FEFC31AD30A5A
:100EE000E30AF30AB3CFF40140805180628073803B
:100EF0003324339496CFC414D504E604F70409F7D9
:100F00000FEF1FEF2FEF3FE0B701A601C4010E94D2
:100F1000BE84811119C080E02C960FB6F894DEBF14
:100F20000FBECDBFDF91CF911F910F91FF90EF903A
:100F3000DF90CF90BF90AF909F908F907F906F90F9
:100F40005F904F903F900895F501468157816085ED
:100F50007185411551056105710539F097018601CB
:100F6000C4010E94BE848823B1F2D5011696CD92A9
:100F7000DD92ED92FC921997332051F0D701C60112
:100F80000196A11DB11DF40180839183A283B383D7
:100F9000F5018789908DA18DB28D892B8A2B8B2BA2
:100FA00039F4C78AD08EE18EF28E84818068848382
:100FB00081E0B2CF2F923F924F925F926F927F92D9
:100FC0008F929F92AF92BF92CF92DF92EF92FF9259
:100FD0000F931F93CF93DF93EC015B012A018D8167
:100FE000811115C08FEF9FEFDF91CF911F910F916E
:100FF000FF90EF90DF90CF90BF90AF909F908F9039
:101000007F906F905F904F903F902F9008958C81CC
:1010100080FFE8CF0B891C892D893E894A855B8535
:101020006C857D85C201B0E0A0E068017901C41A39
:10103000D50AE60AF70AC816D906EA06FB0618F426
:101040002801441A550A42011E0126E0220E311CD5
:101050008114910409F4B3C04A855B856C857D8554
:101060006A0181E0D8228B8D9C8D8A019B01E9E089
:101070003695279517950795EA95D1F7ED81E230DA
:10108000E1F5FC01628D738D848D958D600F711F6C
:10109000821F931F612C22E0722E6C187D0886142B
:1010A000970408F434012C8126FD04C06114F2E099
:1010B0007F0671F400916A0210916B0220916C021C
:1010C00030916D02061717072807390709F053C03A
:1010D00040E00E944C83882309F484CFC6018B5BD7
:1010E0009C4ED5019C01260D371DFC012E173F0794
:1010F00009F460C041914D93F9CFFC0174807A945A
:101100007022C114D10471F471100CC0452B462B10
:10111000472B39F58F89988DA98DBA8D8E839F8342
:10112000A887B987EB8DFC8D6E817F818885998535
:101130006250710981099109258504C0660F771FE6
:10114000881F991F2A95D2F706851785208931892E
:10115000600F711F821F931F670D711D811D911DEF
:1011600099CF4E815F816885798591010E94608564
:101170008111D8CF37CF750183019601AB01BC0136
:1011800080914515909146150E940482882309F4A8
:1011900029CFA60CB71C8A859B85AC85BD85860D9D
:1011A000971DA11DB11D8A879B87AC87BD878618B7
:1011B00097084ECF281B390BA20EB31EECCFC201ED
:1011C00013CFCF93DF931F92CDB7DEB741E050E04E
:1011D000BE016F5F7F4F0E94DA87019731F48981EA
:1011E00090E00F90DF91CF9108958FEF9FEFF9CFAF
:1011F000FC01818D928D009711F00C94E1888FEFA6
:101200009FEF08950F931F93CF93DF93EC01898D88
:101210009A8D10E000E0009799F00E94E1888C011F
:101220000F3F100769F0898D9A8DFC014285538527
:101230006485758541505109610971090E944C8688
:10124000C801DF91CF911F910F910895CF93DF9344
:10125000EC018D81882389F18C8187FF2AC06E85FE
:101260007F858889998941E00E944C83882329F1F0
:10127000EA8980E2E89FF0011124EB5BFC4E309795
:10128000E1F08D81823040F48B899C89AD89BE89E3
:10129000848F958FA68FB78F8F89988D938F828F2C
:1012A0008F89988DA98DBA8DB58BA48B8C818F7702
:1012B0008C83DF91CF910C940F8380E0DF91CF91ED
:1012C0000895CF92DF92EF92FF921F93CF93DF9317
:1012D000EC0180E2689FF0011124EB5BFC4E9385EA
:1012E000917161F0842F827449F080E0DF91CF9199
:1012F0001F91FF90EF90DF90CF900895142F6A8B8D
:1013000080916A0290916B02A0916C02B0916D0283
:101310008E879F87A88BB98BC488D588F12CE12C48
:101320007601DD24CC24CF8AD88EE98EFA8E828D88
:10133000938DB0E0A0E0AC01BD014C295D296E2980
:101340007F294F8B588F698F7A8F83858871B1F48D
:10135000848D958DA68DB78D8B8B9C8BAD8BBE8B25
:1013600081E08D831F701C831E821F821886198660
:101370001A861B861C861D8681E0B8CF803109F055
:10138000B4CF9E012D5E3F4F8B8D9C8D0E94E185D9
:10139000882309F4AACF84E0E4CFCF93DF93EC0154
:1013A0000E942689882311F01D8281E0DF91CF9170
:1013B0000895FC01818D928D009711F00C9426897F
:1013C00008953F924F925F926F927F928F929F9279
:1013D000AF92BF92CF92DF92EF92FF920F931F9343
:1013E000CF93DF9300D000D000D01F921F92CDB7D3
:1013F000DEB77C01DC0115968C91811115C0FE01D0
:101400003196CE010C966F0130E23193E817F9075F
:10141000E1F7DA0130E087E09D91B92E992329F1B7
:101420009E3239F48A3011F480E0E3C038E08AE07B
:10143000F3CFEFE1FCE04491442321F03196941383
:10144000FACFF2CF831780F34FED490F4E3560F797
:101450004FE9490F4A3118F440EEB42EB90EF601A7
:10146000E30FF11DB0823F5FD7CF89818032E1F277
:10147000322E8B01FB01838D948DD7015C969C935A
:101480008E935B97168217821086118612861386BA
:1014900014861586F80182859385A485B5854389D0
:1014A00054896589768984179507A607B70708F0D8
:1014B0004DC025E0B695A795979587952A95D1F7C4
:1014C000F82FFF70AF2ED80115968C91823008F45A
:1014D000ABCFC8010E94E18897FDA6CFF8018285B5
:1014E0009385A485B5854F96A11DB11D82879387ED
:1014F000A487B587F0E2AF9EB00111246B5B7C4EF0
:101500006115710509F490CFDB018C91882341F0BE
:10151000853E09F061C0BB2029F0BB24B394BACF4B
:10152000B1100EC0F701A28A80916A0290916B02FD
:10153000A0916C02B0916D0286879787A08BB18BCA
:10154000DB018C918111E9CFBB24B394832D82718F
:10155000823109F069CFBB2009F463C0F7016685C9
:1015600077858089918941E00E944C83882309F422
:101570005BCFD70152968C91B0E28B9FC0011124B2
:101580008B5B9C4E009709F44FCFFC013A9626E105
:10159000DF011D922A95E9F72BE0F601DC010190AD
:1015A0000D922A95E1F721E238E2FC01318B208B84
:1015B00040E058E057874687338B228B318F208F4E
:1015C000578B468B0E940F83882309F42DCF432D20
:1015D000D70152966C910AC04BE050E0C6010E94C0
:1015E000CBB0892B09F056CF432D6A2DC7010E943D
:1015F00061892B960FB6F894DEBF0FBECDBFDF9189
:10160000CF911F910F91FF90EF90DF90CF90BF90FF
:10161000AF909F908F907F906F905F904F903F9092
:101620000895F8018581823009F4FECEC8010E9438
:10163000E086882309F4F8CED8015B96ED91FC9101
:101640005C9716968D909D90AD90BC901997B2E0E6
:101650008B1A9108A108B108858504C0880C991CD3
:10166000AA1CBB1C8A95D2F786859785A089B1896B
:10167000880E991EAA1EBB1E848124013501480EC6
:10168000511C611C711C84149504A604B70401F15B
:10169000E1E04E1A5108610871080E940F83882307
:1016A00009F4C2CEE5E4F3E1119285E495E18E17E9
:1016B0009F07D1F740926A0250926B0260926C02CF
:1016C00070926D0280910212816080930212DBCFD2
:1016D000D8015B96ED91FC91258580E092E0A0E039
:1016E000B0E004C0880F991FAA1FBB1F2A95D2F72C
:1016F000F8014389548965897689840F951FA61F4F
:10170000B71F838B948BA58BB68BD70152961C92F7
:1017100085E493E13ACF2F923F924F925F926F927E
:101720007F928F929F92AF92BF92CF92DF92EF9271
:10173000FF920F931F93CF93DF9300D01F92CDB7EB
:10174000DEB78C015B011A01DC0115968C911597AF
:10175000813009F0C8C014968C9181FFC4C082FD0D
:10176000AEC06101D8011A964D915D916D917C9149
:101770001D97C114D10409F429C15B968D919C91E8
:101780005C97FC0174802FEF270D2A013B0139E0A3
:1017900076946794579447943A95D1F7722E7420B3
:1017A0007A01F1E0FF22711020C0E114F104E9F4A4
:1017B00016964D915D916D917C911997411551054A
:1017C0006105710509F098C057968D919D910D9016
:1017D000BC91A02D0097A105B10509F0AFC0C801CB
:1017E0000E94E086882309F47EC080E092E08E1992
:1017F0009F0946018C159D0508F44C01D8015B96A4
:101800004D915C915C9716968D919D910D90BC9138
:10181000A02D0297A109B109FA01258504C0880FFE
:10182000991FAA1FBB1F2A95D2F746855785608945
:101830007189840F951FA61FB71F9C01AD01270D4D
:10184000311D411D511D29013A01811432E09306D9
:1018500009F07AC080916A0290916B02A0916C02AB
:10186000B0916D0284159505A605B70559F48FEF63
:101870009FEFDC0180936A0290936B02A0936C024D
:10188000B0936D029501B301A2018091451590912D
:1018900046150E94A682882331F19EEFB91AC81816
:1018A000D908F80182859385A485B585880D991D91
:1018B000A11DB11D82879387A487B58753CFF801F7
:1018C000438954896589768982859385A485B58500
:1018D000481759076A077B0709F443CFC8010E94DC
:1018E0004C8681113ECF81E090E0D80113969C9305
:1018F0008E93129780E007C09E012F5F3F4F0E949A
:101900006085811102C090E077C089819A81AB81A6
:10191000BC81F801238D348DF901278948EF5FEFF1
:1019200060E070E0203121F048EF5FEF6FEF7FE083
:1019300084179507A607B70708F051CFF8018683EB
:101940009783A087B18751CFE114F10491F5D801B5
:101950001A964D915D916D917C911D9753968D9145
:101960009D910D90BC91A02D481759076A077B07E0
:1019700000F10E940F83882309F4B5CF40926A02D8
:1019800050926B0260926C0270926D028091021212
:1019900081608093021297012B5B3C4ED501C901F7
:1019A000880D991DF9018E179F0759F04D914193AC
:1019B000FACF41E0C301B2010E944C838111EBCF09
:1019C00092CF821B930BA80EB91E69CFF8018389B1
:1019D0009489A589B68984179507A607B70738F4AF
:1019E0008481438B548B658B768B80688483F8016C
:1019F000848183FD18C0C1010F900F900F900F904C
:101A0000DF91CF911F910F91FF90EF90DF90CF90DA
:101A1000BF90AF909F908F907F906F905F904F900E
:101A20003F902F900895C8010E942689882309F4C9
:101A30005ACFE1CFCF93DF931F92CDB7DEB7698343
:101A400041E050E0BE016F5F7F4F0E948B8B0F9093
:101A5000DF91CF910895CF93DF93EC01E98DFA8D5B
:101A6000309749F481E090E09B838A8390E080E0A6
:101A7000DF91CF91089513821282898D9A8D0E94F1
:101A80008B8BE98DFA8D22813381232B59F7F0CF8F
:101A9000FC01DB0112968D919C91139793838283B5
:101AA00085E893E09183808314968C9114978483C6
:101AB00015968C911597858316964D915D916D9134
:101AC0007C91199746835783608771871A964D9149
:101AD0005D916D917C911D974287538764877587CF
:101AE0001E964D915D916D917C91519746875787D8
:101AF000608B718B52968C915297828B53964D913D
:101B00005D916D917C915697438B548B658B768B51
:101B100057964D915D916D917C915A97478B508F5F
:101B2000618F728F5B968D919C91948F838F0895B6
:101B3000DC015996ED91FC91309721F081E095817F
:101B4000911101C080E00895CF93DF93EC01898D5E
:101B50009A8D009741F00E94CD89898D9A8D0E94BF
:101B600054AF1A8E198EDF91CF910895EF92FF92A4
:101B70000F931F93CF93DF93EC017B018A011B82AC
:101B80001A8288EE93E0A0E0B0E08C839D83AE8360
:101B9000BF8389EF93E0998388838DE190E00E9471
:101BA000B8AE9A8F898F009779F02DE1F701DC01AB
:101BB00001900D922A95E1F74CE050E0B801CE017A
:101BC0000C960E9423B1188EDF91CF911F910F9137
:101BD000FF90EF9008952F923F924F925F926F92F5
:101BE0007F928F929F92AF92BF92CF92DF92EF92AD
:101BF000FF920F931F93CF93DF93CDB7DEB7C756F6
:101C0000D1090FB6F894DEBF0FBECDBF5C013B011A
